:100000000C94594C0C947A4C0C940BD30C947A4C61
:100010000C947A4C0C947A4C0C947A4C0C947A4C48
:100020000C947A4C0C947A4C0C947A4C0C9436D5F3
:100030000C947A4C0C947A4C0C94DFB70C947A4C58
:100040000C947A4C0C947A4C0C947A4C0C947A4C18
:100050000C947A4C0C947A4C0C947A4C0C947A4C08
:100060000C947A4C0C9425D30C94B4D20C947A4C06
:100070000C947ECC0C9420CC0C945CCC0C947A4CDC
:100080000C94D6D30C947A4C0C947A4C0C947A4CF5
:100090000C947A4C0C947A4C0C947A4C0C947A4CC8
:1000A0000C947A4C0C947A4C0C947A4C0C94BABE06
:1000B0000C945EBF0C947A4C0C947A4C0C94D0B98E
:1000C0000C947A4C0C947A4C0C947A4C0C947A4C98
:1000D0000C947A4C0C947A4C0C947A4C0C947A4C88
:1000E0000C941BAA0C947A4C0C947A4C0C947A4C79
:1000F0000C947A4C0C947A4C0C947A4C0C947A4C68
:100100000C9491BE0C9435BF0C9468BE0C940CBF3B
:100110000C947A4C0C947A4C0C947A4C0C947A4C47
:100120000C947A4C0C947A4C0C947A4C0C947A4C37
:100130000C947A4C0C9434B90C947A4C0C947A4C00
:100140000C947A4C0C947A4C0C947A4C0C947A4C17
:100150000C947A4C0C947A4C0C9411AA0C947A4C12
:100160000C947A4C0C947A4C0C947A4C0C947A4CF7
:100170000C947A4C0C947A4C0C947A4C0C947A4CE7
:100180000C947A4C0C947A4C0C947A4C0C947A4CD7
:100190000C947A4C0C947A4C0C947A4C0C947A4CC7
:1001A0000C94E3BE0C9487BF0C947A4C0C947A4C5C
:1001B0000C9482B90C947A4C0C947A4C0C947A4C32
:1001C0000C947A4C0C947A4C0C947A4C0C947A4C97
:1001D0000C947A4C0C947A4C0C947A4C0C947A4C87
:1001E0000C947A4C0C947A4C63756D7577758175A7
:1001F0008C75907B907B907B907B907B9275907BB5
:10020000907B907B907B907B907B94759E75A8757E
:10021000B275BC75907B907B907B907B907B907B44
:10022000C675907B1C76907B907B907B907B907BBF
:10023000907B907B5B76907B7779907B907B907BBB
:10024000907B907B907B907B907B7779907B907B71
:10025000907B88768D769776A176A376AD76B87604
:10026000907BC376907B907B0077907B907B907B9C
:10027000907B907B907B907B907B907B907B907B26
:10028000907B907B907B907B0A77907B907B907BA0
:10029000907B907B907B907B907B907B14775177C9
:1002A0008E77D777E177FA77FA7704780E7818782F
:1002B00022782C7831783B7845788E7B8E7B8E7BCC
:1002C0008E7B8E7B8E7B8E7B8E7B8E7B8E7B8E7BE6
:1002D0008E7B8E7B8E7B8E7B8E7B8E7B8E7B8E7BD6
:1002E0008E7B04788E7B8E7B8E7B8E7B8E7B8E7B53
:1002F0008E7B8E7B8E7B8E7B8E7B8E7B8E7B8E7BB6
:100300008E7B8E7B8E7B4F78597863786D788E7B71
:100310008E7B8E7B8E7B8E7B8E7B8E7B8E7BFA772D
:100320001B7BDC7AE07AE87AC47AC87AD07AD47A0D
:10033000F47A077B0F7B137B177B737BEC7AE8786F
:10034000F9780A79907B907B82785475907B1B7941
:100350002C793D797779EB775F79907B9378907BF7
:100360004E79A4787778907B907B907BB578C6782F
:10037000D77801BE09BE11BE19BE21BE29BE31BE4D
:1003800039BE49C1A6C0AEC0B6C0BEC0C6C0CEC090
:10039000D6C0DEC0E6C0EEC0F6C0FEC006C10EC1CB
:1003A0002EC12EC12EC12EC12EC12EC12EC12EC1D5
:1003B0002EC12EC12EC12EC12EC12EC12EC12EC1C5
:1003C0002EC12EC12EC12EC12EC12EC12EC12EC1B5
:1003D0002EC12EC12EC12EC12EC12EC12EC12EC1A5
:1003E0002EC12EC12EC116C11EC12EC12EC12EC1BD
:1003F0002EC12EC12EC12EC12EC12EC12EC12EC185
:100400002EC12EC12EC12EC12EC12EC12EC12EC174
:100410002EC12EC12EC12EC12EC12EC12EC12EC164
:100420002EC12EC12EC12EC12EC12EC12EC12EC154
:100430002EC12EC12EC12EC12EC12EC12EC12EC144
:100440002EC12EC12EC12EC126C1084AD73B3BCE9C
:10045000016E84BCBFFDC12F3D6C74319ABD5683C3
:100460003DDA3D00C77F11BED9E4BB4C3E916BAA7B
:10047000AABE000000803F05A84CCDB2D44EB938CA
:1004800036A9020C50B9918688083CA6AAAA2ABEB1
:10049000000000803F07634236B79BD8A71A39682F
:1004A0005618AEBAAB558C1D3CB7CC5763BD6DED3D
:1004B000FD753EF6177231BF000000803F08000056
:1004C00000BE922449123EABAAAA2ABECDCCCC4C87
:1004D0003E00000080BEABAAAAAA3E00000000BFFA
:1004E000000000803F0000000000084178D3BB43BB
:1004F00087D1133D190E3CC3BD4282AD2B3E68EC43
:100500008276BED98FE1A93E4C80EFFFBE01C4FFC9
:100510007F3F0000000000000C940E780C947E5B7E
:100520000C943BCB0C940A790C94C1CD0C94D27BE7
:100530000C94905B0C945F6B0C9445680C9408C50C
:100540000C947CAB0C94FA770C9445780C94A5D061
:100550000C943E5F0C94E27B0C94CCBD0C94AD7675
:100560000C9453C00C9468AB0C942AD00C94386053
:100570000C94576C0C9407B10C94165F0C9437AC28
:100580000C94965B0C941A5F0C94BC750C9409D176
:100590000C9404600C9492620C94904C0C94CECA0F
:1005A0000C94137B0C94DC7A0C942EC10C94FEC03A
:1005B0000C9459BD0C9473C00C94864C0C9429BEB9
:1005C0000C94A75B0C94FDC50C943A5E0C94E878EF
:1005D0000C944A5F0C942E5C0C947C4C0C94E66159
:1005E0000C9411840C9493780C94EEC00C9449C133
:1005F0000C940A620C94E87A0C9400680C94625E85
:100600000C942E5F0C943B780C94077B0C94D77859
:100610000C947D680C943A5F0C94CC670C94246025
:100620000C94B8760C94845B0C94C65B0C940BB160
:100630000C941B7B0C9494C00C94F3CF0C9420600E
:100640000C94795F0C9488760C9463CA0C9401BE68
:100650000C94A8750C94E75B0C94ED4F0C94365FEA
:100660000C94C75C0C94D47A0C9460AB0C94545EDC
:100670000C94C87A0C94C6C00C94715B0C94465FC1
:100680000C941C600C9481750C94435D0C94B578AB
:100690000C94B6B00C94B25B0C9451630C94C85893
:1006A0000C948E770C948A5B0C9419BE0C944E5F5C
:1006B0000C94A3760C9497670C9410600C94D0BDA6
:1006C0000C9451710C944C7D0C94005C0C94985FCC
:1006D0000C94D15B0C945A5F0C9415840C94CF4C01
:1006E0000C940FB10C940E5F0C94407D0C94047824
:1006F0000C949D5C0C9474AB0C9439BE0C94C37632
:100700000C9406C10C94F47A0C9431BE0C94F978D4
:100710000C9463B20C9426C10C9418780C94EB776B
:100720000C94A26C0C9442880C94D7770C94227889
:100730000C941C760C945B760C94CEC00C94C47A0A
:100740000C94907B0C94C87C0C948F670C94B8BD6F
:100750000C940A770C94305D0C94D4BD0C9477C043
:100760000C948F5E0C949B670C9463750C94B6C0CC
:100770000C94225F0C9497760C94286D0C9405BD14
:100780000C9470AB0C9494750C94695E0C94256772
:100790000C9484AB0C9428600C94756F0C94EC7AD8
:1007A0000C9493670C94A8CA0C949E750C940060EA
:1007B0000C94705E0C941EC10C94A4780C94166575
:1007C0000C94C6780C94E04C0C9477780C945CCB29
:1007D0000C9492750C9481BD0C9400770C94C261BA
:1007E0000C94BEC00C9411BE0C94177B0C944F78E3
:1007F0000C945BBC0C9468610C943D790C9421BE04
:100800000C94BBCB0C94BB720C946A620C942BAF0F
:100810000C9440600C942A630C94B2750C94095E9D
:100820000C9493CF0C94207E0C948B7D0C948A6353
:100830000C948C750C9467BC0C941B790C943C60E4
:100840000C9429AF0C946C620C942A5F0C94517731
:100850000C9454750C94756C0C94E8850C945F7929
:100860000C94F6C00C94AEC00C9420C50C94A6C099
:100870000C941B7D0C94E1770C9454D20C94487D1D
:100880000C94737B0C9407C50C94AE5E0C94C675E7
:100890000C9431620C9401630C9493CE0C94CA7D39
:1008A0000C940EC10C94F1BC0C94CDCB0C948E7BAB
:1008B0000C94207D0C9427AF0C941FBD0C9477757D
:1008C0000C94B7620C94665C0C940A5F0C94BE6145
:1008D0000C9431780C940D840C943A670C9403B109
:1008E0000C94125F0C948D760C9461AF0C944C6058
:1008F0000C94E26B0C941E5F0C9463AF0C945760E5
:100900000C9482780C94D6C00C94E6670C94325FF9
:100910000C9459C50C94D7660C94B0BD0C948B679D
:100920000C94B4BD0C94DC620C94525F0C94BB5BD1
:100930000C94DC5B0C94FD720C9463780C947796A9
:100940000C944E790C94CBB00C942C600C94B15D4B
:100950000C9416C10C94447D0C949C5B0C94286CF4
:100960000C9464AB0C947D6F0C94425F0C946CAB54
:100970000C94E6C00C942C790C94D8BD0C942C7873
:100980000C9480AB0C94BDBD0C94A1760C94E07AD1
:100990000C9477790C9409BE0C9434720C94B5685D
:1009A0000C94DEC00C943CC50C945C530C944F72B8
:1009B0000C9434600C940C600C94BB5F0C94265F18
:1009C0000C9459780C94355E0C94565F0C9414601A
:1009D0000C949E830C946D780C9430600C949C5F06
:1009E0000C9414770C946D750C941A680C94175C25
:1009F0000C94D07A0C9478AB0C94E7B00C94B76C50
:100A00000C943AB20C940F7B0C9418600C94086010
:100A10000C94507D0C9467AF0C94005D0C9427CF20
:100A20000C94F57D0C945B5E0C9459C00C9473BCD3
:100A30005B257325735D20257320257320706F73EC
:100A40006974696F6E2531382E336625730A005B31
:100A5000257325735D202573202573206F666673CB
:100A600065742532302E336625730A005B257325A5
:100A7000735D202573207A65726F206261636B6FEE
:100A800066662531392E336625730A005B2573258A
:100A9000735D202573206C61746368206261636BF1
:100AA0006F66662531382E336625730A005B257321
:100AB00025735D202573206C617463682076656CF6
:100AC0006F636974792531332E306625732F6D6914
:100AD0006E0A005B257325735D20257320736561A5
:100AE0007263682076656C6F636974792531322E84
:100AF000306625732F6D696E0A005B257325735D63
:100B000020257320737769746368206D61782531BF
:100B10003764205B303D6F66662C313D686F6D69D0
:100B20006E672C323D6C696D69742C333D6C696D58
:100B300069742B686F6D696E675D0A005B257325AC
:100B4000735D20257320737769746368206D696E07
:100B500025313764205B303D6F66662C313D686F10
:100B60006D696E672C323D6C696D69742C333D6C18
:100B7000696D69742B686F6D696E675D0A005B252E
:100B80007325735D20257320726164697573207607
:100B9000616C75652532302E346625730A005B253D
:100BA0007325735D202573206A756E6374696F6E9B
:100BB00020646576696174696F6E2531342E346600
:100BC000257320286C6172676572206973206661E5
:100BD00073746572290A005B257325735D20257384
:100BE000206A65726B20686F6D696E672531362EDD
:100BF000306625732F6D696E5E33202A2031206D9B
:100C0000696C6C696F6E0A005B257325735D202526
:100C100073206A65726B206D6178696D756D253121
:100C2000352E306625732F6D696E5E33202A203194
:100C3000206D696C6C696F6E0A005B257325735DAE
:100C40002025732074726176656C206D696E696D04
:100C5000756D2531372E336625730A005B257325A4
:100C6000735D2025732074726176656C206D6178E8
:100C7000696D756D2531372E336625730A005B2546
:100C80007325735D2025732076656C6F63697479B5
:100C9000206D6178696D756D2531312E3066257353
:100CA0002F6D696E0A005B257325735D2025732007
:100CB0006665656472617465206D6178696D756DD6
:100CC0002531312E306625732F6D696E0A005B2544
:100CD0007325735D2025732061786973206D6F64BF
:100CE00065253138642025730A005B6D615D202025
:100CF0006D696E20617263207365676D656E742522
:100D000031382E336625730A005B736C5D202073C7
:100D10006F6674206C696D697420656E61626C65C4
:100D2000253132640A005B63745D202063686F7252
:100D300064616C20746F6C6572616E636525313718
:100D40002E346625730A005B6A615D20206A756E29
:100D50006374696F6E20616363656C657261746949
:100D60006F6E25382E306625730A005B6764695DF7
:100D70002064656661756C742067636F64652064C8
:100D8000697374616E6365206D6F646525326420DC
:100D90005B303D4739302C313D4739315D0A005BCE
:100DA0006770615D2064656661756C742067636F50
:100DB0006465207061746820636F6E74726F6C2557
:100DC0003364205B303D4736312C313D4736312E80
:100DD000312C323D4736345D0A005B67636F5D201E
:100DE00064656661756C742067636F646520636F0A
:100DF0006F72642073797374656D253364205B3181
:100E00002D3620284735342D473539295D0A005BBA
:100E100067756E5D2064656661756C742067636FCD
:100E2000646520756E697473206D6F646525356423
:100E3000205B303D4732302C313D4732315D0A0076
:100E40005B67706C5D2064656661756C74206763B8
:100E50006F646520706C616E6525313064205B3095
:100E60003D4731372C313D4731382C323D47313900
:100E70005D0A00256320776F726B206F666673656D
:100E8000743A2531322E336625730A002563206DAE
:100E9000616368696E6520706F736E3A2531312E1B
:100EA000336625730A00256320706F736974696F58
:100EB0006E3A2531352E336625730A00546F6F6CF8
:100EC000206E756D62657220202020202020202059
:100ED0002025640A00466565642072617465206D92
:100EE0006F64653A20202020202025730A00446981
:100EF0007374616E6365206D6F64653A20202020F5
:100F000020202025730A0050617468204D6F6465AD
:100F10003A202020202020202020202025730A0095
:100F2000506C616E653A2020202020202020202057
:100F3000202020202025730A004D6F74696F6E20D9
:100F40006D6F64653A20202020202020202025730A
:100F50000A00436F6F7264696E6174652073797300
:100F600074656D3A20202025730A00556E697473EC
:100F70003A20202020202020202020202020202057
:100F800025730A00486F6D696E672073746174651C
:100F90003A202020202020202025730A0046656565
:100FA00064686F6C642073746174653A202020203B
:100FB000202025730A004D6F74696F6E2073746171
:100FC00074653A202020202020202025730A004329
:100FD00079636C652073746174653A202020202049
:100FE0002020202025730A00526177206D616368FC
:100FF000696E652073746174653A20202025730A38
:10100000004D616368696E652073746174653A2090
:1010100020202020202025730A004C696E65206E58
:10102000756D6265723A2531302E30660A0046656C
:10103000656420726174653A2531362E33662573F6
:101040002F6D696E0A0056656C6F636974793A2575
:1010500031372E336625732F6D696E0A00B4108305
:10106000106310473935202D20756E6974732D700B
:1010700065722D7265766F6C7574696F6E206D6F19
:10108000646500473934202D20756E6974732D70A6
:1010900065722D6D696E757465206D6F64652028AD
:1010A000692E652E206665656472617465206D6FBA
:1010B00064652900473933202D20696E7665727387
:1010C000652074696D65206D6F646500F010D01047
:1010D000473931202D20696E6372656D656E7461CC
:1010E0006C2064697374616E6365206D6F64650064
:1010F000473930202D206162736F6C7574652064F0
:10110000697374616E6365206D6F646500411129B8
:10111000111311473634202D20636F6E74696E757C
:101120006F7573206D6F6465004736312E31202D49
:101130002065786163742073746F70206D6F6465CF
:1011400000473631202D206578616374207061740A
:1011500068206D6F6465007B116C115D114731393A
:10116000202D20595A20706C616E6500473138205F
:101170002D20585A20706C616E6500473137202D44
:1011800020585920706C616E65000712F511DC1152
:10119000BB119411473830202D2063616E63656C5C
:1011A000206D6F74696F6E206D6F646520286E6F9F
:1011B0006E65206163746976652900473320202DB0
:1011C00020636F756E74657220636C6F636B7769F3
:1011D0007365206172632066656564004732202074
:1011E0002D20636C6F636B77697365206172632078
:1011F0006665656400473120202D206C696E65614D
:1012000072206665656400473020202D206C696E71
:1012100065617220747261766572736520287365EA
:10122000656B2900CE12B4129A12801266124C120B
:101230003212473539202D20636F6F7264696E61F9
:1012400074652073797374656D20360047353820D6
:101250002D20636F6F7264696E617465207379739A
:1012600074656D203500473537202D20636F6F7210
:1012700064696E6174652073797374656D203400E0
:10128000473536202D20636F6F7264696E61746517
:101290002073797374656D203300473535202D2018
:1012A000636F6F7264696E617465207379737465BE
:1012B0006D203200473534202D20636F6F726469D2
:1012C0006E6174652073797374656D2031004735E4
:1012D00033202D206D616368696E6520636F6F72C6
:1012E00064696E6174652073797374656D000113B0
:1012F000FB12F412486F6D696E6700486F6D65648C
:10130000004E6F7420486F6D656400351330132BE9
:1013100013251320131713456E6420486F6C640067
:10132000486F6C6400446563656C00506C616E00CE
:1013300053796E63004F666600481344133F1348A9
:101340006F6C640052756E0053746F700072136896
:101350001362135B1357134A6F6700486F6D696E12
:10136000670050726F6265004D616368696E696EF7
:1013700067004F666600A813A2139C13971393137C
:101380008D13841353687574646F776E00437963AB
:101390006C6500456E640053746F7000416C61723F
:1013A0006D00526561647900496E697469616C69A8
:1013B0007A696E67000B140514FF13FA13F613F223
:1013C00013ED13E713E113DA13D613CD1353687536
:1013D00074646F776E004A6F6700486F6D696E675F
:1013E000004379636C650050726F626500486F6CF2
:1013F000640052756E00456E640053746F70004156
:101400006C61726D00526561647900496E6974693E
:10141000616C697A696E670032141C14473231209E
:101420002D206D696C6C696D65746572206D6F64DB
:101430006500473230202D20696E63686573206D2A
:101440006F6465006C14611455144C145B72616414
:101450006975735D005B696E686962697465645D76
:10146000005B7374616E646172645D005B646973D8
:1014700061626C65645D00861482147D142064656D
:101480006700206D6D0020696E002A2A2A204E4FC9
:1014900054494345202A2A2A205265736574746989
:1014A0006E672062617564207261746520746F20BC
:1014B0002573005B6E65745D206E6574776F726B6B
:1014C000206D6F646525313764205B303D6D61733D
:1014D0007465725D0A005B626175645D20555342FC
:1014E0002062617564207261746525313564205B0A
:1014F000313D393630302C323D31393230302C33B9
:101500003D33383430302C343D35373630302C359F
:101510003D3131353230302C363D3233303430309D
:101520005D0A005B65785D2020656E61626C6520F8
:10153000666C6F7720636F6E74726F6C25313064E8
:10154000205B303D6F66662C313D584F4E2F584F13
:1015500046462C20323D5254532F4354535D0A00CB
:101560005B65655D2020656E61626C652065636802
:101570006F25313864205B303D6F66662C313D6FDE
:101580006E5D0A005B65635D2020657870616E6446
:10159000204C4620746F2043524C46206F6E2054DE
:1015A00058253664205B303D6F66662C313D6F6E8A
:1015B0005D0A00E615E115DB15D515CF15C815C177
:1015C000153233303430300031313532303000357F
:1015D0003736303000333834303000313932303043
:1015E00000393630300030007379730066620000D5
:1015F00000000702407D31626A622834E11ADC4350
:10160000737973006676000000000703447D316241
:101610006A622C34EC51783F737973006870000073
:1016200000000700487D3162516330340000803F84
:101630007379730068760000000007004C7D31620A
:10164000207D343400000041737973006964000028
:1016500000000400507DC87C6A6224340000000051
:10166000000000006E000000000001000A5F005C46
:101670000163112C00000000000000006C696E6521
:10168000000001000A5F175C0163112C00000000DC
:101690000000000076656C0000000002705E2E5CA9
:1016A0006A62243400000000000000006665656482
:1016B000000000028F5E665C6A6224340000000055
:1016C0000000000073746174000000000E5F715B25
:1016D0006A62243400000000000000006D61637342
:1016E00000000000125F7E5B6A622434000000008C
:1016F000000000006379637300000000165F845BE4
:101700006A62243400000000000000006D6F7473F2
:10171000000000001A5F8A5B6A6224340000000047
:1017200000000000686F6C64000000001E5F905BAA
:101730006A6224340000000000000000756E6974C5
:1017400000000000265F9C5B6A62243400000000F9
:1017500000000000636F6F72000000002A5FA75B4B
:101760006A62243400000000000000006D6F6D6F9D
:10177000000000002E5FB25B6A62243400000000AB
:1017800000000000706C616E00000000325FBB5B07
:101790006A62243400000000000000007061746878
:1017A00000000000365FC65B6A622434000000005F
:1017B0000000000064697374000000003A5FD15BB0
:1017C0006A622434000000000000000066726D6F41
:1017D000000000003E5FDC5B6A6224340000000011
:1017E00000000000746F6F6C00000000425FE75B58
:1017F0006A622434000000006D706F006D706F78B5
:10180000000000034C60C75C6A62243400000000E2
:101810006D706F006D706F79000000034C60C75CE5
:101820006A622434000000006D706F006D706F7A82
:10183000000000034C60C75C6A62243400000000B2
:101840006D706F006D706F61000000034C60C75CCD
:101850006A622434000000006D706F006D706F626A
:10186000000000034C60C75C6A6224340000000082
:101870006D706F006D706F63000000034C60C75C9B
:101880006A62243400000000706F7300706F737818
:101890000000000340609D5C6A6224340000000088
:1018A000706F7300706F73790000000340609D5C7F
:1018B0006A62243400000000706F7300706F737AE6
:1018C0000000000340609D5C6A6224340000000058
:1018D000706F7300706F73610000000340609D5C67
:1018E0006A62243400000000706F7300706F7362CE
:1018F0000000000340609D5C6A6224340000000028
:10190000706F7300706F73630000000340609D5C34
:101910006A622434000000006F6673006F6673789B
:10192000000000035760005D6A622434000000007C
:101930006F6673006F667379000000035760005D87
:101940006A622434000000006F6673006F66737A69
:10195000000000035760005D6A622434000000004C
:101960006F6673006F667361000000035760005D6F
:101970006A622434000000006F6673006F66736251
:10198000000000035760005D6A622434000000001C
:101990006F6673006F667363000000035760005D3D
:1019A0006A62243400000000686F6D00686F6D6526
:1019B00000000000225F965B3A5E243400000000C5
:1019C000686F6D00686F6D78000000004060C26154
:1019D0006A62E62B00000000686F6D00686F6D7929
:1019E000000000004060C2616A62E72B0000000056
:1019F000686F6D00686F6D7A000000004060C26122
:101A00006A62E82B00000000686F6D00686F6D610E
:101A1000000000004060C2616A62E92B0000000023
:101A2000686F6D00686F6D62000000004060C26109
:101A30006A62EA2B00000000686F6D00686F6D63DA
:101A4000000000004060C2616A62EB2B00000000F1
:101A500070726200707262650000000007C5C261AA
:101A60006A62EC2B00000000707262007072627893
:101A70000000000307C531626A62ED2B0000000020
:101A800070726200707262790000000307C53162F3
:101A90006A62F12B00000000707262007072627A5C
:101AA0000000000307C531626A62F52B00000000E8
:101AB00070726200707262610000000307C53162DB
:101AC0006A62F92B0000000070726200707262623C
:101AD0000000000307C531626A62FD2B00000000B0
:101AE00070726200707262630000000307C53162A9
:101AF0006A62012C000000006A6F67006A6F6778F5
:101B00000000000007C5BE61545E0B2C0000000001
:101B10006A6F67006A6F67790000000007C5BE61E1
:101B20005B5E0B2C000000006A6F67006A6F677ACB
:101B30000000000007C5BE61625E0B2C00000000C3
:101B40006A6F67006A6F67610000000007C5BE61C9
:101B5000695E0B2C000000007077720070777231A4
:101B600000000000D8BD05BD6A62243400000000FA
:101B7000707772007077723200000000D8BD05BD2A
:101B80006A6224340000000070777200707772334C
:101B900000000000D8BD05BD6A62243400000000CA
:101BA000707772007077723400000000D8BD05BDF8
:101BB0006A6224340000000000000000737200001C
:101BC0000000000061AF27AF29AF243400000000FF
:101BD00000000000717200000000000003B1B6B008
:101BE0006A622434000000000000000071690000F7
:101BF0000000000007B1CBB06A622434000000008E
:101C000000000000716F0000000000000BB1E7B0A1
:101C10006A622434000000000000000065720000C9
:101C20000000000007C537AC6A62243400000000E1
:101C300000000000716600000000000007C5BE61E2
:101C4000355E2434000000000000000072780000BF
:101C5000000000003CC525676A62243400000000D3
:101C6000000000006D7367000000000008C5BE6141
:101C70006A6224340000000000000000636C6561AB
:101C80007200000007C55C535C5324340000000060
:101C900000000000746573740000000007C5CA7D71
:101CA00094C02434000000000000000064656661F8
:101CB0000000000007C5F57D6861243400000000C5
:101CC00000000000626F6F740000000007C5207EF6
:101CD0001B7D2434000000000000000068656C706B
:101CE0000000000007C58B7D6A62243400000000FC
:101CF00000000000680000000000000007C58B7DA8
:101D00006A6224340000000031000000316D61007F
:101D100000000300B4BDC2616C6285530000000086
:101D2000310000003173610000000303B8BD31626F
:101D30005BBC90536666E63F310000003174720070
:101D400000000B04BDBD316267BC94530000A03F8E
:101D500031000000316D690000000300CCBDC2619C
:101D600073BC8653000000413100000031706F00E9
:101D700000000300D0BDC26192628A5300000000DF
:101D80003100000031706D0000000300D4BDC2615D
:101D9000F1BC8B530000004032000000326D610046
:101DA00000000300B4BDC2616C62A4530000803F18
:101DB000320000003273610000000303B8BD3162DD
:101DC0005BBCAF536666E63F3200000032747200BF
:101DD00000000B04BDBD316267BCB3530000A03FDF
:101DE00032000000326D690000000300CCBDC2610A
:101DF00073BCA553000000413200000032706F0038
:101E000000000300D0BDC2619262A953000000002F
:101E10003200000032706D0000000300D4BDC261CA
:101E2000F1BCAA530000004033000000336D610094
:101E300000000300B4BDC2616C62C35300000040E7
:101E4000330000003373610000000303B8BD31624A
:101E50005BBCCE536666E63F33000000337472000D
:101E600000000B04BDBD316267BCD2530000A03F2F
:101E700033000000336D690000000300CCBDC26177
:101E800073BCC453000000413300000033706F0086
:101E900000000300D0BDC2619262C8530000000080
:101EA0003300000033706D0000000300D4BDC26138
:101EB000F1BCC9530000004034000000346D6100E3
:101EC00000000300B4BDC2616C62E25300004040F8
:101ED000340000003473610000000303B8BD3162B8
:101EE0005BBCED536666E63F34000000347472005C
:101EF00000000B04BDBD316267BCF1530000B44368
:101F000034000000346D690000000300CCBDC261E4
:101F100073BCE353000000413400000034706F00D4
:101F200000000300D0BDC2619262E75300000000D0
:101F30003400000034706D0000000300D4BDC261A5
:101F4000F1BCE853000000407800000078616D00AB
:101F500000000300BB5F305D435DA22A0000803FAC
:101F60007800000078766D0000000B00046031629C
:101F70003A67A72A0000484478000000786672009B
:101F800000000B00006031623A67A32A0000484459
:101F90007800000078746E0000000B030C60316262
:101FA0003A67AF2A000000007800000078746D00E6
:101FB00000000B03086031623A67AB2A0000164349
:101FC00078000000786A6D0000000B00106031623C
:101FD000B15DB32A0000A04178000000786A680073
:101FE00000000B0014603162095EB72A0000204235
:101FF00078000000786A640000000B041860316209
:102000003A67BF2ACDCC4C3D7800000078736E0053
:10201000000003002060C26159C0C6290000803F53
:102020007800000078737800000003002460C2612B
:1020300059C0C729000000007800000078737600BE
:1020400000000B00286031623A67C72A0000FA439B
:1020500078000000786C760000000B002C60316284
:102060003A67CB2A0000C84278000000786C620012
:1020700000000B03306031623A67CF2A0000A040B5
:1020800078000000787A620000000B03346031624F
:102090003A67D32A0000803F7900000079616D0023
:1020A00000000300BB5F305D435DD72A0000803F26
:1020B0007900000079766D0000000B000460316249
:1020C0003A67DC2A00004844790000007966720013
:1020D00000000B00006031623A67D82A00004844D3
:1020E0007900000079746E0000000B030C6031620F
:1020F0003A67E42A000000007900000079746D005E
:1021000000000B03086031623A67E02A00001643C2
:1021100079000000796A6D0000000B0010603162E8
:10212000B15DE82A0000A04179000000796A6800EA
:1021300000000B0014603162095EEC2A00002042AE
:1021400079000000796A640000000B0418603162B5
:102150003A67F42ACDCC4C3D7900000079736E00CB
:10216000000003002060C26159C0C8290000803F00
:102170007900000079737800000003002460C261D8
:1021800059C0C92900000000790000007973760069
:1021900000000B00286031623A67FC2A0000FA4315
:1021A00079000000796C760000000B002C60316231
:1021B0003A67002B0000C84279000000796C620089
:1021C00000000B03306031623A67042B0000A0402E
:1021D00079000000797A620000000B0334603162FC
:1021E0003A67082B0000803F7A0000007A616D009A
:1021F00000000300BB5F305D435D0C2B0000803F9F
:102200007A0000007A766D0000000B0004603162F5
:102210003A67112B000048447A0000007A66720089
:1022200000000B00006031623A670D2B000048444B
:102230007A0000007A746E0000000B030C603162BB
:102240003A67192B000000007A0000007A746D00D4
:1022500000000B03086031623A67152B00009642BC
:102260007A0000007A6A6D0000000B001060316295
:10227000B15D1D2B0000A0417A0000007A6A680061
:1022800000000B0014603162095E212B0000204227
:102290007A0000007A6A640000000B041860316262
:1022A0003A67292BCDCC4C3D7A0000007A736E0042
:1022B000000003002060C26159C0CA29000000006C
:1022C0007A0000007A737800000003002460C26185
:1022D00059C0CB290000803F7A0000007A73760055
:1022E00000000B00286031623A67312B0000C843C0
:1022F0007A0000007A6C760000000B002C603162DE
:102300003A67352B0000C8427A0000007A6C620000
:1023100000000B03306031623A67392B0000A040A7
:102320007A0000007A7A620000000B0334603162A8
:102330003A673D2B0000803F6100000061616D0045
:1023400000000300BB5F305D435D412B0000404057
:102350006100000061766D000000030004603162DE
:102360005163462B00006148610000006166720005
:1023700000000300006031625163422B000061489D
:102380006100000061746E00000003030C603162A4
:102390003A674E2B000080BF6100000061746D0041
:1023A000000003030860316251634A2B000080BFC4
:1023B00061000000616A6D0000000300106031627E
:1023C000B15D522B0000B44561000000616A6800F5
:1023D0000000030014603162095E562B0000344691
:1023E00061000000616A640000000304186031624B
:1023F00051635E2BCDCC4C3D6100000061726100E9
:1024000000000B031C6031625163622BD5B74B3E59
:102410006100000061736E00000003002060C26173
:1024200059C0CC290000803F610000006173780032
:10243000000003002460C26159C0CD2900000000E3
:1024400061000000617376000000030028603162C3
:102450005163662B0000164461000000616C760039
:10246000000003002C60316251636A2B0000C842F7
:1024700061000000616C62000000030330603162A3
:1024800051636E2B0000A04061000000617A620081
:1024900000000303346031625163722B000000407E
:1024A0006200000062616D0000000300BB5F305DF0
:1024B000435D762B000000006200000062766D0034
:1024C000000003000460316251637B2B0000614512
:1024D000620000006266720000000300006031626A
:1024E0005163772B000061456200000062746E004A
:1024F000000003030C6031623A67832B000080BF49
:102500006200000062746D00000003030860316225
:1025100051637F2B000080BF62000000626A6D0083
:102520000000030010603162B15D872B0000A04104
:1025300062000000626A64000000030018603162FB
:102540005163932BCDCC4C3D620000006272610060
:1025500000000B031C6031625163972B0000803F29
:102560006300000063616D0000000300BB5F305D2D
:10257000435DAB2B000000006300000063766D003C
:1025800000000300046031625163B02B000061451C
:1025900063000000636672000000030000603162A7
:1025A0005163AC2B000061456300000063746E0052
:1025B000000003030C6031623A67B82B000080BF53
:1025C0006300000063746D00000003030860316263
:1025D0005163B42B000080BF63000000636A6D008C
:1025E0000000030010603162B15DBC2B0000A0410F
:1025F00063000000636A6400000003001860316239
:102600005163C82BCDCC4C3D630000006372610068
:1026100000000B031C6031625163CC2B0000803F33
:1026200070310000703166727100030060AB31627E
:10263000516361520000C842703100007031637311
:102640006C00030064AB31625163655200007A4450
:1026500070310000703163736800030068AB316251
:10266000516369520000FA447031000070316370A8
:102670006C0003036CAB316251636D520000003E8D
:1026800070310000703163706800030370AB316219
:1026900051637152CDCC4C3E703100007031777374
:1026A0006C00030074AB31625163755200007A44D0
:1026B00070310000703177736800030078AB3162CD
:1026C000516379520000FA44703100007031777024
:1026D0006C0003037CAB316251637D520000003E0D
:1026E00070310000703177706800030380AB316295
:1026F00051638152CDCC4C3E703100007031706F0F
:102700006600030384AB316251638552CDCCCC3D6E
:10271000673534006735347800000B033860316268
:102720003A67122A000000006735340067353479B3
:1027300000000B03386031623A67162A000000007F
:10274000673534006735347A00000B033860316236
:102750003A671A2A00000000673534006735346193
:1027600000000B03386031623A671E2A0000000047
:10277000673534006735346200000B03386031621E
:102780003A67222A00000000673534006735346359
:1027900000000B03386031623A67262A000000000F
:1027A000673535006735357800000B0338603162D6
:1027B0003A672A2A00009642673535006735357931
:1027C00000000B03386031623A672E2A00009642FF
:1027D000673535006735357A00000B0338603162A4
:1027E0003A67322A000000006735350067353561E9
:1027F00000000B03386031623A67362A000000009F
:10280000673535006735356200000B03386031628B
:102810003A673A2A000000006735350067353563AE
:1028200000000B03386031623A673E2A0000000066
:10283000673536006735367800000B033860316243
:102840003A67422A0000000067353600673536795E
:1028500000000B03386031623A67462A000000002E
:10286000673536006735367A00000B033860316211
:102870003A674A2A0000000067353600673536613E
:1028800000000B03386031623A674E2A00000000F6
:10289000673536006735366200000B0338603162F9
:1028A0003A67522A00000000673536006735366304
:1028B00000000B03386031623A67562A00000000BE
:1028C000673537006735377800000B0338603162B1
:1028D0003A675A2A000000006735370067353779B4
:1028E00000000B03386031623A675E2A0000000086
:1028F000673537006735377A00000B03386031627F
:102900003A67622A00000000673537006735376193
:1029100000000B03386031623A67662A000000004D
:10292000673537006735376200000B033860316266
:102930003A676A2A00000000673537006735376359
:1029400000000B03386031623A676E2A0000000015
:10295000673538006735387800000B03386031621E
:102960003A67722A00000000673538006735387909
:1029700000000B03386031623A67762A00000000DD
:10298000673538006735387A00000B0338603162EC
:102990003A677A2A000000006735380067353861E9
:1029A00000000B03386031623A677E2A00000000A5
:1029B000673538006735386200000B0338603162D4
:1029C0003A67822A000000006735380067353863AF
:1029D00000000B03386031623A67862A000000006D
:1029E000673539006735397800000B03386031628C
:1029F0003A678A2A0000000067353900673539795F
:102A000000000B03386031623A678E2A0000000034
:102A1000673539006735397A00000B033860316259
:102A20003A67922A0000000067353900673539613E
:102A300000000B03386031623A67962A00000000FC
:102A4000673539006735396200000B033860316241
:102A50003A679A2A00000000673539006735396304
:102A600000000B03386031623A679E2A00000000C4
:102A7000673932006739327800000103386031620B
:102A80006A62832C000000006739320067393279AE
:102A900000000103386031626A62872C0000000088
:102AA000673932006739327A0000010338603162D9
:102AB0006A628B2C0000000067393200673932618E
:102AC00000000103386031626A628F2C0000000050
:102AD00067393200673932620000010338603162C1
:102AE0006A62932C00000000673932006739326354
:102AF00000000103386031626A62972C0000000018
:102B00006732380067323878000001033C60316278
:102B10006A629B2C00000000673238006732387907
:102B2000000001033C6031626A629F2C00000000DB
:102B3000673238006732387A000001033C60316246
:102B40006A62A32C000000006732380067323861E7
:102B5000000001033C6031626A62A72C00000000A3
:102B60006732380067323862000001033C6031622E
:102B70006A62AB2C000000006732380067323863AD
:102B8000000001033C6031626A62AF2C000000006B
:102B90006733300067333078000001033C603162F6
:102BA0006A62B32C0000000067333000673330796D
:102BB000000001033C6031626A62B72C0000000033
:102BC000673330006733307A000001033C603162C4
:102BD0006A62BB2C0000000067333000673330614D
:102BE000000001033C6031626A62BF2C00000000FB
:102BF0006733300067333062000001033C603162AC
:102C00006A62C32C00000000673330006733306312
:102C1000000001033C6031626A62C72C00000000C2
:102C20006A6964006A6964610000000007C50A629D
:102C30002A634C34000000006A6964006A696462B7
:102C40000000000007C50A622A635034000000003B
:102C50006A6964006A6964630000000007C50A626B
:102C60002A635434000000006A6964006A6964647D
:102C70000000000007C50A622A6358340000000003
:102C8000737973006A61000000000F005A5F3162BF
:102C90003A67E0290050C3477379730063740000FA
:102CA00000000F04795F31623A67E4290AD7233CB8
:102CB00073797300736C000000000700985FC261B5
:102CC0006C62E829000000007379730073740000DF
:102CD0000000070073C0C26153C0BB2900000000A0
:102CE000737973006D74000000000702B0BD31629B
:102CF0001FBD815300000040000000006D65000012
:102D00000000000008C581BD81BD24340000000022
:102D1000000000006D6400000000000008C559BDFF
:102D200059BD24340000000073797300656A000007
:102D3000000007000D84C2619262D9330000803F19
:102D4000737973006A760000000007001184C26185
:102D50009E83F33700000040737973006A730000AC
:102D6000000007001584C2619262F5370000803FC1
:102D7000737973007476000000000700FDC5C2611E
:102D80009262F4540000803F737973007176000002
:102D9000000007000FB1C261DC62BA5200000000FF
:102DA00073797300737600000000070067AFC2619B
:102DB000B762C7520000803F7379730073690000E7
:102DC0000000070063AFE6612BAFC8520000FA4372
:102DD0007379730065630000000007008B67C261B0
:102DE0004568DA3300000000737973006565000000
:102DF000000007008F67C261B568DB330000000088
:102E00007379730065780000000007009367C26162
:102E10007D68DC330000803F737973006261756404
:102E2000000004009767C261D766DD330000A04050
:102E3000737973006E657400000007009B67C261C0
:102E40006C623B3400000000696E0000696E310066
:102E50000000000077C0C2616A62BE290000000065
:102E6000696E0000696E32000000000077C0C26128
:102E70006A62BF2900000000696E0000696E3300BD
:102E80000000000077C0C2616A62C0290000000033
:102E9000696E0000696E34000000000077C0C261F6
:102EA0006A62C12900000000696E0000696E350089
:102EB0000000000077C0C2616A62C2290000000001
:102EC000696E0000696E36000000000077C0C261C4
:102ED0006A62C32900000000696E0000696E370055
:102EE0000000000077C0C2616A62C42900000000CF
:102EF000696E0000696E38000000000077C0C26192
:102F00006A62C529000000007379730067706C0065
:102F100000000700465FC261B762F62900000000AA
:102F20007379730067756E00000007004A5FC26125
:102F30009262F7290000803F7379730067636F0026
:102F4000000007004E5FC2616C62F5290000803FFF
:102F5000737973006770610000000700525FC261FF
:102F6000B762F82900000040737973006764690054
:102F700000000700565FC2619262F929000000005C
:102F800000000000676300000000000007C5D27B5E
:102F9000E27B243400000000000000006D610000AE
:102FA00000000B049C5F31623A67ED29CDCCCC3D2B
:102FB00000000000666400000000030020C5C2613C
:102FC0009262F4370000000075646100756461303E
:102FD000000003003CC50A622A63DF3300000000E2
:102FE0007564610075646131000003003CC50A62CC
:102FF0002A63E33300000000756461007564613288
:10300000000003003CC50A622A63E73300000000A9
:103010007564610075646133000003003CC50A6299
:103020002A63EB330000000075646200756462304F
:10303000000003003CC50A622A63EF330000000071
:103040007564620075646231000003003CC50A6269
:103050002A63F33300000000756462007564623215
:10306000000003003CC50A622A63F7330000000039
:103070007564620075646233000003003CC50A6237
:103080002A63FB33000000007564630075646330DD
:10309000000003003CC50A622A63FF330000000001
:1030A0007564630075646331000003003CC50A6207
:1030B0002A630334000000007564630075646332A2
:1030C000000003003CC50A622A63073400000000C8
:1030D0007564630075646333000003003CC50A62D5
:1030E0002A630B340000000075646400756464306A
:1030F000000003003CC50A622A630F340000000090
:103100007564640075646431000003003CC50A62A4
:103110002A6313340000000075646400756464322F
:10312000000003003CC50A622A6317340000000057
:103130007564640075646433000003003CC50A6272
:103140002A631B34000000005F7465005F746578BB
:103150000000000259C531626A622A500000000076
:103160005F7465005F7465790000000259C53162C3
:103170006A622E50000000005F7465005F74657A1B
:103180000000000259C531626A623250000000003E
:103190005F7465005F7465610000000259C53162AB
:1031A0006A623650000000005F7465005F746562FB
:1031B0000000000259C531626A623A500000000006
:1031C0005F7465005F7465630000000259C5316279
:1031D0006A623E50000000005F7472005F74727893
:1031E0000000000259C531626A624F5100000000C0
:1031F0005F7472005F7472790000000259C5316219
:103200006A625351000000005F7472005F74727A4A
:103210000000000259C531626A6257510000000087
:103220005F7472005F7472610000000259C5316200
:103230006A625B51000000005F7472005F7472622A
:103240000000000259C531626A625F51000000004F
:103250005F7472005F7472630000000259C53162CE
:103260006A626351000000005F7473005F74733121
:103270000000000259C531626A62BA5000000000C5
:103280005F7073005F7073310000000259C53162D6
:103290006A62CA50000000005F6373005F637331AD
:1032A0000000000259C531626A62DA500000000075
:1032B0005F6573005F6573310000000259C53162BC
:1032C0006A62EA50000000005F7873005F78733133
:1032D0000000000259C531626A621C5400000000FF
:1032E0005F6665005F6665310000000259C53162A6
:1032F0006A62FA50000000005F7473005F747332FA
:103300000000000259C531626A62BE500000000030
:103310005F7073005F7073320000000259C5316244
:103320006A62CE50000000005F6373005F63733217
:103330000000000259C531626A62DE5000000000E0
:103340005F6573005F6573320000000259C531622A
:103350006A62EE50000000005F7873005F7873329D
:103360000000000259C531626A6234540000000056
:103370005F6665005F6665320000000259C5316214
:103380006A62FE50000000005F7473005F74733364
:103390000000000259C531626A62C250000000009C
:1033A0005F7073005F7073330000000259C53162B3
:1033B0006A62D250000000005F6373005F63733382
:1033C0000000000259C531626A62E250000000004C
:1033D0005F6573005F6573330000000259C5316299
:1033E0006A62F250000000005F7873005F78733308
:1033F0000000000259C531626A624C5400000000AE
:103400005F6665005F6665330000000259C5316282
:103410006A620251000000005F7473005F747334CD
:103420000000000259C531626A62C6500000000007
:103430005F7073005F7073340000000259C5316221
:103440006A62D650000000005F6373005F637334EC
:103450000000000259C531626A62E65000000000B7
:103460005F6573005F6573340000000259C5316207
:103470006A62F650000000005F7873005F78733472
:103480000000000259C531626A6264540000000005
:103490005F6665005F6665340000000259C53162F1
:1034A0006A62065100000000000000005F64616D68
:1034B0000000000007C5AE5EAE5E243400000000D0
:1034C00000000000736530300000020007C5E661AF
:1034D0000163D3520000000000000000736530312A
:1034E0000000020007C5E6610163D552000000003C
:1034F00000000000736530320000020007C5E6617D
:103500000163D752000000000000000073653033F3
:103510000000020007C5E6610163D9520000000007
:1035200000000000736530340000020007C5E6614A
:103530000163DB52000000000000000073653035BD
:103540000000020007C5E6610163DD5200000000D3
:1035500000000000736530360000020007C5E66118
:103560000163DF5200000000000000007365303787
:103570000000020007C5E6610163E152000000009F
:1035800000000000736530380000020007C5E661E6
:103590000163E35200000000000000007365303951
:1035A0000000020007C5E6610163E552000000006B
:1035B00000000000736531300000020007C5E661BD
:1035C0000163E75200000000000000007365313124
:1035D0000000020007C5E6610163E9520000000037
:1035E00000000000736531320000020007C5E6618B
:1035F0000163EB52000000000000000073653133EE
:103600000000020007C5E6610163ED520000000002
:1036100000000000736531340000020007C5E66158
:103620000163EF52000000000000000073653135B7
:103630000000020007C5E6610163F15200000000CE
:1036400000000000736531360000020007C5E66126
:103650000163F35200000000000000007365313781
:103660000000020007C5E6610163F552000000009A
:1036700000000000736531380000020007C5E661F4
:103680000163F7520000000000000000736531394B
:103690000000020007C5E6610163F9520000000066
:1036A00000000000736532300000020007C5E661CB
:1036B0000163FB520000000000000000736532311E
:1036C0000000020007C5E6610163FD520000000032
:1036D00000000000736532320000020007C5E66199
:1036E0000163FF52000000000000000073653233E8
:1036F0000000020007C5E6610163015300000000FD
:1037000000000000736532340000020007C5E66166
:1037100001630353000000000000000073653235B0
:103720000000020007C5E6610163055300000000C8
:1037300000000000736532360000020007C5E66134
:10374000016307530000000000000000736532377A
:103750000000020007C5E661016309530000000094
:1037600000000000736532380000020007C5E66102
:1037700001630B5300000000000000007365323944
:103780000000020007C5E66101630D530000000060
:1037900000000000737973000000000007C5166583
:1037A0008A63243400000000000000007031000033
:1037B0000000000007C516658A632434000000007D
:1037C00000000000310000000000000007C5166581
:1037D0008A63243400000000000000003200000072
:1037E0000000000007C516658A632434000000004D
:1037F00000000000330000000000000007C516654F
:103800008A6324340000000000000000340000003F
:103810000000000007C516658A632434000000001C
:1038200000000000780000000000000007C51665D9
:103830008A632434000000000000000079000000CA
:103840000000000007C516658A63243400000000EC
:10385000000000007A0000000000000007C51665A7
:103860008A632434000000000000000061000000B2
:103870000000000007C516658A63243400000000BC
:1038800000000000620000000000000007C516658F
:103890008A63243400000000000000006300000080
:1038A0000000000007C516658A632434000000008C
:1038B00000000000696E00000000000007C51665EA
:1038C0006A62243400000000000000006735340004
:1038D0000000000007C516658A632434000000005C
:1038E00000000000673535000000000007C51665C0
:1038F0008A632434000000000000000067353600B1
:103900000000000007C516658A632434000000002B
:1039100000000000673537000000000007C516658D
:103920008A6324340000000000000000673538007E
:103930000000000007C516658A63243400000000FB
:1039400000000000673539000000000007C516655B
:103950008A63243400000000000000006739320050
:103960000000000007C516658A63243400000000CB
:1039700000000000673238000000000007C516652F
:103980008A63243400000000000000006733300028
:103990000000000007C516658A632434000000009B
:1039A000000000006D706F000000000007C5166584
:1039B0008A6324340000000000000000706F730070
:1039C0000000000007C516658A632434000000006B
:1039D000000000006F6673000000000007C5166558
:1039E0008A6324340000000000000000686F6D004E
:1039F0000000000007C516658A632434000000003B
:103A000000000000707262000000000007C516652B
:103A10008A63243400000000000000007077720008
:103A20000000000007C516658A632434000000000A
:103A3000000000006A6F67000000000007C51665FF
:103A40008A63243400000000000000006A696400FA
:103A50000000000007C516658A63243400000000DA
:103A600000000000756461000000000007C51665D5
:103A70008A632434000000000000000075646200C6
:103A80000000000007C516658A63243400000000AA
:103A900000000000756463000000000007C51665A3
:103AA0008A63243400000000000000007564640094
:103AB0000000000007C516658A632434000000007A
:103AC000000000005F7465000000000007C5166577
:103AD0008A63243400000000000000005F7472005C
:103AE0000000000007C516658A632434000000004A
:103AF000000000005F7473000000000007C5166539
:103B00008A63243400000000000000005F7073002E
:103B10000000000007C516658A6324340000000019
:103B2000000000005F6373000000000007C5166519
:103B30008A63243400000000000000005F65730009
:103B40000000000007C516658A63243400000000E9
:103B5000000000005F7873000000000007C51665D4
:103B60008A63243400000000000000005F666500E6
:103B70000000000007C516658A63243400000000B9
:103B8000000000006D0000000000000007C5006894
:103B90006A62243400000000000000007100000090
:103BA0000000000007C5E6676A62243400000000D8
:103BB000000000006F0000000000000007C5CC6797
:103BC0006A622434000000000000000024000000AD
:103BD0000000000007C51A686A6224340000000073
:103BE000456E64206F6620636F6D6D616E64206644
:103BF000696C650A00486F6D696E67206572726F47
:103C000072202D2025632061786973207365747498
:103C1000696E6773206D6973636F6E66696775722D
:103C200065640050726F62696E67206572726F72B0
:103C3000202D20256320617869732063616E6E6F8B
:103C400074206D6F766520647572696E672070727E
:103C50006F62696E67005B69645D202054696E79EC
:103C600047204944253330730A005B68765D202085
:103C700068617264776172652076657273696F6ED0
:103C80002531362E32660A005B68705D202068613F
:103C900072647761726520706C6174666F726D25F5
:103CA00031352E32660A005B66765D2020666972C9
:103CB0006D776172652076657273696F6E25313636
:103CC0002E32660A005B66625D20206669726D773F
:103CD000617265206275696C642531382E32660A1E
:103CE00000456E7465722024626F6F743D312074DC
:103CF0006F20656E7465722074686520626F6F74E2
:103D0000206C6F616465722E0A000A0A0A2323235D
:103D10002054696E794720424F4F54204C4F414404
:103D200045522048656C70202323230A00456E7499
:103D300065722024646566613D3120746F20726570
:103D4000736574207468652073797374656D20746D
:103D50006F2074686520666163746F727920646592
:103D60006661756C742076616C7565732E0A546893
:103D700069732077696C6C206F76657277726974ED
:103D80006520616E79206368616E67657320796F65
:103D9000752068617665206D6164652E0A000A0AE7
:103DA0000A2323232054696E794720524553544FE8
:103DB00052452044454641554C54532048656C704B
:103DC000202323230A00496E766F6B652073656C90
:103DD00066207465737420627920656E74657269FB
:103DE0006E672024746573743D4E20776865726534
:103DF000204E206973206F6E65206F663A0A20207E
:103E000024746573743D312020736D6F6B6520746D
:103E10006573740A202024746573743D3220206811
:103E20006F6D696E67207465737420202028796F28
:103E300075206D757374207472697020686F6D6978
:103E40006E67207377697463686573290A2020247C
:103E5000746573743D3320207371756172652074CD
:103E60006573742020202861207365726965732052
:103E70006F662073717561726573290A202024743E
:103E80006573743D342020617263207465737420FF
:103E9000202020202028736F6D65206C617267657B
:103EA00020636972636C6573290A2020247465732A
:103EB000743D3520206477656C6C207465737420C4
:103EC000202020286D6F76657320737061636564B0
:103ED0002062792031207365636F6E64206477659A
:103EE0006C6C73290A202024746573743D3620207D
:103EF00066656564686F6C642074657374202865FA
:103F00006E746572202120616E64207E20746F20A3
:103F1000686F6C6420616E64207265737461727482
:103F20002C20726573706563746976656C79290AF3
:103F3000202024746573743D3720204D20636F6406
:103F4000657320746573742020284D20636F646549
:103F50007320696E7465726D696E676C6564207735
:103F6000697468206D6F766573290A202024746552
:103F700073743D3820204A534F4E2074657374206B
:103F800020202020286D6F74696F6E207465737413
:103F90002072756E207573696E67204A534F4E20EC
:103FA000636F6D6D616E6473290A202024746573DC
:103FB000743D392020696E76657273652074696D71
:103FC0006520746573740A202024746573743D3110
:103FD0003020726F74617279206D6F74696F6E201A
:103FE000746573740A202024746573743D31312024
:103FF000736D616C6C206D6F76657320746573747E
:104000000A202024746573743D313220736C6F77FD
:10401000206D6F76657320746573740A2020247494
:104020006573743D313320636F6F7264696E6174C0
:10403000652073797374656D206F6666736574208F
:104040007465737420284739322C204735342D4746
:104050003539290A0A546573747320617373756D59
:104060006520612063656E7465726564205859200F
:104070006F726967696E20616E64206174206C657F
:104080006173742038306D6D20636C656172616E90
:10409000636520696E20616C6C206469726563746D
:1040A000696F6E730A546573747320617373756DF1
:1040B00065205A20686173206174206C6561737497
:1040C0002034306D6D20706F736969746976652076
:1040D000636C656172616E63650A54657374732005
:1040E000737461727420776974682061204730208E
:1040F0005830205930205A30206D6F76650A486F4D
:104100006D696E67206973207468652065786365E2
:104110007074696F6E2E204E6F20696E69746961CC
:104120006C20706F736974696F6E206F7220636C9E
:10413000656172616E636520697320617373756D6B
:1041400065640A000A0A0A2323232054696E79470A
:104150002053454C4620544553542048656C7020EC
:104160002323230A0045616368202420636F6D6D5B
:10417000616E642061626F766520616C736F20648C
:104180006973706C6179732074686520746F6B65F6
:104190006E20666F72206561636820736574746950
:1041A0006E6720696E205B205D20627261636B65C3
:1041B00074730A546F207669657720736574746927
:1041C0006E677320656E746572206120746F6B6515
:1041D0006E3A0A0A2020243C746F6B656E3E0A0A10
:1041E000466F72206578616D706C65202479667207
:1041F00020746F20646973706C6179207468652025
:1042000059206D6178206665656420726174650A65
:104210000A546F20757064617465207365747469E5
:104220006E677320656E74657220746F6B656E20A7
:10423000657175616C732076616C75653A0A0A2048
:1042400020243C746F6B656E3E3D3C76616C7565F9
:104250003E0A0A466F72206578616D706C65202495
:104260007966723D38303020746F20736574207425
:1042700068652059206D61782066656564207261EB
:10428000746520746F20383030206D6D2F6D696E2D
:104290007574650A466F7220636F6E666967757222
:1042A0006174696F6E2064657461696C73207365F5
:1042B000653A2068747470733A2F2F676974687553
:1042C000622E636F6D2F73796E746865746F732FD0
:1042D00054696E79472F77696B692F54696E7947F6
:1042E0002D436F6E66696775726174696F6E0A003F
:1042F000546865736520636F6D6D616E64732061D2
:1043000072652061637469766520666F7220636FE1
:104310006E66696775726174696F6E3A0A2020244F
:104320007379732053686F772073797374656D2088
:104330002867656E6572616C292073657474696E97
:1043400067730A2020243120202053686F77206D66
:104350006F746F7220312073657474696E67732097
:10436000286F72207768617465766572206D6F744E
:104370006F7220796F752077616E7420312C322C2A
:10438000332C34290A2020247820202053686F778A
:10439000205820617869732073657474696E67733F
:1043A00020286F7220776861746576657220617865
:1043B000697320796F752077616E7420782C792C61
:1043C0007A2C612C622C63290A2020246D20202065
:1043D00053686F7720616C6C206D6F746F722073FF
:1043E000657474696E67730A20202471202020533D
:1043F000686F7720616C6C206178697320736574D5
:1044000074696E67730A2020246F20202053686F20
:104410007720616C6C206F666673657420736574B9
:1044200074696E67730A2020242420202053686F4B
:104430007720616C6C2073657474696E67730A20F1
:1044400020246820202053686F77207468697320C7
:1044500068656C702073637265656E0A0A000A0AEB
:104460000A2323232054696E794720434F4E46493F
:104470004755524154494F4E2048656C70202323C4
:10448000230A000A466F722064657461696C656472
:104490002054696E794720696E666F207365653AAE
:1044A0002068747470733A2F2F6769746875622E70
:1044B000636F6D2F73796E746865746F732F5469B1
:1044C0006E79472F77696B692F0A466F722074687F
:1044D00065206C6174657374206669726D776172B2
:1044E00065207365653A2068747470733A2F2F677E
:1044F00069746875622E636F6D2F73796E74686569
:10450000746F732F54696E79470A506C65617365D7
:10451000206C6F6720616E792069737375657320F5
:10452000617420687474703A2F2F7777772E7379BF
:104530006E746865746F732E636F6D2F666F72751E
:104540006D730A486176652066756E0A000A4E6FC3
:1045500074653A2054696E79472067656E657261AB
:10456000746573206175746F6D6174696320737411
:1045700061747573207265706F7274732062792034
:1045800064656661756C740A546869732063616E52
:104590002062652064697361626C656420627920C1
:1045A000656E746572696E67202473763D300A53B8
:1045B0006565207468652077696B692062656C6F3A
:1045C0007720666F72206D6F726520646574616913
:1045D0006C732E0A00546865736520636F6D6D619E
:1045E0006E6473206172652061637469766520660C
:1045F000726F6D2074686520636F6D6D616E6420ED
:104600006C696E653A0A205E7820202020202020E8
:1046100020202020202052657365742028636F6E4F
:1046200074726F6C207829202D20736F6674776107
:1046300072652072657365740A20203F2020202057
:104640002020202020202020204D616368696E6595
:1046500020706F736974696F6E20616E6420676388
:104660006F6465206D6F64656C2073746174650A96
:104670002020242020202020202020202020202036
:1046800053686F7720616E642073657420636F6E6A
:1046900066696775726174696F6E20736574746999
:1046A0006E67730A20202120202020202020202037
:1046B0002020202046656564686F6C64202D20737F
:1046C000746F70206D6F74696F6E20776974686F96
:1046D0007574206C6F73696E6720706F736974698D
:1046E0006F6E0A20207E20202020202020202020E5
:1046F0002020204379636C65205374617274202DEF
:1047000020726573746172742066726F6D206665C5
:104710006564686F6C640A202068202020202020B7
:104720002020202020202053686F77207468697330
:104730002068656C702073637265656E0A202024A2
:104740006820202020202020202020202053686F57
:104750007720636F6E66696775726174696F6E202A
:1047600068656C702073637265656E0A202024741E
:104770006573742020202020202020204C69737431
:104780002073656C662D74657374730A202024741D
:104790006573743D4E2020202020202052756E200D
:1047A00073656C662D74657374204E0A202024682E
:1047B0006F6D653D312020202020202052756E2015
:1047C0006120686F6D696E67206379636C650A208C
:1047D0002024646566613D31202020202020205265
:1047E0006573746F726520616C6C20736574746995
:1047F0006E677320746F2022666163746F72792212
:104800002064656661756C74730A000A0A0A2323C2
:10481000232054696E79472048656C702023232338
:104820000A005B6A735D20206A736F6E2073657285
:1048300069616C697A65207374796C6525396420C7
:104840005B303D72656C617865642C313D737472C8
:104850006963745D0A005B6A765D20206A736F6E1F
:1048600020766572626F7369747925313564205BD7
:10487000303D73696C656E742C313D666F6F746585
:10488000722C323D6D657373616765732C333D63C4
:104890006F6E666967732C343D6C696E656E756DFD
:1048A0002C353D766572626F73655D0A005B656AE3
:1048B0005D2020656E61626C65206A736F6E206D8D
:1048C0006F646525313364205B303D746578742CEA
:1048D000313D4A534F4E5D0A00E659E059D959D44B
:1048E00059CB59C059B559A9599D598F597859690A
:1048F000595C5950593C592F591A590659035900B6
:1049000059F158DC58C758B858A85896587F58627B
:104910005845582C5816580558F357E657D457BAE7
:1049200057B757B457B157AE57AB57A857A557A26B
:10493000579F579C5799579657935790578D578A1B
:10494000578757845781577E577B577857755772CB
:10495000576F576C5769576657635760575D575A7B
:10496000575757545751574E574B5748574557422B
:10497000573F573C5739573657335730572D572ADB
:10498000572757245721571E571B571857F456D4EB
:1049900056BA56A0568656625645562D561756FD9F
:1049A00055D955BC55AA558A5573555A5538551F72
:1049B000550155E554CD54BB549D548854845480BE
:1049C000547C547854745470546C546854645460D7
:1049D000545C545854545450544C5448542E541409
:1049E000540154E553D353BC539B538A536A534ADF
:1049F0005330531653FF52CC529F527F525D523761
:104A0000521052F451D551BB51A1517C5153513BDD
:104A1000511051E450AE50795067505550465033C4
:104A2000501A50F84FE64FD44FC24FB04F9E4F8CA4
:104A30004F7A4F684F564F444F324F204F0E4FFC26
:104A40004EF84EF44EF04EEC4EE84EE44EE04EDCA6
:104A50004ED84ED44ED04ECC4EC84EC44EC04EBC96
:104A60004EB84EB44EB04EAC4E984E7A4E5E4E336B
:104A70004E0E4EE94DE54DE14DDD4DD94DD54DD1B3
:104A80004DCD4DC94DC54DC14DBD4DB94DB54DB1C6
:104A90004D9D4D814D654D494D2D4D114DF54CD9D7
:104AA0004CBD4CA14C854C694C4D4C494C454C413E
:104AB0004C3D4C394C354C314C1D4CF54BCE4BA834
:104AC0004B7B4B554B284B244B204B1C4B094BE845
:104AD0004AD34A4A6F6767696E67206379636C657A
:104AE000206661696C65640050726F626520656E56
:104AF00064706F696E742069732073746172746975
:104B00006E6720706F696E740050726F626520630B
:104B100079636C65206661696C65640032343900C4
:104B20003234380032343700486F6D696E67204583
:104B300072726F72202D20486F6D696E67207377D7
:104B4000697463686573206D6973636F6E66696706
:104B50007572656400486F6D696E67204572726F8B
:104B600072202D204E65676174697665206C6174D2
:104B70006368206261636B6F666600486F6D696E83
:104B800067204572726F72202D2054726176656CB9
:104B9000206D696E2026206D617820617265207419
:104BA00068652073616D6500486F6D696E672045AB
:104BB00072726F72202D204C617463682076656C70
:104BC0006F63697479206973207A65726F00486F2A
:104BD0006D696E67204572726F72202D205365617A
:104BE0007263682076656C6F6369747920697320DD
:104BF0007A65726F00486F6D696E67204572726FDB
:104C000072202D20426164206F72206E6F206178C7
:104C100069732073706563696669656400486F6DC8
:104C2000696E67206379636C65206661696C656491
:104C30000032333900323338003233370032333602
:104C400000323335003233340032333300536F6671
:104C500074206C696D69742065786365656465644A
:104C6000202D2043206D617800536F6674206C699D
:104C70006D6974206578636565646564202D2043E3
:104C8000206D696E00536F6674206C696D697420C5
:104C90006578636565646564202D2042206D6178C8
:104CA00000536F6674206C696D6974206578636564
:104CB00065646564202D2042206D696E00536F6627
:104CC00074206C696D6974206578636565646564DA
:104CD000202D2041206D617800536F6674206C692F
:104CE0006D6974206578636565646564202D204175
:104CF000206D696E00536F6674206C696D69742055
:104D00006578636565646564202D205A206D61783F
:104D100000536F6674206C696D69742065786365F3
:104D200065646564202D205A206D696E00536F669E
:104D300074206C696D697420657863656564656469
:104D4000202D2059206D617800536F6674206C69A6
:104D50006D6974206578636565646564202D2059EC
:104D6000206D696E00536F6674206C696D697420E4
:104D70006578636565646564202D2058206D6178D1
:104D800000536F6674206C696D6974206578636583
:104D900065646564202D2058206D696E00536F6630
:104DA00074206C696D6974206578636565646564F9
:104DB0000032313900323138003231370032313689
:104DC0000032313500323134003231330032313289
:104DD0000032313100323130003230390032303877
:104DE00000323037003230360054726170657A6FAD
:104DF000696420706C616E6E6572206661696C65B5
:104E00006420746F20636F6E7665726765004C690D
:104E10006D69742073776974636820686974202DE4
:104E20002053687574646F776E206F636375727258
:104E30006564004D616368696E6520697320616C0B
:104E400061726D6564202D20436F6D6D616E64200D
:104E50006E6F742070726F636573736564004D6F5D
:104E60007665206C657373207468616E206D696E61
:104E7000696D756D2074696D65004D6F7665206C88
:104E8000657373207468616E206D696E696D756DF0
:104E9000206C656E6774680047656E657269632093
:104EA00054696E7947206572726F7200313939002A
:104EB0003139380031393700313936003139350070
:104EC0003139340031393300313932003139310070
:104ED0003139300031383900313838003138370055
:104EE000313836003138350031383400313833004C
:104EF0003138320031383100313830005420776F8A
:104F0000726420697320696E76616C696400542054
:104F1000776F7264206973206D697373696E6700BF
:104F20005220776F726420697320696E76616C69B4
:104F300064005220776F7264206973206D69737307
:104F4000696E67005120776F726420697320696E03
:104F500076616C6964005120776F726420697320F8
:104F60006D697373696E67004C20776F7264206996
:104F70007320696E76616C6964004C20776F72648F
:104F8000206973206D697373696E67004820776FBD
:104F9000726420697320696E76616C6964004820D0
:104FA000776F7264206973206D697373696E67002F
:104FB0004520776F726420697320696E76616C6931
:104FC00064004520776F7264206973206D69737384
:104FD000696E67004420776F726420697320696E80
:104FE00076616C6964004420776F72642069732075
:104FF0006D697373696E67005020776F7264206902
:1050000073206E6F7420612076616C696420746F08
:105010006F6C206E756D626572005020776F7264E0
:10502000206973206E6F7420616E20696E746567ED
:105030006572005020776F7264206973206E656717
:105040006174697665005020776F726420697320FF
:105050007A65726F005020776F72642069732069DF
:105060006E76616C6964005020776F72642069739A
:10507000206D697373696E67004172632073706598
:1050800063696669636174696F6E206572726F72BD
:10509000202D20656E64706F696E742069732073B3
:1050A00074617274696E6720706F696E740041720A
:1050B000632073706563696669636174696F6E20EC
:1050C0006572726F72202D20726164697573206140
:1050D0007263206F7574206F6620746F6C657261E7
:1050E0006E6365004172632073706563696669630E
:1050F0006174696F6E206572726F72202D206D6908
:105100007373696E67206F66667365742873290010
:105110004172632073706563696669636174696F66
:105120006E206572726F72202D206D697373696EC7
:105130006720617869732865732900417263207361
:10514000706563696669636174696F6E2065727208
:105150006F72005370696E646C65206D7573742096
:105160006265207475726E696E6720666F72207456
:1051700068697320636F6D6D616E64005370696E52
:10518000646C65206D757374206265206F6666209F
:10519000666F72207468697320636F6D6D616E64F1
:1051A000005370696E646C65205320776F726420C1
:1051B000697320696E76616C6964005370696E640E
:1051C0006C65205320776F7264206973206D69735A
:1051D00073696E67005370696E646C6520737065E7
:1051E0006564206578636565646564206D617869D0
:1051F0006D756D005370696E646C652073706565C4
:10520000642062656C6F77206D696E696D756D00E5
:1052100050726F6772616D6D656420706F696E7436
:105220002073616D652061732063757272656E74A1
:1052300020706F696E740043757474657220636FBB
:105240006D70656E736174696F6E2063616E6E6FF1
:105250007420626520656E61626C656400526571E0
:105260007565737465642076656C6F636974792005
:1052700065786365656473206C696D697473004754
:1052800030206F72204731206D7573742062652065
:1052900061637469766520666F722047353300520A
:1052A0006F7461727920617865732063616E6E6FCF
:1052B0007420626520757365642077697468207452
:1052C00068697320636F6D6D616E6400496E766509
:1052D0007273652074696D65206D6F64652063610C
:1052E0006E6E6F74206265207573656420776974D3
:1052F00068207468697320636F6D6D616E64004629
:1053000065656472617465206E6F74207370656387
:1053100069666965640053656C65637465642070D3
:105320006C616E6520697320696E76616C696400DA
:1053300053656C656374656420706C616E6520698B
:1053400073206D697373696E6700417869732074A7
:10535000617267657420706F736974696F6E20691C
:105360007320696E76616C6964004178697320749A
:10537000617267657420706F736974696F6E2069FC
:1053800073206D697373696E670041786973206972
:10539000732064697361626C65640041786973208D
:1053A000697320696E76616C696420666F7220741F
:1053B00068697320636F6D6D616E64004178697315
:1053C0002063616E6E6F7420626520707265736514
:1053D0006E74004178697320776F7264206D697311
:1053E00073696E670047636F6465206D6F64616CFD
:1053F0002067726F75702076696F6C6174696F6E6B
:10540000004D20636F646520756E737570706F72E8
:105410007465640047636F646520636F6D6D616ED2
:105420006420756E737570706F7274656400476583
:105430006E657269632047636F646520696E70757D
:1054400074206572726F7200313239003132380067
:1054500031323700313236003132350031323400EA
:1054600031323300313232003132310031323000EA
:1054700031313900313138003131370031313600C6
:1054800031313500313134004A534F4E207374723C
:10549000696E6720746F6F206C6F6E67004A534FA0
:1054A0004E20696E7075742068617320746F6F2070
:1054B0006D616E79207061697273004A534F4E209E
:1054C00073796E746178206572726F7200496E70C4
:1054D00075742076616C75652072616E67652065F4
:1054E00072726F7200496E707574206578636565BD
:1054F0006473206D6178696D756D2076616C75657A
:1055000000496E707574206C657373207468616EE9
:10551000206D696E696D756D2076616C75650049E9
:105520006E7075742065786365656473206D61784D
:10553000206C656E67746800436F6D6D616E6420EA
:105540006E6F74206163636570746564206174209C
:10555000746869732074696D6500506172616D656E
:105560007465722063616E6E6F742062652072656F
:10557000616400506172616D6574657220697320A9
:10558000726561642D6F6E6C7900556E7375707005
:105590006F72746564206E756D626572206F722023
:1055A0004A534F4E207479706500426164206E75D5
:1055B0006D62657220666F726D617400496E76610E
:1055C0006C6964206F72206D616C666F726D6564CA
:1055D00020636F6D6D616E6400556E7265636F67F9
:1055E0006E697A656420636F6D6D616E64206F72A1
:1055F00020636F6E666967206E616D650047656E3A
:105600006572696320617373657274696F6E206679
:1056100061696C757265004D656D6F7279206661A8
:10562000756C74206465746563746564005374619B
:10563000636B206F766572666C6F77206465746546
:105640006374656400436F6E74726F6C6C65722076
:10565000617373657274696F6E206661696C7572CF
:10566000650043616E6F6E6963616C206D61636894
:10567000696E6520617373657274696F6E2066610F
:10568000696C75726500506C616E6E657220617335
:1056900073657274696F6E206661696C75726500FE
:1056A0005374657070657220617373657274696F8D
:1056B0006E206661696C75726500456E636F646526
:1056C0007220617373657274696F6E206661696CB4
:1056D00075726500494F207375622D737973746517
:1056E0006D20617373657274696F6E206661696C99
:1056F00075726500436F6E666967207375622D73FE
:10570000797374656D20617373657274696F6E204F
:105710006661696C75726500383900383800383751
:10572000003836003835003834003833003832005D
:105730003831003830003739003738003737003714
:105740003600373500373400373300373200373111
:10575000003730003639003638003637003636002C
:1057600036350036340036330036320036310036F6
:1057700030003539003538003537003536003535DD
:105780000035340035330035320035310035300016
:1057900034390034380034370034360034350034BE
:1057A00034003433003432003431003430003339C3
:1057B000003338003337003336004261642073749D
:1057C00061747573207265706F7274207365747480
:1057D000696E670050657273697374656E636520E6
:1057E0006572726F7200466C6F6174206973204E2F
:1057F000414E00466C6F617420697320696E666962
:105800006E697465004D6F76652074696D652069F9
:1058100073204E414E004D6F76652074696D652092
:10582000697320696E66696E6974650047656E65A7
:1058300072696320657863657074696F6E20726544
:10584000706F7274004661696C656420746F2067C4
:10585000657420706C616E6E657220627566666537
:10586000720053797374656D20616C61726D202DC7
:10587000207368757474696E6720646F776E004971
:105880006E697469616C697A6174696F6E206661B2
:10589000696C75726500526561642D6F6E6C79205C
:1058A0006164647265737300496E76616C6964202B
:1058B000416464726573730044697669646520624B
:1058C00079207A65726F00466C6F6174696E67202B
:1058D000706F696E74206572726F7200496E7465C4
:1058E000726E616C2072616E6765206572726F7294
:1058F00000496E7465726E616C206572726F720021
:1059000031390031380046756E6374696F6E2069F5
:1059100073207374756262656400456E74657269A4
:105920006E6720626F6F74206C6F616465720049EE
:105930006E697469616C697A696E67004275666642
:1059400065722066756C6C202D20666174616C0038
:105950004275666665722066756C6C004275666697
:10596000657220656D707479004E6F207375636881
:1059700020646576696365004D61782066696C65B1
:105980002073697A6520657863656564656400469F
:10599000696C65206E6F74206F70656E00456E6473
:1059A000206F662066696C6500456E64206F662016
:1059B0006C696E650048617264207265736574007D
:1059C0005465726D696E6174656400436F6D706CCF
:1059D000657465004E6F6F700045616761696E00A8
:1059E0004572726F72004F4B005B7031706F665D75
:1059F0002070776D207068617365206F6666202067
:105A0000202531352E3366205B302E2E315D0A0085
:105A10005B70317770685D2070776D2063637720ED
:105A200070686173652068692531352E3366205BA7
:105A3000302E2E315D0A005B703177706C5D207006
:105A4000776D20636377207068617365206C6F25C4
:105A500031352E3366205B302E2E315D0A005B70AF
:105A6000317773685D2070776D2063637720737082
:105A70006565642068692531352E30662052504DA9
:105A80000A005B703177736C5D2070776D20636303
:105A900077207370656564206C6F2531352E306614
:105AA0002052504D0A005B70316370685D20707742
:105AB0006D206377207068617365206869202531E7
:105AC000352E3366205B302E2E315D0A005B70313F
:105AD00063706C5D2070776D2063772070686173F0
:105AE00065206C6F202531352E3366205B302E2EDD
:105AF000315D0A005B70316373685D2070776D20E3
:105B00006377207370656564206869202531352EC0
:105B100030662052504D0A005B703163736C5D201B
:105B200070776D206377207370656564206C6F20DB
:105B30002531352E30662052504D0A005B7031669B
:105B400072715D2070776D206672657175656E6328
:105B5000792020202531352E306620487A0A0053DE
:105B6000595354454D205245414459004C6F61648E
:105B7000696E6720636F6E666967732066726F6D0A
:105B800020454550524F4D00496E697469616C69FA
:105B90007A696E6720636F6E6669677320746F2021
:105BA00064656661756C742073657474696E67737F
:105BB000007B226572223A7B226662223A25302ED1
:105BC00032662C227374223A25642C226D7367226C
:105BD0003A222573227D7D0A007B65723A7B6662DC
:105BE0003A25302E32662C73743A25642C6D736717
:105BF0003A222573227D7D0A005B71765D2020713B
:105C000075657565207265706F7274207665726255
:105C10006F73697479253764205B303D6F66662C3D
:105C2000313D73696E676C652C323D747269706CBE
:105C3000655D0A00716F3A25640A0071693A25644E
:105C40000A0071723A25640A005B73765D20207346
:105C50007461747573207265706F727420766572EA
:105C6000626F73697479253664205B303D6F6666B8
:105C70002C313D66696C74657265642C323D7665C5
:105C800072626F73655D0A005B73695D20207374D7
:105C90006174757320696E74657276616C25313438
:105CA0002E3066206D730A004D6F746F722025636D
:105CB00020706F77657220656E61626C6564207319
:105CC000746174653A25322E30660A005B257325AF
:105CD000735D206D257320706F776572206D616E26
:105CE0006167656D656E7425313064205B303D649D
:105CF000697361626C65642C313D616C77617973A5
:105D0000206F6E2C323D696E206379636C652C3395
:105D10003D7768656E206D6F76696E675D0A005B22
:105D2000257325735D206D257320706F6C6172691A
:105D3000747925313864205B303D6E6F726D616C13
:105D40002C313D726576657273655D0A005B257363
:105D500025735D206D2573206D6963726F737465A3
:105D6000707325313664205B312C322C342C385D35
:105D70000A005B257325735D206D257320747261A5
:105D800076656C20706572207265766F6C757469CB
:105D90006F6E2531302E346625730A005B2573251E
:105DA000735D206D2573207374657020616E676C60
:105DB000652532302E336625730A005B2573257303
:105DC0005D206D2573206D617020746F206178698E
:105DD0007325313564205B303D582C313D592C32D0
:105DE0003D5A2E2E2E5D0A005B6D745D20206D6F76
:105DF000746F722069646C652074696D656F757469
:105E00002531342E3266205365630A001B5E175E0F
:105E1000125E2064656700206D6D0020696E004988
:105E20006E7075742025732073746174653A202038
:105E30002020202025640A005B73745D2020737786
:105E400069746368207479706525313864205B302B
:105E50003D4E4F2C313D4E435D0A00546573742016
:105E6000232564206E6F7420666F756E640A004E81
:105E7000362047393220583735205930205A300AD9
:105E80004E3720463530302E300A4E3820473159B3
:105E9000302E3239315A2D322E3139380A4E3920CE
:105EA0005837342E37363759302E3035385A2D3250
:105EB0002E3335350A4E3130205837342E373039AD
:105EC000592D302E3030305A2D322E3337310A4E84
:105ED0003131205837342E3532395A2D322E323660
:105EE000340A4E3132205837342E36333459302E5E
:105EF0003130355A2D322E3331390A4E3133205854
:105F000037342E38343359302E3331345A2D322E23
:105F10003138330A4E3134205837352E303030592D
:105F2000302E3437315A2D322E3132360A4E313539
:105F30002059302E3635305A2D322E3130300A4E1F
:105F40003136205837342E37383359302E343334E5
:105F50005A2D322E3133310A4E3137205837342EF4
:105F600035363659302E3231375A2D322E323434BE
:105F70000A4E3138205837342E333530592D302ED3
:105F80003030305A2D322E3138320A4E31392058C5
:105F900037342E3137305A2D322E3134340A4E32C6
:105FA00030205837342E34323959302E3235395A60
:105FB0002D322E3136350A4E3231205837342E35B7
:105FC000333359302E3336335A2D322E3139310A8C
:105FD0004E3232205837342E36383959302E35313A
:105FE000395A2D322E3131340A4E3233205837345B
:105FF0002E38343459302E3637345A2D322E30392B
:10600000360A4E3234205837352E30303059302E43
:106010003833305A2D322E3131340A4E3235205930
:10602000312E3031305A2D322E3134340A4E323640
:10603000205837342E37383759302E3739375A2DC4
:10604000322E3039380A4E3237205837342E363215
:106050003859302E3633385A2D322E3130380A4ED8
:106060003238205837342E34363959302E343738B8
:106070005A2D322E3135370A4E3239205837342EC8
:1060800033303959302E3331395A2D322E313130A7
:106090000A4E3330205837342E30343459302E30B5
:1060A00035335A2D322E3130380A4E33312058379D
:1060B000332E39393059302E3030305A2D322E307F
:1060C00037370A4E3332205837332E3831315A2D74
:1060D000312E3934370A4E3333205837332E39377F
:1060E0003359302E3136325A2D322E3037390A4E4E
:1060F0003334205837342E32343359302E3433323F
:106100005A2D322E3038340A4E3335205837342E3B
:1061100034353959302E3634395A2D322E313537FF
:106120000A4E3336205837342E36373659302E380B
:1061300036355A2D322E3130390A4E333720583702
:10614000342E38333859312E3032375A2D322E31E1
:1061500031310A4E3338205837352E3030305931EE
:106160002E3138395A2D322E3136300A4E333920FD
:1061700059312E3336395A2D322E3139340A4E34B4
:1061800030205837342E38343259312E3231315A8A
:106190002D322E3133340A4E3431205837342E36D6
:1061A000383459312E3035335A2D322E3132300AAF
:1061B0004E3432205837342E34323159302E37395C
:1061C000305A2D322E3137360A4E34332058373478
:1061D0002E33313659302E3638345A2D322E313353
:1061E000370A4E3434205837342E31353859302E52
:1061F0003532365A2D322E3037370A4E3435205844
:1062000037332E39343759302E3331365A2D322E1A
:106210003036370A4E3436205837332E3839345911
:10622000302E3236335A2D322E3034360A4E343731
:10623000205837332E37333759302E3130355A2DD9
:10624000312E3931380A4E3438205837332E363310
:106250003159302E3030305A2D312E3837320A4EE7
:106260003439205837332E3435325A2D312E3831C7
:10627000350A4E3530205837332E36363559302EC4
:106280003231345A2D312E3931340A4E35312058BD
:1062900037332E38323559302E3337345A2D322E8B
:1062A0003032380A4E3532205837332E3837395984
:1062B000302E3432375A2D322E3037360A4E35339F
:1062C000205837342E30393259302E3634315A2D49
:1062D000322E3039340A4E3534205837342E33308C
:1062E0003659302E3835345A2D322E3139320A4E45
:1062F0003535205837342E35313959312E3036382E
:106300005A2D322E3134310A4E3536205837342E3C
:1063100037333359312E3238315A2D322E3134330E
:106320000A4E3537205837342E38343059312E3311
:1063300038385A2D322E3137340A4E3538205837F6
:10634000342E38393359312E3434325A2D322E31DD
:1063500036390A4E3539205837352E3030305931DC
:106360002E3534385A2D322E3132310A4E36302005
:1063700059312E3732385A2D322E3037360A4E36B2
:1063800031205837342E38343359312E3537315A7D
:106390002D322E3133300A4E3632205837342E37D4
:1063A000333859312E3436365A2D322E3139350A9A
:1063B0004E3633205837342E34373659312E32305A
:1063C000345A2D322E3134370A4E36342058373471
:1063D0002E32313559302E3934335A2D322E323057
:1063E000320A4E3635205837332E39303059302E58
:1063F0003632385A2D322E3130310A4E3636205848
:1064000037332E38343859302E3537365A2D322E10
:106410003039360A4E3637205837332E353836590C
:10642000302E3331345A2D312E3931330A4E36382D
:10643000205837332E33373759302E3130355A2DD7
:10644000312E3830380A4E3639205837332E32370D
:106450003259302E3030305A2D312E3738370A4EDF
:106460003730205837332E3138325A2D312E3738C5
:10647000370A4E3731205837332E3039325A2D31C2
:106480002E3735300A4E3732205837332E343130DC
:1064900059302E3331385A2D312E3836380A4E378E
:1064A00033205837332E37383159302E3638395A51
:1064B0002D322E3038360A4E3734205837342E30AD
:1064C000393959312E3030375A2D322E3232340A82
:1064D0004E3735205837342E32303559312E313140
:1064E000335A2D322E3231310A4E37362058373456
:1064F0002E33363459312E3237325A2D322E31372F
:10650000360A4E3737205837342E36323959312E25
:106510003533375A2D322E3139310A4E373820581B
:1065200037342E36383259312E3539305A2D322EF5
:106530003137370A4E3739205837342E38393459E5
:10654000312E3830325A2D322E3036360A4E38300F
:10655000205837352E30303059312E3930385A2DB9
:10656000322E3034360A4E38312059322E303837F8
:106570005A2D322E3035310A4E3832205837342ECB
:1065800038333959312E3932375A2D322E3036328E
:106590000A4E3833205837342E36373959312E3792
:1065A00036365A2D322E3133360A4E38342058378B
:1065B000342E36323559312E3731335A2D322E3171
:1065C00037300A4E3835205837342E353732593166
:1065D0002E3635395A2D322E3138300A4E38362083
:1065E0005837342E33353859312E3434355A2D320C
:1065F0002E3135370A4E3837205837342E31393757
:1066000059312E3238345A2D322E3139350A4E381E
:1066100038205837342E30393059312E3137375AE7
:106620002D322E3234350A4E3839205837332E3930
:10663000383359312E3037305A2D322E3232350A16
:106640004E3930205837332E38323359302E3931C5
:10665000305A2D322E3133380A4E393120583733E3
:106660002E33393459302E3438325A2D312E3931B7
:10667000370A4E3932205837332E31383059302EC0
:106680003236385A2D312E3832350A4E39332058A9
:1066900037322E39363659302E3035345A2D312E88
:1066A0003731310A4E3934205837322E3931335987
:1066B0002D302E3030305A2D312E3639330A4E39A6
:1066C00035205837322E3733335A2D312E36343663
:1066D0000A4E3936205837322E39393759302E3252
:1066E00036345A2D312E3735330A4E393720583744
:1066F000332E32363059302E3532375A2D312E392D
:1067000030320A4E3938205837332E363239593024
:106710002E3839365A2D322E3037370A4E39392035
:106720005837332E38343059312E3130375A2D32D4
:106730002E3232340A4E313030205837332E383929
:106740003359312E3136305A2D322E3234350A4EED
:106750003130312058373559305A300A004E312007
:1067600054314D360A4E32204731370A4E332047D6
:1067700032310A4E382046313830300A4E392047FF
:10678000310A4E3130302047393220582D32352EE3
:10679000313737592D33342E303732205A2D312EA0
:1067A000303030202854454D502C2052454D4F5606
:1067B00045204C41544552290A4E33343320582D3C
:1067C00032352E353935592D33342E3334390A4E7E
:1067D00033343420582D32352E373031592D33345F
:1067E0002E3433360A4E33343520582D32352E3779
:1067F0003931592D33342E3532300A4E3334362068
:10680000582D32352E383634592D33342E3630311A
:106810000A4E33343720582D32352E393230592D27
:1068200033342E3637390A4E33343820582D32352A
:106830002E393630592D33342E3735340A4E333411
:106840003920582D32352E393832592D33342E38DF
:1068500032360A4E33353020582D32352E393837FE
:10686000592D33342E3839350A4E33353120582DD1
:1068700032352E393736592D33342E3936310A4ECA
:1068800033353220582D32352E393438592D3335A1
:106890002E3032330A4E33353320582D32352E39CF
:1068A0003033592D33352E3038320A4E33353420BB
:1068B000582D32352E383431592D33352E31333869
:1068C0000A4E33353520582D32352E373633592D73
:1068D00033352E3139300A4E33353620582D323586
:1068E0002E363639592D33352E3233390A4E33355B
:1068F0003720582D32352E353539592D33352E3236
:1069000038340A4E33353820582D32352E3433334F
:10691000592D33352E3332350A4E33353920582D23
:1069200032352E323931592D33352E3336330A4E26
:1069300033363020582D32352E313334592D3335FE
:106940002E3339370A4E33363120582D32342E3912
:106950003633592D33352E3432380A4E3336322001
:10696000582D32342E373737592D33352E343535AF
:106970000A4E33363320582D32342E353737592DC1
:1069800033352E3437370A4E33363420582D3234CF
:106990002E333637592D33352E3439360A4E3336A9
:1069A0003520582D32342E313434592D33352E358F
:1069B00031310A4E33363620582D32332E393039A4
:1069C000592D33352E3532320A4E33363720582D75
:1069D00032332E363631592D33352E3532390A4E73
:1069E00033363820582D32332E343033592D333549
:1069F0002E3533320A4E33363920582D32332E316C
:106A00003333592D33352E3533320A4E3337302058
:106A1000582D32322E383533592D33352E35323705
:106A20000A2F4E3235313820473058302E33323726
:106A3000592D33332E3532315A2D312E3030300A24
:106A40004E32353139204D3330004E31204732300F
:106A50000A4E3520473430204731370A4E31302036
:106A60005431204D30360A284E31352047393020F8
:106A70004730205830205930205A30290A4E3230C1
:106A8000205335303030204D3033200A4E323520FF
:106A900058302E3036342059302E333236205A308A
:106AA0000A4E343020473031204631362E300A4EDF
:106AB00035302058302E3036342059302E3332368F
:106AC0000A4E35352058302E3036302059302E328F
:106AD00039330A4E36302058302E3037372059306F
:106AE0002E3236370A4E36352058302E313131208D
:106AF00059302E3235370A4E37302058302E313447
:106B0000392059302E3235320A4E37352058302E42
:106B10003138382059302E3235350A4E3830205829
:106B2000302E3232372059302E3236380A4E383530
:106B30002058302E3235372059302E3237310A4E18
:106B400039302058302E3333352059302E323635F7
:106B50000A4E39352058302E3431322059302E32F9
:106B600037310A4E3130302058302E3437342059E6
:106B7000302E3238370A4E3130352058302E3439E5
:106B8000312059302E3238390A4E313130205830C8
:106B90002E3531372059302E3237330A4E313135C8
:106BA0002058302E3534342059302E3236330A4EA8
:106BB0003132302058302E3538302059302E323690
:106BC000310A4E3132352058302E35393520593082
:106BD0002E3236330A4E3133302058302E36323191
:106BE0002059302E3237340A4E3133352058302E6A
:106BF0003635392059302E3330360A4E3134302074
:106C000058302E3637332059302E3333350A4E3133
:106C100034352058302E3637392059302E3336311E
:106C20000A4E3135302058302E3637382059302E24
:106C30003338390A4E3135352058302E363730202A
:106C400059302E3432300A4E3136302058302E36FC
:106C500037302059302E3434360A4E3136352058EC
:106C6000302E3638302059302E3437340A4E3137F2
:106C7000302058302E3730342059302E3439370AEE
:106C80004E3137352058302E3733322059302E359B
:106C900031350A4E3138302058302E3739342059AA
:106CA000302E3533350A4E3138352058302E3837AE
:106CB000322059302E3536370A4E3139302058308F
:106CC0002E3935302059302E3630340A4E31393590
:106CD0002058312E3033312059302E3634370A4E79
:106CE0003230302058312E3134392059302E37325D
:106CF000320A4E3230352058312E33303820593058
:106D00002E3835340A4E3231302058312E3433305B
:106D10002059302E3938340A4E3231352058312E30
:106D20003434372059302E3938360A4E323230203A
:106D300058312E3632382059302E3832320A4E32FF
:106D400032352058312E3733322059302E373134F6
:106D50000A4E3233302058322E3030392059302EFE
:106D60003338310A4E3233352058322E3131362005
:106D700059302E3236360A4E3234302058322E32C6
:106D800032382059302E3135370A4E3234352058BA
:106D9000322E3238302059302E3132330A4E3235CD
:106DA000302058322E3333322059302E3039340AC5
:106DB0004E3235352058322E3432332059302E3071
:106DC00037300A4E3236302058322E343839205976
:106DD000302E3036350A4E3236352058322E353583
:106DE000372059302E3036360A4E3237302058325E
:106DF0002E3632372059302E3038340A4E3237355D
:106E00002058322E3639332059302E3130390A4E3F
:106E10003238302058322E3733302059302E31332B
:106E2000330A4E3238352058322E3830352059301A
:106E30002E3139300A4E3239302058322E3832391C
:106E40002059302E3231360A4E3239352058322E02
:106E50003838302059302E3239310A4E3330302014
:106E600058322E3838342059302E3330300A4E33D1
:106E700030352058322E3839382059302E333332BD
:106E80000A4E3331302058322E3930352059302EC9
:106E90003336370A4E3331352058322E39313020CF
:106EA00059302E3430370A4E3332302058322E3992
:106EB00030382059302E3434360A4E33323520588B
:106EC000322E3930312059302E3439350A4E333391
:106ED000302058322E3839372059302E3439350A7F
:106EE0004E3333352058322E3839302059302E3534
:106EF00032340A4E3334302058322E38343220594E
:106F0000302E3630340A4E3334352058322E383154
:106F1000342059302E3636350A4E3335302058322B
:106F20002E3739342059302E3735300A4E33353527
:106F30002058322E3739312059302E3833380A4E06
:106F40003336302058322E3831392059302E3937E7
:106F5000360A4E3336352058322E383337205931E1
:106F60002E3034340A4E3337302058322E383632F1
:106F70002059312E3131320A4E3337352058322ED6
:106F80003837372059312E3134350A4E33383020D6
:106F900058322E3931322059312E3231370A4E33A0
:106FA00038352058322E3931372059312E32323689
:106FB0000A4E3339302058322E3935312059312E8E
:106FC0003238310A4E3339352058322E3937302095
:106FD00059312E3239350A4E3430302058322E395C
:106FE00039362059312E3239350A4E343035205851
:106FF000332E3031332059312E3237350A4E343169
:10700000302058332E3032342059312E3235340A64
:107010004E3431352058332E3037302059312E310F
:1070200035310A4E3432302058332E30373720591C
:10703000312E3133340A4E3432352058332E31322A
:10704000352059312E3033390A4E343330205833FD
:107050002E3133382059312E3031390A4E34333500
:107060002058332E3230352059302E3930380A4EE0
:107070003434302058332E3238322059302E3739BC
:10708000370A4E3434352058332E333631205930B8
:107090002E3639310A4E3435302058332E343236BC
:1070A0002059302E3539320A4E3435352058332E9A
:1070B0003435362059302E3534330A4E34363020AC
:1070C00058332E3437392059302E3439330A4E3460
:1070D00036352058332E3439342059302E34373257
:1070E0000A4E3437302058332E3530352059302E63
:1070F0003434360A4E3437352058332E3531382063
:1071000059302E3431370A4E3438302058332E352A
:1071100033302059302E3339310A4E343835205827
:10712000332E3536342059302E3330300A4E343930
:10713000302058332E3537372059302E3235330A28
:107140004E3439352058332E3536382059302E32CA
:1071500031320A4E3530302058332E3534342059F0
:10716000302E3137360A4E3530352058332E3534EF
:10717000312059302E3134360A4E353130205833D3
:107180002E3535332059302E3131390A4E353135CF
:107190002058332E3537362059302E3130360A4EAE
:1071A0003532302058332E3539372059302E313092
:1071B000320A4E3532352058332E36313820593088
:1071C0002E3130390A4E3533302058332E3633398C
:1071D0002059302E3132390A4E3533352058332E6E
:1071E0003635302059302E3135390A4E353430207D
:1071F00058332E3636332059302E3137380A4E3533
:1072000034352058332E3637382059302E31393224
:107210000A4E3535302058332E3639392059302E24
:107220003139370A4E3535352058332E3732332031
:1072300059302E3139360A4E3536302058332E37F4
:1072400036342059302E3137390A4E3536352058EC
:10725000332E3830352059302E3136350A4E3537F9
:10726000302058332E3838342059302E3135390AF1
:107270004E3537352058332E3934392059302E3198
:1072800036350A4E3538302058332E3936362059A7
:10729000302E3137350A4E3538352058332E3937B0
:1072A000382059302E3139340A4E35393020583390
:1072B0002E3937382059302E3232330A4E3539358F
:1072C0002058332E3936302059302E3234350A4E7C
:1072D0003630302058332E3833342059302E333165
:1072E000310A4E3630352058332E37363220593059
:1072F0002E3334350A4E3631302058332E3732365D
:107300002059302E3338390A4E3631352058332E35
:107310003730332059302E3435380A4E363230204B
:1073200058332E3638322059302E3533300A4E3607
:1073300032352058332E3637392059302E353334F4
:107340000A4E3633302058332E3632362059302EFE
:107350003638310A4E3633352058332E35363820FC
:1073600059302E3832380A4E3634302058332E34C5
:1073700034342059312E3038300A4E3634352058C6
:10738000332E3430352059312E3136370A4E3635CA
:10739000302058332E3430342059312E3136370ACC
:1073A0004E3635352058332E3338372059312E326A
:1073B00030380A4E3636302058332E333834205980
:1073C000312E3230380A4E3636352058332E333689
:1073D000352059312E3236350A4E36373020583363
:1073E0002E3335352059312E3238350A4E36373561
:1073F0002058332E3334382059312E3330380A4E4A
:107400003638302058332E3333332059312E33352C
:10741000300A4E3638352058332E33323120593128
:107420002E3339310A4E3639302058332E3331312C
:107430002059312E3432380A4E3639352058332E01
:107440003333392059312E3432330A4E373030201D
:1074500058332E3434302059312E3430360A4E37DA
:1074600030352058332E3531302059312E343038D4
:107470000A4E3731302058332E3538352059312EC9
:107480003432310A4E3731352058332E36313120DF
:1074900059312E3433390A4E3732302058332E3694
:1074A00031312059312E3434310A4E37323520589B
:1074B000332E3631352059312E3434310A4E37339C
:1074C000302058332E3633362059312E3438380A8E
:1074D0004E3733352058332E3633342059312E353C
:1074E00031370A4E3734302058332E363232205955
:1074F000312E3534330A4E3734352058332E36305A
:10750000352059312E3536330A4E37353020583331
:107510002E3537362059312E3537350A4E37353529
:107520002058332E3534342059312E3538310A4E17
:107530003736302058332E3437392059312E3539EB
:10754000320A4E3736352058332E343531205931F2
:107550002E3539380A4E3737302058332E333837E6
:107560002059312E3632360A4E3737352058332ED1
:107570003339302059312E3633360A4E37383020E1
:1075800058332E3533322059312E3630320A4E37A9
:1075900038352058332E3630312059312E35393791
:1075A0000A4E3739302058332E3636382059312E8E
:1075B0003539380A4E3739352058332E373832208E
:1075C00059312E3631320A4E3830302058332E376A
:1075D00039342059312E3631380A4E38303520585A
:1075E000332E3836382059312E3633360A4E38315C
:1075F000302058332E3931382059312E3635350A5E
:107600004E3831352058332E3934352059312E3605
:1076100036370A4E3832302058332E393634205916
:10762000312E3638350A4E3832352058332E393619
:10763000372059312E3638350A4E383330205833FA
:107640002E3937342059312E3639390A4E383335F0
:107650002058332E3938342059312E3732350A4EDE
:107660003834302058332E3938342059312E3735BC
:10767000380A4E3834352058332E393730205931B6
:107680002E3739300A4E3835302058332E393435BC
:107690002059312E3831370A4E3835352058332E9F
:1076A0003931382059312E3832360A4E38363020AA
:1076B00058332E3839312059312E3832370A4E3866
:1076C00036352058332E3834322059312E3830395F
:1076D0000A4E3837302058332E3739382059312E5A
:1076E0003738340A4E3837352058332E3734362061
:1076F00059312E3737320A4E3838302058332E362B
:1077000039382059312E3736340A4E38383520581A
:10771000332E3633352059312E3736360A4E383926
:10772000302058332E3535332059312E3738350A2D
:107730004E3839352058332E3437382059312E38C9
:1077400032300A4E3930302058332E3430392059F7
:10775000312E3836340A4E3930352058332E3334F2
:10776000352059312E3931380A4E393130205833CD
:107770002E3236342059322E3032330A4E393135DA
:107780002058332E3234382059322E3035310A4EBB
:107790003932302058332E3234302059322E30389E
:1077A000310A4E3932352058332E33313620593292
:1077B0002E3038360A4E3933302058332E33393094
:1077C0002059322E3130340A4E3933352058332E79
:1077D0003431342059322E3132310A4E393430208E
:1077E00058332E3433312059322E3135330A4E3945
:1077F00034352058332E3433332059322E3138303B
:107800000A4E3935302058332E3432372059322E33
:107810003230350A4E3935352058332E3431332045
:1078200059322E3232340A4E3936302058332E3304
:1078300039322059322E3234320A4E3936352058F8
:10784000332E3333352059322E3234340A4E393701
:10785000302058332E3237382059322E3233360A00
:107860004E3937352058332E3235362059322E32A4
:1078700034320A4E3938302058332E3233392059B9
:10788000322E3235310A4E3938352058332E3231C6
:10789000312059322E3238300A4E3939302058339F
:1078A0002E3137342059322E3335360A4E39393598
:1078B0002058332E3135392059322E3339370A4E7C
:1078C000313030302058332E3135302059322E347B
:1078D00033380A4E313030352058332E3134302091
:1078E00059322E3438310A4E313031302058332E4F
:1078F0003133322059322E3531300A4E3130313564
:107900002058332E3131382059322E3534330A4E37
:10791000313032302058332E3039392059322E351B
:1079200037360A4E313032352058332E303531203B
:1079300059322E3633310A4E313033302058332EFF
:107940003030332059322E3636360A4E3130333508
:107950002058322E3935372059322E3638350A4ED6
:10796000313034302058322E3930372059322E36CB
:1079700039390A4E313034352058322E38363020DD
:1079800059322E3731310A4E313035302058322EAF
:107990003831392059322E3732370A4E31303535A9
:1079A0002058322E3736382059322E3734350A4E89
:1079B000313036302058322E3731362059322E377A
:1079C00035370A4E313036352058322E363735208D
:1079D00059322E3735370A4E313037302058322E53
:1079E0003537392059322E3733310A4E3130373559
:1079F0002058322E3537302059322E3732330A4E46
:107A0000313038302058322E3535392059322E3722
:107A100032300A4E313038352058322E353330204E
:107A200059322E3730310A4E313039302058322E0B
:107A30003530312059322E3639330A4E313039350E
:107A40002058322E3437312059322E3638330A4EF0
:107A5000313130302058322E3434332059322E36E2
:107A600036380A4E313130352058322E33393620EF
:107A700059322E3633340A4E313131302058322EBD
:107A80003335342059322E3539310A4E31313135C2
:107A90002058322E3335322059322E3539310A4EA4
:107AA000313132302058322E3332352059322E3592
:107AB00034330A4E313132352058322E33313520AD
:107AC00059322E3532310A4E313133302058322E70
:107AD0003330372059322E3439380A4E313133356C
:107AE0002058322E3239362059322E3436340A4E4E
:107AF000313134302058322E3239332059322E343D
:107B000032370A4E313134352058322E3239352051
:107B100059322E3336360A4E313135302058322E16
:107B20003332312059322E3330330A4E313135352C
:107B30002058322E3335382059322E3234370A4EFF
:107B4000313136302058322E3431392059322E32EC
:107B500030330A4E313136352058322E3431392007
:107B600059322E3137390A4E313137302058322EC2
:107B70003430352059322E3135380A4E31313735CF
:107B80002058322E3336322059322E3132330A4EBB
:107B9000313138302058322E3335342059322E319D
:107BA00030340A4E313138352058322E33353420B6
:107BB00059322E3039310A4E313139302058322E77
:107BC0003338302059322E3036350A4E313139357E
:107BD0002058322E3431302059322E3035310A4E71
:107BE000313230302058322E3431302059322E305C
:107BF00034370A4E313230352058322E3430352069
:107C000059322E3032380A4E313231302058322E2D
:107C10003430382059322E3031300A4E313231353D
:107C20002058322E3431362059312E3939350A4E0A
:107C3000313232302058322E3433332059312E39FC
:107C400038320A4E313232352058322E3433382011
:107C500059312E3936330A4E313233302058322ED4
:107C60003434372059312E3934380A4E31323335D5
:107C70002058322E3436312059312E3933380A4EBD
:107C8000313234302058322E3438302059312E39A8
:107C900033310A4E313234352058322E34373820C1
:107CA00059312E3839390A4E313235302058322E7A
:107CB0003438372059312E3837350A4E3132353580
:107CC0002058322E3530342059312E3835340A4E72
:107CD000313236302058322E3532372059312E3855
:107CE00034380A4E313236352058322E3534392068
:107CF00059312E3834390A4E313237302058322E2D
:107D00003537372059312E3836310A4E3132373532
:107D10002058322E3630342059312E3836360A4E1D
:107D2000313238302058322E3633312059312E3806
:107D300035340A4E313238352058322E3634302020
:107D400059312E3832370A4E313239302058322EDE
:107D50003634302059312E3739320A4E31323935E6
:107D60002058322E3632392059312E3735390A4EC5
:107D7000313330302058322E3631322059312E37BF
:107D800032370A4E313330352058322E35373620CF
:107D900059312E3639340A4E313331302058322E93
:107DA0003533362059312E3636320A4E313331359D
:107DB0002058322E3437302059312E3631360A4E83
:107DC000313332302058322E3334352059312E356C
:107DD00035310A4E313332352058322E3330372088
:107DE00059312E3532310A4E313333302058322E4C
:107DF0003236302059312E3438320A4E3133333551
:107E00002058322E3234332059312E3437370A4E2F
:107E1000313334302058322E3232382059312E341A
:107E200036390A4E313334352058322E3232322030
:107E300059312E3434380A4E313335302058322EF1
:107E40003232382059312E3432350A4E31333535FD
:107E50002058322E3235342059312E3430350A4EE6
:107E6000313336302058322E3236382059312E33C5
:107E700037330A4E313336352058322E32373920D7
:107E800059312E3334320A4E313337302058322EA6
:107E90003330382059312E3238370A4E31333735A6
:107EA0002058322E3334302059312E3235340A4E98
:107EB000313338302058322E3430372059312E3279
:107EC00030310A4E313338352058322E3434312097
:107ED00059312E3135360A4E313339302058322E51
:107EE0003435342059312E3133310A4E313339355E
:107EF0002058322E3436302059312E3130360A4E49
:107F0000313430302058322E3436342059312E312D
:107F100030320A4E313430352058322E3437312049
:107F200059312E3033360A4E313431302058322E0A
:107F30003436362059302E3937310A4E3134313506
:107F40002058322E3435312059302E3839370A4EE8
:107F5000313432302058322E3431352059302E37DA
:107F600039310A4E313432352058322E34303320F4
:107F700059302E3736370A4E313433302058322EAE
:107F80003338382059302E3736350A4E31343335B0
:107F90002058322E3330362059302E3834310A4EA4
:107FA000313434302058322E3232322059302E398A
:107FB00031310A4E313434352058322E31313420AB
:107FC00059302E3939350A4E313435302058322E59
:107FD0003030322059312E3037360A4E3134353573
:107FE0002058312E3930352059312E3133390A4E4F
:107FF000313436302058312E3735342059312E3235
:1080000032330A4E313436352058312E363337204C
:1080100059312E3237380A4E313437302058312E0C
:108020003538322059312E3330310A4E313437351C
:108030002058312E3535382059312E3331350A4EFE
:10804000313438302058312E3436302059312E33E7
:1080500035320A4E313438352058312E33393920F3
:1080600059312E3336300A4E313439302058312EC2
:108070003333382059312E3335340A4E31343935C3
:108080002058312E3238372059312E3332390A4EAA
:10809000313530302058312E3234382059312E329B
:1080A00039340A4E313530352058312E32313720AF
:1080B00059312E3235340A4E313531302058312E77
:1080C0003231342059312E3235320A4E3135313584
:1080D0002058312E3137322059312E3139350A4E60
:1080E000313532302058312E3132382059312E314D
:1080F00033390A4E313532352058312E3131302066
:1081000059312E3131370A4E313533302058302E27
:108110003935382059302E3934310A4E313533351E
:108120002058302E3839312059302E3837330A4E06
:10813000313534302058302E3832352059302E38F1
:1081400030380A4E313534352058302E3735352009
:1081500059302E3734370A4E313535302058302ECD
:108160003631392059302E3633330A4E31353535D4
:108170002058302E3437372059302E3532360A4EBB
:10818000313536302058302E3437372059302E359F
:1081900032340A4E313536352058302E34313120C4
:1081A00059302E3437360A4E313537302058302E7C
:1081B0003333312059302E3435340A4E313537358A
:1081C0002058302E3237382059302E3432370A4E6C
:1081D000313538302058302E3233312059302E335B
:1081E00039370A4E313538352058302E3138332062
:1081F00059302E3337390A4E313539302058302E28
:108200003133352059302E3336350A4E3135393534
:108210002058302E3037362059302E3334310A4E24
:108220003136303520473030204633302E300A4E3C
:1082300031363130204D3035200A4E31363135203F
:10824000473930205830205930205A300A4E3136C4
:108250003135204D33300A28456E64206F66204347
:108260004E432050726F6772616D2900284D53474D
:108270002A2A2A2A204D6963726F7374657020540C
:10828000657374205B76315D202A2A2A2A290A47E1
:1082900030302047313720473231204734302047B3
:1082A000343920473830204739300A673078307900
:1082B000307A300A7B22316D69223A317D0A7B2285
:1082C000326D69223A317D0A7B22336D69223A315F
:1082D0007D0A7B22346D69223A317D0A673020782D
:1082E00031300A7B22316D69223A327D0A78300AB8
:1082F0007B22316D69223A347D0A7831300A7B2243
:10830000316D69223A387D0A78300A673020793138
:10831000300A7B22326D69223A327D0A79300A7B3B
:1083200022326D69223A347D0A7931300A7B223259
:108330006D69223A387D0A79300A6730207A313007
:108340000A7B22336D69223A327D0A7A300A7B2217
:10835000336D69223A347D0A7A31300A7B22336DDB
:1083600069223A387D0A7A300A6730206131300A52
:108370007B22346D69223A327D0A61300A7B2234D5
:108380006D69223A347D0A6131300A7B22346D698D
:10839000223A387D0A61300A6D3200284D53472A4F
:1083A0002A2A2A20436F6F7264696E617465206F98
:1083B0006666736574732074657374205B76315DD3
:1083C000202A2A2A2A290A67303067313767323152
:1083D0006734306734396738306739300A67353485
:1083E0000A673932783079307A300A663630300AA6
:1083F000284D53472A2A2A2A207465737420473946
:1084000032206F6666736574732A2A2A2A290A281D
:108410006D73675374657020313A204D6F76652017
:1084200066726F6D20302C3020746F2033302C300A
:10843000206D6D20696E20706F7369746976652098
:108440005820646972656374696F6E290A286D73B8
:10845000675374657020323A205265736574206FDB
:10846000726967696E20746F20302E3020757369D1
:108470006E6720473932290A286D73675374657017
:1084800020333A204D6F766520746F2032302C30C7
:108490002E2053686F756C64206D6F7665203230C6
:1084A000206D6D20696E20706F7369746976652028
:1084B0005820646972656374696F6E20616E642010
:1084C000737461747573207265706F727420736851
:1084D0006F756C642073746172742066726F6D20A6
:1084E000302C30290A286D73675374657020343A34
:1084F000204D6F766520746F20302E302020205361
:10850000686F756C64206D6F7665203230206D6DFC
:1085100020696E206E6567617469766520582064F5
:108520006972656374696F6E20616E642073746133
:10853000747573207265706F72742073686F756CD8
:10854000642073746172742066726F6D2032302CF7
:1085500030290A67317833300A67393278300A6750
:10856000317832300A6731783079300A2473720AF0
:1085700067393278300A673470302E350A284D5307
:10858000472A2A2A2A207465737420473535206FBC
:108590006666736574732A2A2A2A290A286D736706
:1085A0005374657020313A2053657420436F6F72A5
:1085B00064696E6174652073797374656D2032200F
:1085C0005B6735355D20746F206F66667365742058
:1085D0006F662035302C3530290A286D7367537447
:1085E000657020323A2053656C65637420473535D9
:1085F00020636F6F7264696E617465207379737440
:10860000656D290A286D73675374657020333A20AD
:108610004D6F766520746F20302C302E20486561B8
:10862000642073686F756C64206D6F766520646973
:1086300061676F6E616C6C7920696E202B582061C8
:108640006E64202B5920616E64207374617475739D
:10865000207265706F72742073686F756C6420731C
:10866000746172742066726F6D20302C30290A6735
:1086700031304C3270327835307935300A673535E3
:108680000A6730783079300A673470302E350A281E
:108690004D53472A2A2A2A2074657374204735339C
:1086A000206162736F6C757465206F766572726994
:1086B000646573202A2A2A2A290A286D736753744D
:1086C000657020313A2052756E206120737175619A
:1086D000726520696E204735352073797374656D36
:1086E000290A286D73675374657020323A205275D9
:1086F0006E20612073717561726520772F47353365
:10870000206F76657272696465290A6730783079FE
:10871000300A673078323079300A67307832307911
:1087200032300A673078307932300A673078307901
:10873000300A673470302E350A6735336730783049
:1087400079300A673533673078323079300A6735E7
:108750003367307832307932300A673533673078B2
:10876000307932300A6735336730783079300A67CC
:1087700030783079300A673470302E350A284D53FE
:10878000472A2A2A2A2074657374205265747572E8
:108790006E20746F20686F6D65202A2A2A2A290AA4
:1087A000286D73675374657020313A205265747573
:1087B000726E20746F20686F6D65207573696E67C7
:1087C00020473238290A286D736753746570203248
:1087D0003A20526573657420746F204735342063E6
:1087E0006F6F72642073797374656D290A6732380C
:1087F0000A6735340A6D333000284D53472A2A2A38
:108800002A205465737420616363757261637920F3
:108810006F6620736C6F77206D6F766573205B7663
:10882000315D202A2A2A2A290A6735350A673078D5
:108830003079300A673470302E350A673470302E44
:10884000350A67317831306632320A6735340A6763
:1088500030783079300A6D333000284D53472A2A5A
:108860002A2A205465737420766572792073686FA4
:108870007274206D6F766573205B76315D202A2AD5
:108880002A2A290A6730783079300A673470302E06
:10889000350A673178302E3166313030300A783021
:1088A0000A78302E310A78300A78302E310A783042
:1088B0000A78302E310A78300A78302E310A783032
:1088C0000A78302E310A78300A78302E310A783022
:1088D0000A78302E310A78300A78302E310A783012
:1088E0000A78302E310A78300A78302E310A783002
:1088F0000A78302E310A78300A78302E310A7830F2
:108900000A78302E310A78300A78302E310A6734EE
:1089100070302E350A78300A78302E30310A7830AF
:108920000A78302E30310A78300A78302E30310A09
:1089300078300A78302E30310A78300A78302E308C
:10894000310A78300A78302E30310A78300A78309F
:108950002E30310A78300A78302E30310A78300AD9
:1089600078302E30310A78300A78302E30310A785B
:10897000300A78302E30310A78300A78302E303193
:108980000A78300A78302E30310A78300A78302E62
:1089900030310A6730783079300A6D3200284D5313
:1089A000472A2A2A2A20526F7461727920417869F5
:1089B00073204D6F74696F6E2054657374205B76FD
:1089C000315D202A2A2A2A290A6730306731376721
:1089D00032316734306734396738306739300A6785
:1089E00030783079307A306130623063300A673500
:1089F000350A6730783079300A6633363030300ADD
:108A00006730613336300A623336300A63333630CA
:108A10000A61300A62300A63300A673161313434E6
:108A2000300A62313434300A63313434300A613010
:108A30000A62300A63300A67316131343430623798
:108A40003230633336300A783079307A30613062D0
:108A50003063300A67317836306131343430623710
:108A60003230633336300A783079307A30613062B0
:108A70003063300A673178363079353061313434DB
:108A80003062373230633336300A783079307A30BA
:108A90006130623063300A6731783630793530784A
:108AA0003235613134343062373230633336300A34
:108AB000783079307A306130623063300A6735342B
:108AC0000A6730783079300A6D333000284D5347CB
:108AD0002A2A2A2A20496E76657273652054696DA8
:108AE00065204D6F74696F6E2054657374205B76DA
:108AF000315D202A2A2A2A290A67303067313767F0
:108B000032316734306734396738306739300A6753
:108B100035350A6730783079300A6739330A66307C
:108B20002E30310A67317831300A7931300A7A31A2
:108B3000300A6131300A78300A79300A7A300A61B5
:108B4000300A67317831307931307A2D3130613106
:108B5000300A6730783079307A3061300A66302EEA
:108B6000310A6732783130792D31307A2D323069DF
:108B700031300A6730783079307A300A67337831AB
:108B800030792D31307A2D32306931300A673078C2
:108B90003079307A300A673278323079307A2D3253
:108BA000306931300A6730783079307A300A67338B
:108BB00078323079306931300A6730783079307AFC
:108BC000300A6732783079307A2D33306931300AA3
:108BD0006733783079307A306931300A67307830ED
:108BE00079307A300A67327830793069323020282B
:108BF0004357203336302064656772656573290AF0
:108C00006733783079306932302028434357203336
:108C100036302064656772656573290A6739340ADE
:108C20006735340A6730783079300A6D3330007B2D
:108C3000226763223A226730306731376732316703
:108C40003430673439673830673930227D0A7B2207
:108C50006763223A22673535227D0A7B22676322C9
:108C60003A22673078307930227D0A7B226763228E
:108C70003A2266353030227D0A7B226763223A220F
:108C8000284D53477371756172657329227D0A7B84
:108C9000226763223A226730783230227D0A7B22B3
:108CA0006763223A22793230227D0A7B226763226F
:108CB0003A227830227D0A7B226763223A22793079
:108CC000227D0A7B226763223A2267317831302283
:108CD0007D0A7B226763223A22793130227D0A7B2A
:108CE000226763223A227830227D0A7B2267632240
:108CF0003A227930227D0A7B226763223A22284D6C
:108D00005347636972636C657329227D0A7B22670E
:108D100063223A226732783130792D31306931302F
:108D2000227D0A7B226763223A22673078307930CD
:108D3000227D0A7B226763223A22673378313079B9
:108D40002D3130693130227D0A7B226763223A223D
:108D5000673078307930227D0A7B226763223A229D
:108D600067327832307930693130227D0A7B226770
:108D700063223A22673078307930227D0A7B22677D
:108D800063223A2267337832307930693130227D7C
:108D90000A7B226763223A22673078307930227D5D
:108DA0000A7B226763223A22673278307930693150
:108DB00030227D0A7B226763223A2267337830793A
:108DC00030693130227D0A7B226763223A2267357F
:108DD00034227D0A7B226763223A22673078307919
:108DE00030227D0A7B226763223A226D3330227D56
:108DF00000284D53472A2A2A2A204D636F64657341
:108E00002074657374205B76315D202A2A2A2A2912
:108E10000A6735350A6730783079300A6D330A676A
:108E20003470310A6D350A673470310A6D340A675F
:108E30003470310A6D350A673470310A6D370A674C
:108E40003470310A6D390A673470310A6D380A6737
:108E50003470310A6D390A663530300A673078323D
:108E6000300A7932300A6D330A78300A6D340A7963
:108E7000300A6D350A67317831300A6D370A793139
:108E8000300A6D380A78300A6D390A79300A67324B
:108E9000783130792D31306931300A6D330A6730DD
:108EA000783079300A6D340A6733783130792D3172
:108EB000306931300A6D350A6730783079300A6DA3
:108EC000370A673278323079306931300A6D380AC2
:108ED0006730783079300A6D390A67337832307903
:108EE000306931300A6730783079300A673278304B
:108EF00079306931300A6733783079306931300A36
:108F00006735340A6730783079300A6D333000289D
:108F10004D53472A2A2A2A2046656564686F6C6487
:108F20002054657374205B76315D202A2A2A2A2911
:108F30000A284D53472A2A2A2A204D616E75616CF2
:108F40006C7920656E746572202120616E64207ECC
:108F500020647572696E67206D6F76656D656E74DD
:108F600020746F2074657374202A2A2A2A290A67BC
:108F700035350A6730783079300A673470330A67DC
:108F800030306731376732316734306734396738AA
:108F9000306739300A663630300A67307831303021
:108FA0007637362E3736350A783079300A673534D9
:108FB0000A6730783079300A6D333000284D5347D6
:108FC0002A2A2A2A204477656C6C20546573742001
:108FD0005B76315D202A2A2A2A290A6730306731D8
:108FE000376732316739300A6735350A673078308C
:108FF00079300A663530300A67307831300A6734A4
:1090000070310A67307832300A673470310A67305D
:109010007831300A673470310A67307830300A6747
:109020003470310A79350A6735340A673078307917
:10903000300A6D330A673470310A6730783130791D
:1090400031300A6D350A673470310A673078323052
:109050007932300A6D340A673470310A67307833F8
:10906000307933300A6D380A673470310A673078E6
:1090700034307934300A6D390A673470310A673018
:109080007835307935300A6730783079300A6D3389
:1090900030004E3120673030673137673231673406
:1090A000306734396738306739300A4E31302067DD
:1090B00030783079300A4E323020663530300A4E02
:1090C0003330206732783130792D313069313020BA
:1090D00028435720323730206465677265657329ED
:1090E0000A4E3430206730783079300A4E353020DF
:1090F0006733783130792D3130693130202843435E
:10910000572039302064656772656573290A4E36C9
:1091100030206730783079300A4E38302067327826
:1091200032307930693130202843572031383020AF
:1091300064656772656573290A4E37302067307839
:109140003079300A4E3830206733783230793069E0
:10915000313020284343572031383020646567720E
:10916000656573290A4E3930206730783079300AC6
:109170004E39392046313230300A4E313030206796
:1091800032783079306932302028435720333630F6
:109190002064656772656573290A4E313130206736
:1091A00032783079306932302028435720333630D6
:1091B00020616761696E290A4E313230206637308E
:1091C0003020284368616E6765206665656420729B
:1091D000617465207768696C6520696E204732206C
:1091E0006D6F74696F6E206D6F6465290A4E31333F
:1091F0003020673278307930693230202843572068
:10920000333630203372642074696D65290A4E311B
:109210003430206732783079306932302028435733
:1092200020333630203474682074696D65290A4E05
:1092300031353020663530300A4E313630206733D4
:10924000783079307A3430693230202843435720DF
:10925000333630206465677265657320776974689A
:10926000206C696E6561722074726176656C290A82
:109270004E313730206733783079307A3069323088
:1092800020284343572033363020616761696E29B7
:109290000A4E313830206637303020286D73672A07
:1092A0002A2A2A4368616E676520666565642072B4
:1092B000617465207768696C6520696E204733208A
:1092C0006D6F74696F6E206D6F64652A2A2A2A2972
:1092D0000A4E3139302067337830793069323020A6
:1092E0002843435720333630203372642074696D2D
:1092F00065290A4E32303020673378307930693250
:10930000302028434357203336302034746820748B
:10931000696D65290A4E32313020286D73672A2A1B
:109320002A2A473138204576616C20746573742A87
:109330002A2A2A290A4E3232302047312058333027
:109340002E373037205A35302E37323720463530D9
:10935000300A4E32333020473138204730322058DF
:1093600036372E373338205A32332E3631372052A3
:10937000323520463235300A4E32343020673830AC
:109380000A4E323530206730783079307A300A4EE4
:10939000323630206D333000284D53472A2A2A2A8E
:1093A0002053717561726573204D6F74696F6E2003
:1093B00054657374205B76315D202A2A2A2A290A93
:1093C0006730306731376732316734306734396737
:1093D00038306739300A6730783079300A6730784A
:1093E0003230202874726176657273652061203294
:1093F000306D6D2073717561726520696E20582023
:10940000616E642059290A7932300A78300A79303D
:109410000A673178313066353030202864726177E0
:1094200020612031306D6D20737175617265206926
:109430006E205820616E64205920617420463530BA
:1094400030290A7931300A78300A79300A67307A5F
:109450003230202874726176657273652061203223
:10946000306D6D2073717561726520696E205820B2
:10947000616E64205A290A7832300A7A300A7830CC
:109480000A67317832307932307A323066353030AE
:1094900020286665656420612032306D6D20646926
:1094A00061676F6E616C20696E20582C20592061B5
:1094B0006E64205A290A783079307A300A7834304C
:1094C0007934307A3430202874726176657273652D
:1094D00020612034306D6D206375626520696E20D7
:1094E000582C205920616E64205A290A783430792A
:1094F000307A300A78307934307A34300A7834303F
:109500007934307A300A783079307A34300A7830E9
:109510007934307A300A78343079307A34300A78D5
:109520003079307A300A6738300A673078307930ED
:109530000A673078310A673078300A6D3330002896
:109540004D53472A2A2A2A20486F6D696E67205496
:10955000657374205B76315D202A2A2A2A290A67DE
:1095600032382E32783079307A300A6D3330002834
:109570004D53472A2A2A2A20536D6F6B6520546564
:109580007374205B76315D202A2A2A2A290A473003
:10959000302047313720473231204734302047349C
:1095A0003920473830204739300A6D3367347031FD
:1095B0000A6D35673470310A6D34673470310A6D65
:1095C00033673470310A6D35673470310A6D37672F
:1095D0003470310A6D39673470310A6D3867347010
:1095E000310A6D390A6730783079307A300A67305D
:1095F00030207832300A78300A7932300A79300AED
:109600007A32300A7A300A6132300A61300A4730E1
:10961000302078323020793230207A323020613276
:10962000300A473030207830207930207A3020617D
:10963000300A4730312066333020783220793220AA
:109640007A322061320A7830207930207A302061F5
:10965000300A673078310A673078300A6D32002C72
:10966000000A00257300256C750025312E30660038
:109670002573002C000A0025733A25730025733AE0
:10968000256C750025733A25312E30660025733A16
:109690002573005B74765D20207465787420766590
:1096A00072626F7369747925313564205B303D7364
:1096B000696C656E742C313D766572626F73655DA1
:1096C0000A0025660A00256C750A0025640A002533
:1096D000730A0074696E7967205B25735D2065727B
:1096E000723A2025733A202573200074696E7967D9
:1096F000205B25735D206F6B3E2000CECA63CA3BA2
:10970000CB5CCBBBCBA8CA93CE63CA27CF93CFC1C8
:10971000CDA8CA0000400640061040B800B893CE5D
:1097200063CA27CF93CFC1CDA8CA00004006200648
:109730000840B800B809D163CA2AD0A5D054D2F3E2
:10974000CFA0084006050609010809D163CA2AD03E
:10975000A5D0CDCBA8CAB00840060540B0308000E7
:1097600000000000F0E0D0C0100100CF67332221DC
:109770001F1B1301016E616E00696E66004E414E43
:10978000494E495459494E46CDCCCC3D0AD7233C8D
:1097900017B7D13877CC2B329595E6241FB14F0AF5
:1097A000000020410000C84200401C4620BCBE4CC6
:1097B000CA1B0E5AAEC59D7400407A10F35A00A021
:1097C000724E18090010A5D4E80000E8764817008A
:1097D00000E40B54020000CA9A3B000000E1F505CA
:1097E000000080969800000040420F000000A08614
:1097F00001000000102700000000E8030000000046
:109800006400000000000A000000000001000000E9
:1098100000002C76D888DC674F0823DFC1DFAE5903
:10982000E1B1B796E5E3E453C63AE651997696E896
:10983000E6C28426EB898C9B62ED407C6FFCEFBC1A
:109840009C9F40F2BAA56FA5F490055A2AF75C9345
:109850006B6CF9676DC11BFCE0E40D47FEF520E67B
:10986000B500D0ED902E0300943577050080841E5E
:10987000080000204E0A000000C80C333333330FB9
:10988000986E12831141EF8D2114893BE65516CF56
:10989000FEE6DB18D1844B381BF77C1D901DA4BB62
:1098A000E424203284725E228100C9F124ECA1E517
:1098B0003D2711241FBECFEFCDBFDFE5DEBF00E0A7
:1098C0000CBF13E2A0E0B0E2E6EAFBEC01E00BBF64
:1098D00002C007900D92A438B107D9F725E5A4E896
:1098E000B3E201C01D92A930B207E1F70E94B7842C
:1098F0000C94D1E50C940000FC016081718182819F
:1099000093810E94A2D76093632C0895FC0160812B
:109910007181828193810E94A2D76093622C089505
:10992000AF92BF92CF92DF92EF92FF920F931F936D
:10993000CF93DF937B018C0186EEC82E8BE2D82E6D
:10994000E601AA24A394BC2EBC18F7016191719181
:10995000819191917F012CEA35EC47E257E30E9417
:1099600031D918164CF4F80140815181628173811C
:109970008B2D0E942586A8820C5F1F4F2196FBE24B
:10998000CC3EDF0701F7DF91CF911F910F91FF9040
:10999000EF90DF90CF90BF90AF900C943086FC0199
:1099A00060817181828193810E94A2D76093642C2F
:1099B000613019F481E00E94E77B81E00C94087C1F
:1099C000CF93DF93CDB7DEB76897CDBFDEBFFC0185
:1099D00060817181828193810E94A2D76093652CFE
:1099E00081E0613019F40E94E77B0CC00E94087C82
:1099F000CE01019628E1FC0111922A95E9F7BC01FC
:109A00000E94CF4C6896CDBFDEBFDF91CF91089505
:109A10000F931F93CF93DF93CDB7DEB72D97CDBFB5
:109A2000DEBF27E0E2EDF0E28E010F5F1F4FD801AD
:109A300001900D922A95E1F7BC01660F771F680F20
:109A4000791F660F771F660F771F660F771F6451A8
:109A50007A4E45E050E0CE0108960E9441E36885C9
:109A600070E0C8010E946FE3009739F46B8570E0E5
:109A7000C8010E946FE3009711F0801B01C08FEFB7
:109A80002D96CDBFDEBFDF91CF911F910F9108952D
:109A9000EF92FF920F931F93CF93DF938C01F62EDB
:109AA000E72EEC012D96FC016185728583859485F6
:109AB0000E94A2D71F926F93DF93CF930F5E1F4F29
:109AC0001F930F93DF93CF93EF92FF92E5E0F5E5BD
:109AD00081818F9380818F930E9408E4EDB7FEB758
:109AE0003C96EDBFFEBFDF91CF911F910F91FF908C
:109AF000EF9008950F931F93CF93DF93EC01162FF0
:109B0000072F8C819D810E94084D83305CF58F3F2B
:109B1000A1F528C09E01235F3F4F9F938F938C85B3
:109B20008F938B858F938A858F9389858F933F93AE
:109B30002F936196DF93CF933F932F930F931F93B0
:109B4000809106558F93809105558F930E9408E46C
:109B50008DB79EB740968DBF9EBFDF91CF911F916D
:109B60000F910895EBE7F4E1659174914FE450E0B3
:109B70008BEF97E30E9441E3CDCFE0915C2CF0E0C6
:109B8000EE0FFF1FE958FB4E659174914FE450E0D2
:109B90008BEF97E30E9441E3BDCF0F931F93CF93C9
:109BA000DF93EC01162F072F8C819D810E94084DB9
:109BB00083307CF58F3FC1F52CC0AE014F5E5F4F07
:109BC0009E01235F3F4F9F938F938C858F938B854F
:109BD0008F938A858F9389858F935F934F933F935C
:109BE0002F935F934F933F932F930F931F938091E6
:109BF00006558F93809105558F930E9408E48DB789
:109C00009EB742968DBF9EBFDF91CF911F910F915E
:109C10000895EBE7F4E1659174914FE450E08BEF28
:109C200097E30E9441E3C9CFE0915C2CF0E0EE0F96
:109C3000FF1FE958FB4E659174914FE450E08BEFA4
:109C400097E30E9441E3B9CFDF92EF92FF920F9327
:109C50001F93CF93DF93CDB7DEB72897CDBFDEBF7D
:109C60008B01E42ED52E37E0E9EDF0E2DE0111960E
:109C700001900D923A95E1F728870E94084DF82E41
:109C8000288582E08F1518F0E22FF0E002C0E2E0B4
:109C9000F0E0EE0FFF1FE958FB4E659174914FE421
:109CA00050E08BEF97E30E9441E39F938F93F8017D
:109CB00083818F9382818F9381818F9380818F9312
:109CC000E1E0F0E0EC0FFD1FEF0DF11D80811F9230
:109CD0008F93DF92EF92809106558F938091055577
:109CE0008F930E9408E4CDBFDEBF2896CDBFDEBFB4
:109CF000DF91CF911F910F91FF90EF90DF9008952A
:109D00004F925F926F927F92AF92BF92CF92DF920B
:109D1000EF92FF920F931F93CF93DF93C6EEDBE298
:109D20000BEA1AE25C018991813009F042C0F80126
:109D3000C480D580E680F780408051806280738047
:109D4000A3019201C701B6010E9485D59F772CEA35
:109D500035EC47E257E30E942ED787FD2AC020E06A
:109D600034E244E759ECC701B6010E9431D9181614
:109D70005CF4F5012081318142815381C701B60134
:109D80000E9431D9181604F120E034E244E759EC7E
:109D9000C301B2010E9431D918165CF4F50120818B
:109DA000318142815381C301B2010E942ED787FDC8
:109DB0000BC00B5C1F4FF4E0AF0EB11C8BE2CC3E2E
:109DC000D80709F0B0CF02C08CED01C080E0DF9170
:109DD000CF911F910F91FF90EF90DF90CF90BF90A8
:109DE000AF907F906F905F904F9008958091E22B9D
:109DF000811105C08091E12B8093E02B29C0823036
:109E000031F487E08093E02B8091E12B21C08330F7
:109E100031F489E08093E02B8091E12B19C08430EC
:109E200031F48AE08093E02B8091E12B11C0809186
:109E3000E32B813031F485E08093E02B8091E12B9E
:109E400007C0823019F486E08093E02B8091E12BEB
:109E5000863019F08091E02B08958BE08093E02B01
:109E600008958091E12B08958093E32B813059F080
:109E700018F0823041F0089581E19CE280930F2C2C
:109E80009093102C08958AE491E580930F2C909381
:109E9000102C0895FC0184810895845B9F4FFC0180
:109EA00080810895855B9F4FFC0180810895825BCE
:109EB0009F4FFC0180810895815B9F4FFC01808151
:109EC0000895875B9F4FFC01808108950C94269B29
:109ED000CD96FC0160817181828193810895FC019E
:109EE000648308958B5A9F4FFC01608308958F5BB4
:109EF0009F4FFC0140835183628373830895609375
:109F0000112C7093122C8093132C9093142C82EEAE
:109F100091E20C946266BF92CF92DF92EF92FF9231
:109F20000F931F93CF93DF93D0905E2C7C0103E8B7
:109F30001CE280915D2C90E0EC01CC0FDD1FC80F7E
:109F4000D91FCC0FDD1FCC0FDD1FCC0FDD1FC6507E
:109F5000D64D81E0D816A9F0B881A981CA80BB800E
:109F60004091D62C413091F4F80120813181428119
:109F700053816B2F7A2F8C2D9B2D0E9486D59B01B0
:109F800009C020E030E080E090E004C02B2F3A2FA1
:109F90008C2D9B2DA901BC01F701458F568F678F32
:109FA00070A3F4E0EF0EF11C0C5F1F4F24968CE2BF
:109FB0000B39180771F6DF91CF911F910F91FF9028
:109FC000EF90DF90CF90BF900895835B9F4FFC018F
:109FD000608381E19CE20C948B4F4F925F926F9271
:109FE0007F928F929F92AF92BF92CF92DF92EF9229
:109FF000FF920F931F93CF93DF93CDB7DEB7689790
:10A00000CDBFDEBF8C016091D62C70E080E090E087
:10A010000E94D0D72B013C01F801608171818281BF
:10A0200093810E94A2D770E05B01AA0CBB1CA60E14
:10A03000B71EAA0CBB1CAA0CBB1CAA0CBB1CC501DE
:10A040008650964D5C0103E81CE2FE0131964F01FB
:10A05000F501C190D190E190F1905F01F80161911B
:10A060007191819191918F01A30192010E94D3D9A5
:10A070009B01AC01C701B6010E9486D5F401619332
:10A080007193819391934F01FCE20B391F0701F704
:10A09000CE0101960E94099B81E19CE20E948B4FB8
:10A0A0006896CDBFDEBFDF91CF911F910F91FF90DA
:10A0B000EF90DF90CF90BF90AF909F908F907F9068
:10A0C0006F905F904F90089581519C4269F4E62F04
:10A0D000F0E0EE0FFF1FEE0FFF1FE559F34D60811B
:10A0E0007181828193810895862F0C94FE9ACF927C
:10A0F000DF92EF92FF920F931F93CF93DF93EC01C8
:10A100008CE2C131D80709F04AC070E0FB01EE0FC4
:10A11000FF1FEE0FFF1FE559F34DC080D180E28095
:10A12000F38080915E2C813059F180915D2C90E01C
:10A13000FC01EE0FFF1FE80FF91FEE0FFF1FE60FE8
:10A14000F71FEE0FFF1FEE0FFF1FE650F64D0081C9
:10A150001181B281A3812091D62C2130B1F4FB0171
:10A16000EE0FFF1FEE0FFF1FED57F34D20813181E2
:10A1700042815381B8018B2F9A2F0E9486D508C047
:10A1800060E070E080E090E003C0B8018B2F9A2F70
:10A190009B01AC01C701B6010E9485D503C0862F83
:10A1A0000E94129BC55BDF4F2881211106C023E36B
:10A1B00033E34BEC51E40E9435D7DF91CF911F91EF
:10A1C0000F91FF90EF90DF90CF90089588E1E6E146
:10A1D000FCE2ABE6BCE201900D928A95E1F780913A
:10A1E0005A2C81110CC08091152C813041F41092B1
:10A1F0004E2C10924F2C1092502C1092512C0895EE
:10A200004F925F926F927F928F929F92AF92BF9286
:10A21000CF92DF92EF92FF920F931F93CF93DF9332
:10A22000CDB7DEB76997CDBFDEBF8091E22B81113C
:10A2300055C08091072C813009F050C00E94F6C9AA
:10A2400081114CC01092072C92E1692E9AE2792E6E
:10A2500026E3822E912C8E010E5E1F4F30EEA32E30
:10A2600030E2B32E33C0F70181917F011F928F93AB
:10A270005F924F92BF92AF921F930F930E94D3E4CD
:10A28000B8018BE493E20E94C8638D839E83F6013C
:10A2900081919191A191B1916F018A879B87AC8740
:10A2A000BD87CE0101960E94DF60CDBFDEBF98ED75
:10A2B000E91690E2F906B9F6E8E16E0E711CFFEFBF
:10A2C0008F1A9F0A8CE38816910441F0240183EDD4
:10A2D000E82E80E2F82E630188E7C8CF80E0699617
:10A2E000CDBFDEBFDF91CF911F910F91FF90EF9017
:10A2F000DF90CF90BF90AF909F908F907F906F90A6
:10A300005F904F9008952F923F924F925F926F927D
:10A310007F928F929F92AF92BF92CF92DF92EF92F5
:10A32000FF920F931F93CF93DF93CDB7DEB729979B
:10A33000CDBFDEBF4C015B014090602C50905E2C85
:10A3400020905D2C6090D62C70905C2C6B0186E187
:10A350009CE28887998752EAE52E5AE2F52E98E129
:10A36000299E100111248401D6016D917D918D915A
:10A370009D916D012CEA35EC47E257E30E942ED700
:10A3800087FD80C0F70180818150823008F07AC05B
:10A3900041104CC0F1E05F1609F1E885F985E20D46
:10A3A000F31DEC51F2408081898391819D83B281BC
:10A3B000A381E1E06E1217C0E885F985E359FF4FEC
:10A3C0002081318142815381BC018B2F9A2F0E94C1
:10A3D00086D569837D838E839F8307C019821D8202
:10A3E0001E821F8202C0BE83AF8371100CC023E3A4
:10A3F00033E34BEC51E4D8016D917D918D919C91AB
:10A400000E94D3D905C0F801608171818281938156
:10A4100029813D814E815F810E9486D5A885B985BD
:10A420006D937D938D939C9313972CC0A885B985CC
:10A430008D919D910D90BC91A02D89839A83AB83C2
:10A44000BC8371100EC023E333E34BEC51E4F801FD
:10A4500060817181828193810E94D3D99B01AC017B
:10A4600005C0D8012D913D914D915C9169817A8112
:10A470008B819C810E9486D5E885F98560837183F4
:10A48000828393838885998504968887998795E345
:10A49000E90EF11C0C5F1F4FA885B985A252BC4282
:10A4A00009F062CF60905C2C7090602CF0915E2C73
:10A4B000F983C0905D2C2091D62C2D838CE0A80EC2
:10A4C000B11CA1E4BBE2A887B98742E2E42E4CE2CA
:10A4D000F42EB8E1CB9E600111248401F501619155
:10A4E0007191819191915F012CEA35EC47E257E33C
:10A4F0000E942ED787FD8CC0A885B9858C918823B2
:10A5000009F486C08150823030F4F8012484358407
:10A51000468457843BC0611016C023E333E34BEC01
:10A5200051E4D8011C966D917D918D919C911F975E
:10A530000E94D3D920E030E044EB53E40E94D3D909
:10A540001B012C010DC020E030E044EB53E4F80186
:10A5500064857585868597850E94D3D91B012C015A
:10A560002BED3FE049EC50E4A885B98591966D91BB
:10A570007D918D919C9194970E94D3D99B01AC01C0
:10A58000C201B1010E9435D71B012C01711031C0ED
:10A59000B981B130E1F0F701EC0DFD1DEC51F24055
:10A5A000A081B18192808380ED81E130A1F4F70137
:10A5B000E359FF4F2081318142815381BD01892DB3
:10A5C000982D0E9486D5DB01982E892E04C0A0E02C
:10A5D000B0E0912C812CA2019101BD01892D982D13
:10A5E0000E9486D5D7016D937D938D939C9313978D
:10A5F0000FC0A2019101F701608171818281938175
:10A600000E9486D5D7016D937D938D939C9313976C
:10A61000E885F985F596E887F987F4E0EF0EF11CF7
:10A620000C5F1F4F88859985805E9B4209F056CF4D
:10A630002996CDBFDEBFDF91CF911F910F91FF9083
:10A64000EF90DF90CF90BF90AF909F908F907F90D2
:10A650006F905F904F903F902F9008958091DE29EA
:10A660009091DF298F3E924111F08FE508958091FE
:10A67000952D9091962D8F3E9241B9F78091672C40
:10A680009091682C8F3E924181F78091DD2C9091C2
:10A69000DE2C8F3E924149F78091A2519091A351B7
:10A6A0008F3E924111F780915F52909160528F3EA0
:10A6B0009241D9F680E008958091E22B811104C087
:10A6C00083E08093E12B03C085E08093E12B80E061
:10A6D0000895CF93C82F0E94D4B680E00E9475B22F
:10A6E0008C2F0E94F7AB86E08093E12B8C2FCF91CB
:10A6F000089580935B2C80E0089580935C2C80E02B
:10A7000008958093602C80E00895AF92BF92CF921D
:10A71000DF92EF92FF920F931F93CF93DF939FEF00
:10A72000980F963008F041C0A0905C2C7A018B0104
:10A7300098E1899F60011124F601E252F64D6F0104
:10A74000C0E0D0E0BB24B394F70161917191819195
:10A7500091917F012CEA35EC47E257E30E9431D911
:10A760001816E4F4A1100CC023E333E34BEC51E4DE
:10A77000F80160817181828193810E94D3D905C0E3
:10A78000F8016081718182819381F601EC0FFD1FD8
:10A79000648F758F868F978FB092072C24960C5FED
:10A7A0001F4FC831D10581F602C08EE601C080E09E
:10A7B000DF91CF911F910F91FF90EF90DF90CF909D
:10A7C000BF90AF900895CF93DF93CDB7DEB7689772
:10A7D000CDBFDEBF80935D2C682F70E080E090E0FD
:10A7E0000E94CED769837A838B839C831D821E82CD
:10A7F0001F82188619861A861B861C861D861E8651
:10A800001F86188A198A1A8A1B8A1C8A1D8A1E8A20
:10A810001F8A188EAE014F5F5F4FBA018DEE9FE425
:10A820000E94678780E06896CDBFDEBFDF91CF9141
:10A830000895CF93DF93E1E1FCE286E5DF011D920D
:10A840008A95E9F78BE5AFEDBCE2ED01982F1992FF
:10A850009A95E9F7AAE3BDE2ED0119928A95E9F725
:10A860008FEE92E18093DE299093DF298093952DDE
:10A870009093962D8093672C9093682C8093DD2C79
:10A880009093DE2C8093A2519093A35180935F52BA
:10A8900090936052E0930F2CF093102C8091F72945
:10A8A00080935C2C8091F5290E94E3538091F629D6
:10A8B00080935B2C8091F82980935F2C8091F929FB
:10A8C0008093602C81E080935A2C8093D72C94E065
:10A8D0009093152C1092082C1092092C10920A2C8F
:10A8E0008093E12B8093E02B0E9413B1DF91CF91F5
:10A8F0000C94A988CF92DF92EF92FF92CF93C82F4A
:10A900006A017B01E82FF0E0DF01AA0FBB1FAA0F4D
:10A91000BB1FA559B34DCD92DD92ED92FC921397DA
:10A92000EE0FFF1FEE0FFF1FEA5EF34DC082D182D4
:10A93000E282F382B701A6010E941A86B701A6013E
:10A940008C2F0E942586CF91FF90EF90DF90CF90C3
:10A950000C9430869F92AF92BF92CF92DF92EF928B
:10A96000FF920F931F93CF93DF93CDB7DEB7689716
:10A97000CDBFDEBF962EA72EC62ED72E7C0100E0BF
:10A9800010E0B12CF60161917191819191916F016B
:10A990002CEA35EC47E257E30E9431D91816A4F5AA
:10A9A00080915C2C81110EC023E333E34BEC51E426
:10A9B000F70160817181828193810E94D3D9AB01BB
:10A9C000BC0105C0F7014081518162817381E1E0E2
:10A9D000F0E0EC0FFD1FE00FF11F40835183628315
:10A9E0007383C8018252964DFC01E357FD4F4083AB
:10A9F000518362837383E555F109408351836283F8
:10AA000073838B2D0E941A86B3940C5F1F4FF4E062
:10AA1000EF0EF11C0831110509F0B4CF492D5A2D64
:10AA2000BE016F5F7F4F80E99CE40E94678780E0F2
:10AA30006896CDBFDEBFDF91CF911F910F91FF9040
:10AA4000EF90DF90CF90BF90AF909F9008954F927E
:10AA50005F926F927F928F929F92AF92BF92CF92AE
:10AA6000DF92EF92FF920F931F93CF93DF93CDB7B7
:10AA7000DEB76897CDBFDEBF21E02093D62C809053
:10AA80005D2C90905C2C5B016C010BE61CE2882D28
:10AA900090E07C01EE0CFF1CE80EF91EEE0CFF1C92
:10AAA000EE0CFF1CEE0CFF1CC7018650964D7C017E
:10AAB000F50161917191819191915F012CEA35ECE1
:10AAC00047E257E30E9431D9181664F5F701208157
:10AAD000318142815381F80160817181828193814A
:10AAE0000E9485D52B013C0191100EC023E333E376
:10AAF0004BEC51E4F60160817181828193810E9467
:10AB0000D3D99B01AC0105C0F6012081318142817E
:10AB10005381C301B2010E9485D5F801608F718F06
:10AB2000828F938FF4E0CF0ED11C0C5F1F4F84E017
:10AB3000E80EF11C9CE20338190709F0B9CF682D23
:10AB400070E080E090E00E94CED769837A838B83A7
:10AB50009C831D821E821F82188619861A861B8678
:10AB60001C861D861E861F86188A198A1A8A1B8AC9
:10AB70001C8A1D8A1E8A1F8A188EAE014F5F5F4F86
:10AB8000BA018DEE9FE40E94678780E06896CDBF92
:10AB9000DEBFDF91CF911F910F91FF90EF90DF907B
:10ABA000CF90BF90AF909F908F907F906F905F906D
:10ABB0004F900895CF93DF93CDB7DEB76897CDBFA1
:10ABC000DEBF1092D62C1092832C1092842C1092FF
:10ABD000852C1092862C1092872C1092882C109223
:10ABE000892C10928A2C10928B2C10928C2C109203
:10ABF0008D2C10928E2C10928F2C1092902C1092E3
:10AC0000912C1092922C1092932C1092942C1092C2
:10AC1000952C1092962C1092972C1092982C1092A2
:10AC2000992C10929A2C60915D2C70E080E090E05D
:10AC30000E94CED769837A838B839C831D821E8278
:10AC40001F82188619861A861B861C861D861E86FC
:10AC50001F86188A198A1A8A1B8A1C8A1D8A1E8ACC
:10AC60001F8A188EAE014F5F5F4FBA018DEE9FE4D1
:10AC70000E94678780E06896CDBFDEBFDF91CF91ED
:10AC80000895CF93DF93CDB7DEB76897CDBFDEBF12
:10AC90001092D62C60915D2C70E080E090E00E94D4
:10ACA000CED769837A838B839C831D821E821F8209
:10ACB000188619861A861B861C861D861E861F8688
:10ACC000188A198A1A8A1B8A1C8A1D8A1E8A1F8A58
:10ACD000188EAE014F5F5F4FBA018DEE9FE40E9468
:10ACE000678780E06896CDBFDEBFDF91CF91089582
:10ACF000CF93DF93CDB7DEB76897CDBFDEBF81E0DE
:10AD00008093D62C60915D2C70E080E090E00E94F2
:10AD1000CED769837A838B839C831D821E821F8298
:10AD2000188619861A861B861C861D861E861F8617
:10AD3000188A198A1A8A1B8A1C8A1D8A1E8A1F8AE7
:10AD4000188EAE014F5F5F4FBA018DEE9FE40E94F7
:10AD5000678780E06896CDBFDEBFDF91CF91089511
:10AD6000CF931092152C0E9483518091E829813055
:10AD700069F486E19CE20E94804EC82F882331F05E
:10AD80000E94F7AB82E08093E12B17C081E19CE247
:10AD90000E948B4F85E08093E12B8091E22B811103
:10ADA00005C081E08093E22B0E946BAF81E19CE2C1
:10ADB0000E94339B0E94E650C0E08C2FCF910895F3
:10ADC00088E1EBE6FCE2ABE9BCE201900D928A95EA
:10ADD000E1F780E008950F931F93CF93DF93CDB7F2
:10ADE000DEB76A97CDBFDEBF8C0181E080935E2C19
:10ADF00081E19CE2698F7A8F0E948B4F698D7A8DF9
:10AE0000C8010E94B0560E94A1868823E1F388E120
:10AE1000E0E0F0E2DE01119601900D928A95E1F7F3
:10AE2000BE016F5F7F4F8BE99CE20E94B0566A962D
:10AE3000CDBFDEBFDF91CF911F910F91089588E1C3
:10AE4000EBE6FCE2A3EBBCE201900D928A95E1F700
:10AE500080E008950F931F93CF93DF93CDB7DEB7B4
:10AE60006A97CDBFDEBF8C0181E080935E2C81E1CB
:10AE70009CE2698F7A8F0E948B4F698D7A8DC80111
:10AE80000E94B0560E94A1868823E1F388E1E0E0A9
:10AE9000F0E2DE01119601900D928A95E1F7BE0174
:10AEA0006F5F7F4F83EB9CE20E94B0566A96CDBFE6
:10AEB000DEBFDF91CF911F910F910895FB01DC015F
:10AEC00080915A2C811111C09B01AD0160E070E0AE
:10AED00080E89FE30E9435D760934E2C70934F2CEF
:10AEE0008093502C9093512C18C080915C2C811130
:10AEF00009C023E333E34BEC51E4CD010E94D3D9E5
:10AF0000FB0101C0CD01AF01BC0140934E2C509319
:10AF10004F2C6093502C7093512C80E008958093B7
:10AF20005A2C80E0089580935F2C80E00895609310
:10AF3000562C7093572C8093582C9093592C0E9428
:10AF4000BF8780E008950F931F93CF93DF93EC01A9
:10AF50008B0180915A2C882399F080914E2C9091EE
:10AF60004F2CA091502CB091512CBC01CD019F775A
:10AF70002CEA35EC47E257E30E942ED787FD30C01C
:10AF800081E08093152CB801CE010E9483518091FD
:10AF9000E829813069F486E19CE20E94804EC82F46
:10AFA000882331F00E94F7AB82E08093E12B19C037
:10AFB00081E19CE20E948B4F85E08093E12B8091A0
:10AFC000E22B811105C081E08093E22B0E946BAFE0
:10AFD00081E19CE20E94339BC82F0E94E65001C091
:10AFE000CEE88C2FDF91CF911F910F910895CF93D1
:10AFF000DF93CDB7DEB76897CDBFDEBF682F70E0B7
:10B0000080E090E00E94CED769837A838B839C8313
:10B010001D821E821F82188619861A861B861C8630
:10B020001D861E861F86188A198A1A8A1B8A1C8A00
:10B030001D8A1E8A1F8A188EAE014F5F5F4FBA01AC
:10B040008CE79CE40E94678780E06896CDBFDEBFF6
:10B05000DF91CF910895CF93DF93CDB7DEB7689797
:10B06000CDBFDEBF6091632C70E080E090E00E9475
:10B07000CED769837A838B839C831D821E821F8235
:10B08000188619861A861B861C861D861E861F86B4
:10B09000188A198A1A8A1B8A1C8A1D8A1E8A1F8A84
:10B0A000188EAE014F5F5F4FBA0186E89CE40E94A4
:10B0B000678780E06896CDBFDEBFDF91CF910895AE
:10B0C000CF93DF93CDB7DEB76897CDBFDEBF682FD4
:10B0D00070E080E090E00E94CED769837A838B8312
:10B0E0009C831D821E821F82188619861A861B86E3
:10B0F0001C861D861E861F86188A198A1A8A1B8A34
:10B100001C8A1D8A1E8A1F8A188EAE014F5F5F4FF0
:10B11000BA018FEC9CE40E94678780E06896CDBFFF
:10B12000DEBFDF91CF910895CF93DF93CDB7DEB728
:10B130006897CDBFDEBF682F70E080E090E00E948E
:10B14000CED769837A838B839C831D821E821F8264
:10B15000188619861A861B861C861D861E861F86E3
:10B16000188A198A1A8A1B8A1C8A1D8A1E8A1F8AB3
:10B17000188EAE014F5F5F4FBA0180EE9CE40E94D3
:10B18000678780E06896CDBFDEBFDF91CF910895DD
:10B19000CF93FC0160817181828193810E94A2D74B
:10B1A0006093E12B1092E32B81E19CE280930F2CC2
:10B1B0009093102C8091E22B813011F41092E22BAD
:10B1C0001092E42B10920A2C0E94EC9AC091E12B71
:10B1D000C430C9F40E94DA558091F5290E94E353E6
:10B1E0008091F62980935B2C8091F9298093602CC3
:10B1F00080E00E9475B280E00E94945881E08093C4
:10B200005A2CC093152C81E0CF910C942FAE8093D3
:10B21000D32C8093D42C8093DC2C80E008952CEAEE
:10B2200035EC47E257E36091812D7091822D80913A
:10B23000832D9091842D0E9431D91816B4F48091F9
:10B24000262D9091272DA091282DB091292DBC015C
:10B25000CD019F772CEA35EC47E257E30E942ED7C9
:10B2600087FF03C01092D32C03C081E08093D32CBE
:10B2700080E008958093D32C8091262D9091272DE6
:10B28000A091282DB091292D8093CB2C9093CC2C7C
:10B29000A093CD2CB093CE2C80E008952CEA35EC11
:10B2A00047E257E36091812D7091822D8091832D2B
:10B2B0009091842D0E9431D91816B4F48091262DD6
:10B2C0009091272DA091282DB091292DBC01CD0161
:10B2D0009F772CEA35EC47E257E30E942ED787FF91
:10B2E00003C01092D42C03C081E08093D42C80E062
:10B2F00008958093D42C8091262D9091272DA09194
:10B30000282DB091292D8093CF2C9093D02CA093F1
:10B31000D12CB093D22C80E008952CEA35EC47E292
:10B3200057E36091812D7091822D8091832D9091B2
:10B33000842D0E9431D91816B4F48091262D909155
:10B34000272DA091282DB091292DBC01CD019F77EB
:10B350002CEA35EC47E257E30E942ED787FF03C063
:10B360001092DC2C03C081E08093DC2C80E00895F7
:10B370008093DC2C8091262D9091272DA091282D53
:10B38000B091292D8093D82C9093D92CA093DA2CAE
:10B39000B093DB2C80E00895BC0187EE90E20C9422
:10B3A000856681E08093082C089581E08093092CC4
:10B3B000089581E080930A2C08951F93CF93DF9323
:10B3C000CDB7DEB76897CDBFDEBF0E94269B813028
:10B3D000C9F10E94CCD30E94248780E00E9480AFF4
:10B3E0000E9489B010E0812F0E94FE9AAB01BC013F
:10B3F000812F0E947A541F5F1630A9F780E090E0F9
:10B40000A0E4B0E489839A83AB83BC831D821E824F
:10B410001F82188619861A861B861C861D861E8624
:10B420001F86188A198A1A8A1B8A1C8A1D8A1E8AF4
:10B430001F8A188EBE016F5F7F4FCB010E94C858D4
:10B4400080E001C08AE66896CDBFDEBFDF91CF9174
:10B450001F9108958091082C8130A9F42091E32B4D
:10B46000213079F48091E42B81110BC082E080932C
:10B47000E32B8AE491E580930F2C9093102C20937A
:10B48000E42B1092082C8091092C813091F480914A
:10B49000E32B882331F0823061F49091E42B9430D7
:10B4A00051F40E94269B811104C01092092C0E9425
:10B4B000DD599091E42B80910A2C8130C1F42091C8
:10B4C000092C211114C09150933088F010920A2C4D
:10B4D00095E09093E42B9093E12B9091E22B9111C6
:10B4E00004C08093E22B0E946BAF0E9498A380E07F
:10B4F000089585E08093E12B8091E22B811105C0B6
:10B5000081E08093E22B0C946BAF0895CF93DF938F
:10B51000CDB7DEB76897CDBFDEBF8091E22B882321
:10B5200011F180E090E0A0E4B0E489839A83AB83DA
:10B53000BC831D821E821F82188619861A861B866E
:10B540001C861D861E861F86188A198A1A8A1B8ADF
:10B550001C8A1D8A1E8A1F8A188EBE016F5F7F4F4C
:10B56000CB010E94C8586896CDBFDEBFDF91CF9156
:10B570000895CF93DF93CDB7DEB76897CDBFDEBF19
:10B5800080E090E0A0E4B0E489839A83AB83BC833D
:10B590001D821E821F82188619861A861B861C86AB
:10B5A0001D861E861F86188A198A1A8A1B8A1C8A7B
:10B5B0001D8A1E8A1F8A188EAE014F5F5F4FBA0127
:10B5C00088EC98E50E9467876896CDBFDEBFDF9163
:10B5D000CF910895CF93DF93CDB7DEB76897CDBFF6
:10B5E000DEBF80E090E0A0E8B0E489839A83AB837B
:10B5F000BC831D821E821F82188619861A861B86AE
:10B600001C861D861E861F86188A198A1A8A1B8A1E
:10B610001C8A1D8A1E8A1F8A188EAE014F5F5F4FDB
:10B62000BA0188EC98E50E9467876896CDBFDEBFB7
:10B63000DF91CF910895CF93DF93CDB7DEB72797F2
:10B64000CDBFDEBF97E0E9EDF0E2DE01119601909B
:10B650000D929A95E1F7873050F4E1E0F0E0EC0FBD
:10B66000FD1FE80FF11D87FDFA95808101C080E282
:10B670002796CDBFDEBFDF91CF910895EF92FF9265
:10B680000F931F93CF93DF931F92CDB7DEB77C014B
:10B690008B01642F70E080E090E049830E94CED758
:10B6A000F701618772878387948782E08783498166
:10B6B000E42FF0E0EE0FFF1FE00FF11F6591749192
:10B6C0004FE450E08BEF97E30E9441E3BC01C701D8
:10B6D0000F90DF91CF911F910F91FF90EF900C94FD
:10B6E0002766CF93DF93EC010E94F64E482F65EB5F
:10B6F00073E1CE01DF91CF910C943E5B4091E12B41
:10B7000066E773E10C943E5B4091E22B6DE473E1DC
:10B710000C943E5B4091E32B69E373E10C943E5B38
:10B720004091E42B6BE073E10C943E5B4091E52B80
:10B730006EEE72E10C943E5BE0910F2CF091102CB8
:10B74000E55BFF4F408168E174E10C943E5BE09162
:10B750000F2CF091102CE45BFF4F408164E272E10A
:10B760000C943E5BE0910F2CF091102C44816AE820
:10B7700071E10C943E5BE0910F2CF091102CE65B94
:10B78000FF4F408167E571E10C943E5BE0910F2C27
:10B79000F091102CE25BFF4F40816DE071E10C9461
:10B7A0003E5BE0910F2CF091102CE15BFF4F40814C
:10B7B0006CEC70E10C943E5BE0910F2CF091102C3E
:10B7C000E75BFF4F40816DE570E10C943E5BCF93EA
:10B7D000DF93EC01E0910F2CF091102CEF5AFF4F0A
:10B7E000608170E080E090E00E94CED769877A8720
:10B7F0008B879C8782E08F8380E0DF91CF910895D3
:10B80000CF93DF93EC016091112C7091122C8091F9
:10B81000132C9091142C0E94CED769877A878B873E
:10B820009C8782E08F8380E0DF91CF910895CF9352
:10B83000DF93EC01E0910F2CF091102C608171816D
:10B84000828193810E94CED769877A878B879C8774
:10B8500082E08F8380E0DF91CF910895CF93DF93D3
:10B86000EC018091E32B811105C019861A861B8695
:10B870001C8614C00E94F59A69877A878B879C87FB
:10B880002091955121110AC025E832E441E25DE39F
:10B890000E94D3D969877A878B879C878C819D8109
:10B8A000FC01EE0FFF1FE80FF91FEE0FFF1FEE0F59
:10B8B000FF1FEE0FFF1FED50FA4E85919491888780
:10B8C00084E08F8380E0DF91CF910895CF93DF9361
:10B8D000EC0120910F2C3091102CF901FD96608124
:10B8E00071818281938169877A878B879C873E9655
:10B8F000208121110AC025E832E441E25DE30E9483
:10B90000D3D969877A878B879C878C819D81FC013D
:10B91000EE0FFF1FE80FF91FEE0FFF1FEE0FFF1FC7
:10B92000EE0FFF1FED50FA4E85919491888784E0C9
:10B930008F8380E0DF91CF910895CF93DF93EC0167
:10B940008C819D810E94084D682F80910F2C9091D1
:10B95000102C0E94775069877A878B879C878C810F
:10B960009D81FC01EE0FFF1FE80FF91FEE0FFF1F77
:10B97000EE0FFF1FEE0FFF1FED50FA4E85919491D1
:10B98000888784E08F8380E0DF91CF910895CF9303
:10B99000DF93EC018C819D810E94084D20910F2C3A
:10B9A0003091102C21513C4269F4E82FF0E0EE0F69
:10B9B000FF1FEE0FFF1FE559F34D608171818281FA
:10B9C000938102C00E94FE9A69877A878B879C8741
:10B9D0008C819D81FC01EE0FFF1FE80FF91FEE0F18
:10B9E000FF1FEE0FFF1FEE0FFF1FED50FA4E859168
:10B9F0009491888784E08F8380E0DF91CF910895D0
:10BA0000CF93DF93EC018C819D810E94084DE091E2
:10BA10000F2CF091102C94E0899FE00DF11D112462
:10BA2000458D568D678D70A149875A876B877C87B6
:10BA30008C819D81FC01EE0FFF1FE80FF91FEE0FB7
:10BA4000FF1FEE0FFF1FEE0FFF1FED50FA4E859107
:10BA50009491888784E08F8380E0DF91CF9108956F
:10BA6000CF93DF93EC010E94C26169857A858B8553
:10BA70009C850E94A2D7462F64E474E1CE01DF9139
:10BA8000CF910C943E5BCF93DF93EC018C819D8131
:10BA90000E94084D833054F48F3FA9F407C0CE01B3
:10BAA0000E946C6280E01CC08DE61AC020E030E08D
:10BAB00040E450E469857A858B859C850E9431D964
:10BAC000181694F3ECCF20E030E040E050E46985B4
:10BAD0007A858B859C850E9431D918162CF3DFCF8F
:10BAE000DF91CF91089595E3899FF0011124ED54E2
:10BAF000F54D60817181828193810895CF92DF92AB
:10BB0000EF92FF92CF93DF936A017B0125E3829F3F
:10BB1000C00111248252964DFC01EB52FF4F40832D
:10BB2000518362837383EC01C352DF4F20E034E220
:10BB300044E759E4C701B6010E94D3D99B01AC0187
:10BB400060E070E080E89FE30E9435D768837983E6
:10BB50008A839B83DF91CF91FF90EF90DF90CF900E
:10BB60000895CF92DF92EF92FF92CF93DF93EC0193
:10BB7000C984DA84EB84FC8420E034E244E759E4AD
:10BB8000C701B6010E9431D9181664F420E034E2EE
:10BB900044E759E4C701B6010E9435D769877A871F
:10BBA0008B879C87CE010E943A67C984DA84EB8434
:10BBB000FC848C819D810E94084D25E3829FC001F9
:10BBC00011248252964DFC01EB52FF4FC082D1826C
:10BBD000E282F382EC01C352DF4F20E034E244E71B
:10BBE00059E4C701B6010E94D3D99B01AC0160E0C2
:10BBF00070E080E89FE30E9435D7688379838A8369
:10BC00009B8380E0DF91CF91FF90EF90DF90CF900A
:10BC10000895CF92DF92EF92FF92CF93DF93EC01E2
:10BC2000C984DA84EB84FC8420E034E244E759E4FC
:10BC3000C701B6010E9431D9181664F420E034E23D
:10BC400044E759E4C701B6010E9435D769877A876E
:10BC50008B879C87CE010E943A6780E0DF91CF916D
:10BC6000FF90EF90DF90CF90089581E08093092CB2
:10BC700080E008952CEA35EC47E257E3FC0161854A
:10BC80007285838594850E9431D9181614F40E9418
:10BC9000136F80E0089560910B2C70910C2C8091B3
:10BCA0000D2C90910E2C08950E94516380E00E940B
:10BCB000967180E008950E94516381E00E94967120
:10BCC00080E008950E94516382E00E94967180E0B6
:10BCD00008950E94516383E00E94967180E0089568
:10BCE000CF93DF93EC01E0910F2CF091102CE55BEA
:10BCF000FF4FE081F0E0EE0FFF1FE958FB4E65912A
:10BD000074914FE450E08BEF97E30E9441E3AC0164
:10BD100066E470E1CE01DF91CF910C94E2C5CF9340
:10BD2000DF93EC01E0910F2CF091102CE55BFF4FBD
:10BD3000E081F0E0EE0FFF1FE958FB4E6591749132
:10BD40004FE450E08BEF97E30E9441E3AC016EE2D9
:10BD500070E1CE01DF91CF910C94E2C5CF93DF93D8
:10BD6000EC018BEE90E20E94A6E4CE010E94705E90
:10BD7000CE010E948F5E6AE170E1CE010E94A9C5EA
:10BD800061E070E1CE010E9474C568EE7FE0CE01F3
:10BD90000E9474C56FEC7FE0CE010E9474C566EB13
:10BDA0007FE0CE010E9474C56DE97FE0CE010E9464
:10BDB00074C564E87FE0CE010E9474C56BE67FE045
:10BDC000CE010E9474C562E57FE0CE010E9474C579
:10BDD00069E37FE0CE010E9474C560E27FE0CE019E
:10BDE0000E9474C567E07FE0CE010E9474C56EEECC
:10BDF0007EE0CE010E9474C565ED7EE0CE010E941A
:10BE000074C56CEB7EE0CE010E94A9C580E0DF9195
:10BE1000CF9108956AE170E10C94A9C561E070E1E9
:10BE20000C9474C568EE7FE00C9474C56FEC7FE0F1
:10BE30000C9474C566EB7FE00C9474C56DE97FE0EB
:10BE40000C9474C564E87FE00C9474C56BE67FE0E5
:10BE50000C9474C562E57FE00C9474C569E37FE0DF
:10BE60000C9474C560E27FE00C9474C567E07FE0D9
:10BE70000C9474C56EEE7EE00C9474C565ED7EE0A6
:10BE80000C9474C56CEB7EE00C94A9C560E47EE074
:10BE90000C94A9C56FE07EE00C94A9C56AED7DE025
:10BEA0000C94A9C56FE97DE00C94A9C56BE67DE013
:10BEB0000C94A9C5CF93DF93EC01E0910F2CF09186
:10BEC000102CE55BFF4FE081F0E0EE0FFF1FE9581B
:10BED000FB4E659174914FE450E08BEF97E30E9425
:10BEE00041E3AC0167E47DE0CE01DF91CF910C949A
:10BEF000E2C5CF93DF93EC01E0910F2CF091102C71
:10BF0000E55BFF4FE081F0E0EE0FFF1FE958FB4ECD
:10BF1000659174914FE450E08BEF97E30E9441E309
:10BF2000AC0166E27DE0CE01DF91CF910C94E2C5D9
:10BF300069E07DE00C948AC5CF93DF93EC01E0913A
:10BF40000F2CF091102CE55BFF4FE081F0E0EE0F3D
:10BF5000FF1FE958FB4E659174914FE450E08BEF61
:10BF600097E30E9441E3AC016AEE7CE0CE01DF91F1
:10BF7000CF910C94E2C50F931F93CF93DF938C0165
:10BF8000FC0161857285838594850E94A2D7E62F86
:10BF9000F0E0EE0FFF1FEC5BFB4E659174914FE4F8
:10BFA00050E08BEF97E30E9441E3E8012D969F93C9
:10BFB0008F93F80161857285838594850E94A2D74D
:10BFC0001F926F93DF93CF930F5E1F4F1F930F93BB
:10BFD000DF93CF938EEC9CE09F938F93E5E0F5E5A4
:10BFE00081818F9380818F930E9408E4EDB7FEB723
:10BFF0003E96EDBFFEBFDF91CF911F910F91089547
:10C0000066EA7CE00C947A4D6EE77CE00C947A4D05
:10C010006CE57CE00C947A4D6AE37CE00C947A4DFC
:10C0200068E07CE00C947A4D67ED7BE00C947A4DEF
:10C030006EE97BE00C947A4D6EE77BE00C947A4DD0
:10C040006CE37BE00C94484D6AEF7AE00C94484D29
:10C0500063ED7AE00C947A4D6DEA7AE00C947A4DB7
:10C060006CE87AE00C947A4D6CE67AE00C947A4DA8
:10C070006FE47AE00C94CD4D60E37AE00C94CD4D02
:10C08000BC01675F7F4F20915C2C46EA5EE0FC01BB
:10C09000848195810C94244EBC01675F7F4F21E021
:10C0A0004CE85EE0FC01848195810C94244EBC0137
:10C0B000675F7F4F21E043E75EE0FC01848195816B
:10C0C0000C94244E0F931F93CF93DF93EC010C81BC
:10C0D0001D810E94ED6808171907C0F48C819D81AD
:10C0E000FC01EE0FFF1FE80FF91FEE0FFF1FEE0F11
:10C0F000FF1FEE0FFF1FE850FA4E25913491CE013D
:10C10000F901DF91CF911F910F91199485E1DF9192
:10C11000CF911F910F9108950F931F93CF93DF93AA
:10C12000EC010C811D810E94ED6808171907C0F40D
:10C130008C819D81FC01EE0FFF1FE80FF91FEE0FB0
:10C14000FF1FEE0FFF1FEE0FFF1FEA50FA4E259163
:10C150003491CE01F901DF91CF911F910F91199484
:10C1600085E1DF91CF911F910F9108950F931F9358
:10C17000CF93DF93EC010C811D810E94ED680817BD
:10C180001907C0F48C819D81FC01EE0FFF1FE80FA1
:10C19000F91FEE0FFF1FEE0FFF1FEE0FFF1FEC50FA
:10C1A000FA4E25913491CE01F901DF91CF911F9183
:10C1B0000F911994DF91CF911F910F910895CF9313
:10C1C000DF93EC018C819D810E9400698823C9F076
:10C1D0008C819D81FC01EE0FFF1FE80FF91FEE0F10
:10C1E000FF1FEE0FFF1FEE0FFF1FEE50FA4EE49100
:10C1F000E1FF05C0CE01DF91CF910C94408580E036
:10C2000001C085E1DF91CF9108950F931F93CF93E4
:10C21000DF93EC0181E00E947D531C821D8280E04F
:10C2200090E08E010F5E1F4F47C08C819D819C0165
:10C23000220F331FF901E80FF91FEE0FFF1FEE0F5A
:10C24000FF1FEE0FFF1FEE50FA4EE491E0FF2EC0ED
:10C25000280F391F220F331F220F331F220F331FC6
:10C2600024503A4EF9014591559165917491498751
:10C270005A876B877C87BC01660F771F680F791F11
:10C28000660F771F660F771F660F771F64517A4E10
:10C2900045E050E0C8010E9441E3CE010E94626087
:10C2A000CE010E94DF602C813D8101C09C012F5F87
:10C2B0003F4F2C833D83C9010E94F0688111B5CFA7
:10C2C0000E94ADACDF91CF911F910F910C9465ACA2
:10C2D000CF93DF93EC012CEA35EC47E257E3698515
:10C2E0007A858B859C850E942ED787FF05C0CE015D
:10C2F000DF91CF910C94F57DCE010E94056182E023
:10C300008F8340E050E060E87FE349875A876B877E
:10C310007C8780E0DF91CF9108958091D733909111
:10C32000D8338F3E924111F08AE5089580911F34F1
:10C33000909120348F3E9241B9F78091AD2E90912B
:10C34000AE2E8F3E924181F78091CF319091D031C6
:10C350008F3E924149F78091D1319091D2318F3EF9
:10C36000924111F78091D5339091D6338F3E92410F
:10C37000D9F680914A388111D7CF0895FC011782F0
:10C3800089E60895CF93DF93EC018C819D81FC01B8
:10C39000EE0FFF1FE80FF91FEE0FFF1FEE0FFF1F3D
:10C3A000EE0FFF1FE650FA4EA591B4916C9170E02C
:10C3B00080E090E00E94CED769877A878B879C8740
:10C3C00082E08F8380E0DF91CF910895CF93DF9358
:10C3D000EC018C819D81FC01EE0FFF1FE80FF91F1E
:10C3E000EE0FFF1FEE0FFF1FEE0FFF1FE650FA4E7E
:10C3F000A591B4916D917D918D919C910E94CED724
:10C4000069877A878B879C8782E08F8380E0DF91C2
:10C41000CF910895CF93DF93DC0114968D919C9179
:10C420001597FC01EE0FFF1FE80FF91FEE0FFF1F1E
:10C43000EE0FFF1FEE0FFF1FE650FA4EC591D4918D
:10C44000488159816A817B8119964D935D936D93E3
:10C450007C931C9783E017968C9380E0DF91CF91BB
:10C460000895CF93DF93DC0114968D919C911597DD
:10C47000FC01EE0FFF1FE80FF91FEE0FFF1FEE0F7D
:10C48000FF1FEE0FFF1FE650FA4EC591D491488171
:10C4900059816A817B8119964D935D936D937C934D
:10C4A0001C97FC01EE0FFF1FE80FF91FEE0FFF1F97
:10C4B000EE0FFF1FEE0FFF1FED50FA4E8591949186
:10C4C00018968C93189784E017968C9380E0DF91F0
:10C4D000CF91089588E608950F931F93CF93DF932C
:10C4E000EC018C819D81FC01EE0FFF1FE80FF91F0D
:10C4F000EE0FFF1FEE0FFF1FEE0FFF1FE650FA4E6D
:10C500000591149169857A858B859C850E94A2D7B7
:10C51000F801608382E08F8380E0DF91CF911F91EB
:10C520000F910895CF93DF93EC0169857A858B8510
:10C530009C850E94A2D76230B0F48C819D81FC0161
:10C54000EE0FFF1FE80FF91FEE0FFF1FEE0FFF1F8B
:10C55000EE0FFF1FE650FA4EA591B4916C9382E066
:10C560008F8380E001C08EE6DF91CF910895CF9355
:10C57000DF93EC0169857A858B859C850E94A2D723
:10C580006330B0F48C819D81FC01EE0FFF1FE80F3A
:10C59000F91FEE0FFF1FEE0FFF1FEE0FFF1FE650FC
:10C5A000FA4EA591B4916C9382E08F8380E001C034
:10C5B0008EE6DF91CF910895CF93DF93EC016985EB
:10C5C0007A858B859C850E94A2D76430B0F48C81DB
:10C5D0009D81FC01EE0FFF1FE80FF91FEE0FFF1FFB
:10C5E000EE0FFF1FEE0FFF1FE650FA4EA591B4911C
:10C5F0006C9382E08F8380E001C08EE6DF91CF9163
:10C6000008950F931F93CF93DF93EC018C819D814D
:10C61000FC01EE0FFF1FE80FF91FEE0FFF1FEE0FDB
:10C62000FF1FEE0FFF1FE650FA4E0591149169852A
:10C630007A858B859C850E94A2D7F80160837183DF
:10C640008283938382E08F8380E0DF91CF911F917B
:10C650000F910895CF93DF93DC0114968D919C91F7
:10C660001597FC01EE0FFF1FE80FF91FEE0FFF1FDC
:10C67000EE0FFF1FEE0FFF1FE650FA4EC591D4914B
:10C6800019964D915D916D917C911C9748835983CA
:10C690006A837B8383E017968C9380E0DF91CF9150
:10C6A0000895CF93DF93DC0114968D919C9115979B
:10C6B000FC01EE0FFF1FE80FF91FEE0FFF1FEE0F3B
:10C6C000FF1FEE0FFF1FE650FA4EC591D491199649
:10C6D0004D915D916D917C911C97488359836A833C
:10C6E0007B83FC01EE0FFF1FE80FF91FEE0FFF1F0A
:10C6F000EE0FFF1FEE0FFF1FED50FA4E8591949144
:10C7000018968C93189784E017968C9380E0DF91AD
:10C71000CF9108951F93CF93DF93EC018091D9338C
:10C720008823D1F01DE10A80DB81C02D209711F410
:10C7300080E013C08F818F3FD9F3811104C0CE01F7
:10C740000E948C6006C0CE010E946260CE010E94F1
:10C75000DF60115041F7ECCF85E6DF91CF911F915B
:10C760000895CF93DF93EC01BC0189EF90E20E9422
:10C770007AE3892B41F0BE018CEF90E20E947AE3CC
:10C7800021E0892B09F420E0822FDF91CF910895D9
:10C790000F931F93CF93DF93CDB7DEB72997CDBF0C
:10C7A000DEBF8B0144E050E0BC01CE0101960E9447
:10C7B0009AE346E050E0B801CE0101960E948AE378
:10C7C0000E94ED68009709F43FC07981AA81BB817E
:10C7D0001C810D812CEE35E140E050E0F9016491BF
:10C7E000671327C03196E491E11103C0A11121C064
:10C7F00029C0EA131EC0F9013296E491E11103C089
:10C80000B11117C01FC0EB1314C0F9013396E491A6
:10C81000E11103C011110DC015C0E1130AC0F901E7
:10C820003496E491E11103C0011103C00BC0E0177D
:10C8300049F04F5F5F4F285E3F4F4817590709F097
:10C84000CDCF02C0CA0102C08FEF9FEF2996CDBFA6
:10C85000DEBFDF91CF911F910F910895CF93DF93AA
:10C86000FC012189222371F1EC016196BE0180E077
:10C8700091E20E947AE3892B39F1BE0189EF90E2BF
:10C880000E947AE3892B11F1BE0183E091E20E94BC
:10C890007AE3892BD9F0BE0187EE90E20E947AE319
:10C8A000892BB1F0BE0186E091E20E947AE3892BE8
:10C8B00079F0BE0182EE91E20E947AE3892B51F475
:10C8C00085E009C080E007C082E005C083E003C0C6
:10C8D00084E001C081E0DF91CF910895FC018FEFEA
:10C8E0008783148215821186128613861486108619
:10C8F000118A1586178A108EA081B181109711F4C4
:10C9000016820DC017968C911797873029F41696CA
:10C910008C918F5F868303C016968C918683CF019E
:10C920000895EF92FF920F931F93CF93DF93EC0143
:10C930000C811D810E94ED680817190708F06FC06F
:10C940000C811D81CE010E946E640C831D837E01CB
:10C9500081E1E80EF11CB801660F771F600F711FAF
:10C96000660F771F660F771F660F771F64517A4E29
:10C97000C7010E9422E38E01035F1F4F2C813D817E
:10C98000B901660F771F620F731F660F771F660F5F
:10C99000771F660F771F68517A4EC8010E9422E305
:10C9A0008D85882311F18C819D81FC01EE0FFF1F85
:10C9B000E80FF91FEE0FFF1FEE0FFF1FEE0FFF1F17
:10C9C000EE50FA4EE491E2FF02C01D8610C0F8015D
:10C9D00001900020E9F7BF01601B710B605F7F4F82
:10C9E0006C0F7D1FC7010E9483E38C819D81FC0138
:10C9F000EE0FFF1FE80FF91FEE0FFF1FEE0FFF1FD7
:10CA0000EE0FFF1FEA50FA4E25913491CE01F90145
:10CA1000DF91CF911F910F91FF90EF901994DF91CB
:10CA2000CF911F910F91FF90EF9008958F929F9259
:10CA3000AF92BF92CF92DF92EF92FF920F931F932C
:10CA4000CF93DF9300D01F92CDB7DEB76C015C01AE
:10CA500081E1A80EB11C87E0F6018783A8EEEA2EDB
:10CA6000A5E1FA2E00E010E01DC0B701CE0101964D
:10CA70000E9422E3BE016F5F7F4FC5010E947AE3EF
:10CA8000892B59F44601F9E18F0E911CF601058FAF
:10CA9000168FC4010E94916464010F5F1F4FF8E17B
:10CAA000EF0EF11CC8010E94F0688111DECF2496C0
:10CAB000CDBFDEBFDF91CF911F910F91FF90EF901F
:10CAC000DF90CF90BF90AF909F908F900895CF93BD
:10CAD000DF931092D3311092D431A6E9BEE2EFEA8F
:10CAE000FEE291E08FEFA083B18379965B96ED93A0
:10CAF000FC935C975D961D921C925E97EF01639785
:10CB0000988322961882219788832A9618825996AC
:10CB100021E3EF3CF20739F71092B8311092B931A6
:10CB20001092AF2E1092B02E1092B52E87E0809307
:10CB3000B62E82E790E08093C02E9093C12E88ECB1
:10CB40009EE2DF91CF9108950F931F93CF93DF93D0
:10CB50000E946765EC018FEE92E18093D73390934A
:10CB6000D83380931F34909320348093AD2E9093CC
:10CB7000AE2E8093CF319093D0318093D13190936A
:10CB8000D2318093D5339093D63381E00E947D5388
:10CB90001C821D82CE010E9417852091283430917D
:10CBA000293440912A3450912B3469857A858B85BC
:10CBB0009C850E942ED7882339F0CE01DF91CF913A
:10CBC0001F910F910C9405610E946AAC1C821D821A
:10CBD00080E090E08E010F5E1F4F2FC06C817D8141
:10CBE0009B01220F331FF901E60FF71FEE0FFF1F06
:10CBF000EE0FFF1FEE0FFF1FEE50FA4EE491E0FF25
:10CC000017C0620F731F660F771F660F771F660FBF
:10CC1000771F64517A4E45E050E0C8010E9441E31D
:10CC2000CE010E941785CE010E9462606C817D81D9
:10CC30006F5F7F4F6C837D83CB010E94F068811111
:10CC4000CDCFDF91CF911F910F910C94ADACEF92AE
:10CC5000FF920F931F93CF93DF938C012091D331D9
:10CC60003091D431EB0109900020E9F72197C61BE0
:10CC7000D70BAE01420F531F41305240D8F4F90197
:10CC8000EB52FE4C7F01AE014F5F5F4FCF010E9420
:10CC90005BE34091D3315091D4314F5F5F4F4C0FE4
:10CCA0005D1F4093D3315093D431F801E78AF08E61
:10CCB00080E001C08DE0DF91CF911F910F91FF9037
:10CCC000EF900895CF93DF932EE1C8ECDEE23F8131
:10CCD0003F3F59F00A80DB81C02D209719F480E096
:10CCE00090E010C0215099F7FACFBC018BE493E299
:10CCF0000E94C8638C839D83019689F3CE010E94B4
:10CD00009164CE01DF91CF910895EF92FF920F933E
:10CD10001F93CF93DF938B012EE1C8ECDEE23F81BE
:10CD20003F3F59F00A80DB81C02D209719F480E045
:10CD300090E01DC0215099F7FACF7E0121E1E20E6B
:10CD4000F11C45E050E0BC01C7010E949AE3B80124
:10CD5000CE010E9427668111EACFB7018BE493E2EE
:10CD60000E94C8638C839D8385E08F83CE01DF9111
:10CD7000CF911F910F91FF90EF9008952091D9339B
:10CD8000213021F42091F737213029F4BC0187EEBE
:10CD900090E20C94856680E090E008959091D933FC
:10CDA000913019F4642F0C9493830C94F4C40F9372
:10CDB0001F93CF93DF93CDB7DEB7C058D109CDBF56
:10CDC000DEBFFC0161857285838594850E94A2D7B0
:10CDD0008FEF860F863030F08AE391E20E94BE66C4
:10CDE0008EE62AC06093DD3381E08093DE33E62F48
:10CDF000F0E0EE0FFF1FED54FA4E659174914FE491
:10CE000050E08BEF97E30E9441E39F938F938AE872
:10CE100094E19F938F938E010F5F1F4F1F930F938A
:10CE20000E94FCE4C8010E94BE660F900F900F9014
:10CE30000F900F900F9080E0C058DF4FCDBFDEBF46
:10CE4000DF91CF911F910F910895CF93DF93EC0164
:10CE50000E94C4D3682F70E080E090E00E94CED79B
:10CE600069877A878B879C8782E08F8380E0DF9158
:10CE7000CF9108950F931F93CF93DF93EC0181E13E
:10CE80009CE20E94524F882329F009851A858B85E0
:10CE90009C8511C023E333E34BEC51E469857A852B
:10CEA0008B859C850E94D3D98B01AB01BC0149873E
:10CEB0005A876B877C872C813D81F901EE0FFF1F1C
:10CEC000E20FF31FEE0FFF1FEE0FFF1FEE0FFF1F0E
:10CED000E650FA4EA591B491A801BC014D935D9323
:10CEE0006D937C931397F901EE0FFF1FE20FF31F71
:10CEF000EE0FFF1FEE0FFF1FEE0FFF1FED50FA4E5C
:10CF000085919491888784E08F8380E0DF91CF9131
:10CF10001F910F91089564E875E10C948AC560E64D
:10CF200075E10C948AC563E275E10C948AC566EDDF
:10CF300074E10C948AC563EB74E10C948AC51F9369
:10CF4000CF93DF93EC0110E08881882301F10E94E8
:10CF5000676545E050E0BE0189ED9EE20E949AE3DC
:10CF600069ED7EE28BE493E20E94C8638093CC2E4D
:10CF70009093CD2E88EC9EE20E94916442E063E0A3
:10CF800080E00E94CE661F5F26961D31E9F684E0A0
:10CF9000DF91CF911F910895CF93DF93CDB7DEB787
:10CFA000EC97CDBFDEBF8CE3E8E1F0E2DE01119645
:10CFB00001900D928A95E1F7CE0101960E949F673C
:10CFC000EC96CDBFDEBFDF91CF910895CF93DF9375
:10CFD000CDB7DEB7AA97CDBFDEBF8AE2E4E5F0E2C7
:10CFE000DE01119601900D928A95E1F7CE0101962E
:10CFF0000E949F67AA96CDBFDEBFDF91CF910895B3
:10D00000CF93DF93CDB7DEB76E97CDBFDEBF8EE196
:10D01000EEE7F0E2DE01119601900D928A95E1F7BC
:10D02000CE0101960E949F676E96CDBFDEBFDF9155
:10D03000CF910895CF93DF93EC0143E759E763E77E
:10D0400070E0498B5A8B6B8B7C8B0E94166542E09B
:10D0500063E080E00E94CE66CE010E940068CE01AF
:10D060000E94E66720E731E340E0298B3A8B4B8B47
:10D07000CE010E94166542E063E080E00E94CE6629
:10D08000CE01DF91CF910C94CC67CF92DF92EF92DB
:10D09000FF92FC01C184D284E384F48420E030E078
:10D0A00040E85FE3C701B6010E9431D91816FCF0D1
:10D0B000C701B6010E94A2D76093DA33C701B60157
:10D0C0009F772CEA35EC47E257E30E9431D91816D6
:10D0D0003CF460E470E080E00E9491CA80E008C007
:10D0E00060E870E080E00E9491CA80E001C08EE6B6
:10D0F000FF90EF90DF90CF900895CF92DF92EF9264
:10D10000FF92FC01C184D284E384F48420E030E007
:10D1100040E050E4C701B6010E9431D91816FCF076
:10D12000C701B6010E94A2D76093DC33C701B601E4
:10D130009F772CEA35EC47E257E30E9431D9181665
:10D140003CF464E070E080E00E9491CA80E008C096
:10D1500068E070E080E00E9491CA80E001C08EE645
:10D16000FF90EF90DF90CF900895CF92DF92EF92F3
:10D17000FF92FC01C184D284E384F48420E030E097
:10D1800040E85FE3C701B6010E9431D91816FCF0F0
:10D19000C701B6010E94A2D76093DB33C701B60175
:10D1A0009F772CEA35EC47E257E30E9431D91816F5
:10D1B0003CF460E170E080E00E9491CA80E008C029
:10D1C00060E270E080E00E9491CA80E001C08EE6DB
:10D1D000FF90EF90DF90CF90089585E991E008955A
:10D1E00021E08C34914008F020E0822F08959C01CA
:10D1F0002856314081E02932310508F080E0089559
:10D2000021E08936914008F020E0822F0895CF92E6
:10D21000DF92EF92FF92CF93DF93EC01C984DA841F
:10D22000EB84FC84A7019601C701B6010E94F4DAE1
:10D2300081113CC0E894F7F82FEF3FEF4FE75FE72D
:10D24000C701B6010E94F4DA81110AC02FEF3FEF47
:10D250004FE75FE7C701B6010E942ED7181634F1D9
:10D260008C819D81FC01EE0FFF1FE80FF91FEE0F6F
:10D27000FF1FEE0FFF1FEE0FFF1FEE50FA4EE4915F
:10D28000E3FF14C081E19CE20E94524F81110EC065
:10D2900025E832E441E25DE369857A858B859C85EA
:10D2A0000E94D3D969877A878B879C87DF91CF913A
:10D2B000FF90EF90DF90CF9008958091DE33882328
:10D2C00049F01092DE336091DD3380E00E9499CA0C
:10D2D00080E0089583E00895FF920F931F93CF930A
:10D2E000DF931F921F92CDB7DEB7F82EE1E2F4E391
:10D2F00022EA33E0DF01C9011D920197E9F72FEE21
:10D3000032E1208331832093C1373093C23701EE5D
:10D310001AE12CED33E40093283410932934209340
:10D320002A3430932B340CEE11E528E73FE30093C9
:10D330002C3410932D3420932E3430932F3400E06E
:10D3400010E020E83FE30093303410933134209311
:10D3500032343093333483E0809323348F2D4A83E7
:10D3600069830E94A9CA6981862F0E94B4CA4A8132
:10D37000842F0E94BFCAF0923A34F09238340F9052
:10D380000F90DF91CF911F910F91FF900895CEE5FF
:10D39000D4E310E60E94B37C8230E1F30E94BA7CB1
:10D3A0008230C1F30E94314F863009F052C10E9491
:10D3B0006EC9C0904534D0904634E0904734F09028
:10D3C0004834C616D706E806F90620F70E946EC94B
:10D3D0006C597F4F8F4F9F4F609345347093463405
:10D3E00080934734909348340E94297CD3CF0E9485
:10D3F00002C0882329F08CEC0E946953823051F2DC
:10D400000E942A5A823031F20E94F2A1823011F237
:10D410000E948D6180934B3881112EC08091213400
:10D42000909122348F3E924109F019C18091C13709
:10D430009091C2378F3E924109F011C116C10E94EE
:10D44000EC8580934B38811117C00E948FB6809372
:10D450004B38811111C00E942B7480934B3881117D
:10D460000BC00E94AFC980934B38811105C00E9448
:10D4700063B7823031F48ECF0E9469538230B9F79E
:10D4800089CF0E9461AE823009F484CF0E94CDAF73
:10D49000823009F47FCF0E9494B0823009F47ACFB1
:10D4A0000E945190823009F475CF0E94626F8230E1
:10D4B00009F470CF0E942172823009F46BCF0E9470
:10D4C0000674823009F466CF0E940051823009F45C
:10D4D00061CF0E94A186843008F0D1C05BCF4FEFAE
:10D4E00050E06EE574E3809138340E9447CA8111A0
:10D4F00039C0C0935C34D0935D34FE0101900020AC
:10D50000E9F7EE55F443E0933C34F0933D3443E6C1
:10D5100050E06EE574E38DE597E30E949AE3809115
:10D520005E3490E00E941AE385329105F1F154F4E3
:10D5300081329105B9F18432910509F447C0892BF4
:10D54000D1F157C08834910509F440C01CF4CF973D
:10D55000E9F14FC08B37910509F443C08E3791052F
:10D5600039F147C0883009F015CF8091D933811146
:10D5700011C080EE9BE39F938F93809106558F930C
:10D58000809105558F930E9408E40F900F900F90A3
:10D590000F9003C088E00E94F7AB80913A348093EB
:10D5A0003834F8CE0E94D159F5CE0E94D559F2CE2A
:10D5B0000E94D959EFCE8091D933813009F4EACE57
:10D5C0006DE577E380E00E948CC2E4CE1092D933FF
:10D5D0008EE594E30E944CC16DE577E30E948CC216
:10D5E000D9CE81E08093D9338EE594E30E944B7EBF
:10D5F000D1CE8091D933813019F547EF50E06EE5F7
:10D6000074E38DE595E30E949AE38DE595E39F939E
:10D610008F938AE691E29F938F938EE594E39F9395
:10D620008F930E94D3E480915C3490915D340E948A
:10D630004B7E0F900F900F900F900F900F90AACEEF
:10D640008EE594E30E9460746DE577E30E948CC2DE
:10D65000A1CE0E94314F823009F4D2CEC8CE1093B1
:10D660004B3880E60E94695309CF10924B380E94D4
:10D670002E5380934B38882309F4E1CEFDCE809160
:10D68000BF289091C0280E9438D2682F70E080E0B7
:10D6900090E00E94D0D723E333E34BE451E40E94AF
:10D6A00031D987FF77CE0E945D69823009F017CFAC
:10D6B00071CE809338340895809339340895CF9390
:10D6C000C82F80918D23882379F040E050E0BA0183
:10D6D0008C2F0E947A54EC2FFF27E7FDF095EA513A
:10D6E000F44D81E080830AC06C2F8AE491E50E94AA
:10D6F0007750AB01BC018C2F0E947A544091B42327
:10D700005091B5236091B6237091B7238C2F0E945E
:10D710007E5D88E29DE680938E2390938F2382E046
:10D72000CF910895CF92DF92EF92FF920F931F93C4
:10D73000CF93DF93CDB7DEB7E097CDBFDEBF98E1E3
:10D740007E01A9E1EA0EF11CF701A92F1192AA9519
:10D75000E9F7FE0131966F0111929A95E9F7F6010A
:10D7600094E08902E00DF11D1124408F518F628FEA
:10D77000738F80E090E0A0E8BFE380839183A28371
:10D78000B38300934E2C10934F2C2093502C309346
:10D79000512C0E9424870E94D959B601C7010E94CA
:10D7A000A35780934B38811101C082E0E096CDBF32
:10D7B000DEBFDF91CF911F910F91FF90EF90DF902F
:10D7C000CF9008950F931F93E0918723FF27E7FDE4
:10D7D000F095E554F64D9381913099F4009198239A
:10D7E0001091992320919A2330919B234091A0235B
:10D7F0005091A1236091A2237091A3230E94926B68
:10D800001DC0E0918823FF27E7FDF095E554F64D14
:10D810009381913099F4009198231091992320914C
:10D820009A2330919B234091A0235091A123609192
:10D83000A2237091A32370580E94926B88E29CE609
:10D8400080938E2390938F2382E01F910F910895F0
:10D850000F931F93CF93C82F85E3C802F0011124C3
:10D86000E954F54D40815181628173818C2F0E9472
:10D870007E5D009198231091992320919A233091F5
:10D880009B2340919423509195236091962370910E
:10D8900097238C2F0E94926B87EB9CE680938E23BC
:10D8A00090938F2382E0CF911F910F9108950F9352
:10D8B0001F93009198231091992320919A233091DE
:10D8C0009B234091A4235091A5236091A62370919E
:10D8D000A7230E94926B8FE59BE680938E23909303
:10D8E0008F2382E01F910F9108950E9424878091D9
:10D8F000AD230E94E3538091AC230E947D5380911D
:10D90000AE230E9481538091AF230E948F57809154
:10D91000B0239091B123A091B223B091B32380930F
:10D920004E2C90934F2CA093502CB093512C64E02C
:10D9300081E19CE20E946F4F0E94865A1092E22B76
:10D9400080E00895CF93C82F4091B4235091B52320
:10D950006091B6237091B7230E947E5D8C2F0E9448
:10D96000756C80E00E942FAE80EFCF9108950F93E9
:10D970001F93E0918723FF27E7FDF095E554F64DCF
:10D980009381913039F082EA9CE680938E239093C4
:10D990008F2318C000919C2310919D2320919E23DA
:10D9A00030919F234091A0235091A1236091A22305
:10D9B0007091A3230E94926B87E59CE680938E234F
:10D9C00090938F2382E01F910F910895FF920F9300
:10D9D0001F93CF93DF93CDB7DEB7C058D109CDBF2A
:10D9E000DEBFF82E0E9467658EEFF81205C087E74C
:10D9F00091E20E94BE6619C08F2D0E941B5B1F9290
:10DA00008F9325EF3BE33F932F938E010F5F1F4FC3
:10DA10001F930F930E94FCE4C8010E94BE660F9002
:10DA20000F900F900F900F900F9042E062E080EF08
:10DA30000E94CE668F2D0E94756C80EFC058DF4F1C
:10DA4000CDBFDEBFDF91CF911F910F91FF90089561
:10DA50004F925F926F927F929F92AF92BF92CF92BE
:10DA6000DF92EF92FF920F931F93CF93DF938F3F3D
:10DA700009F045C02CEA35EC47E257E36091492DA7
:10DA800070914A2D80914B2D90914C2D0E9431D94F
:10DA900018160CF469C12CEA35EC47E257E36091A3
:10DAA000412D7091422D8091432D9091442D0E94E3
:10DAB00031D918160CF45DC12CEA35EC47E257E376
:10DAC0006091452D7091462D8091472D9091482D64
:10DAD0000E9431D918160CF455C12CEA35EC47E2F6
:10DAE00057E360914D2D70914E2D80914F2D909167
:10DAF000502D0E9431D918160CF43FC171C18230EB
:10DB0000A1F52CEA35EC47E257E36091412D709185
:10DB1000422D8091432D9091442D0E9431D91816A9
:10DB20000CF427C12CEA35EC47E257E36091452D10
:10DB30007091462D8091472D9091482D0E9431D9AA
:10DB400018160CF41FC12CEA35EC47E257E360913C
:10DB50004D2D70914E2D80914F2D9091502D0E9402
:10DB600031D918160CF409C131C18823D9F281309A
:10DB700051F32CC17E018DEEE80EF11CF70180817E
:10DB80009181A281B381BC01CD019F772CEA35EC54
:10DB900047E257E30E942ED787FD46C06E01F1EFA2
:10DBA000CF0ED11CF601408051806280738020E04E
:10DBB00030E0A901C301B2010E942ED787FD34C015
:10DBC000FE01EF52FF4F2081318142815381349712
:10DBD00060817181828193810E9485D59B01AC0116
:10DBE0005F77C301B2010E9486D52B013C019F776C
:10DBF0002CEA35EC47E257E30E942ED787FD14C08C
:10DC0000AB2CAA0C8A2D0E94FCBF809385239924FB
:10DC100093949A0C892D0E94FCBF809386232091B7
:10DC20008523822780FD02C08B2DDBC0B092842328
:10DC3000F80180819181A281B381BF77809398237D
:10DC400090939923A0939A23B0939B23F70140814B
:10DC50005181628173817F7740939C2350939D23F0
:10DC600060939E2370939F2320FF2DC0A092872353
:10DC70009092882377FA709477F870944092942366
:10DC8000509295236092962370929723F60180819B
:10DC90009181A281B3818093A0239093A123A0932B
:10DCA000A223B093A323CB50DF4F88819981AA810F
:10DCB000BB818093A4239093A523A093A623B09324
:10DCC000A7238A2D2AC090928723A092882340926E
:10DCD0009423509295236092962370929723F60195
:10DCE00080819181A281B381B0588093A0239093C9
:10DCF000A123A093A223B093A323CB50DF4F88810D
:10DD00009981AA81BB81B0588093A4239093A523C5
:10DD1000A093A623B093A723892D0E94FCBF8D7FDB
:10DD2000813039F088E29DE680938E2390938F2393
:10DD300069C0809188230E94FCBF811103C08FEFCE
:10DD4000809388238B2D0E94735D6093B42370931E
:10DD5000B5238093B6239093B72382EE9BE68093FE
:10DD60008E2390938F234EC082E090E032E0B32E5A
:10DD70000DC080E090E0B12C09C083E090E023E08A
:10DD8000B22E04C081E090E0BB24B394FC01EA51C0
:10DD9000F44D108225E3289FE001299FD00D112426
:10DDA000C252D64D8E0107511F4FF80180819181DB
:10DDB000A281B381BC01CD019F772CEA35EC47E20B
:10DDC00057E30E942ED787FFD5CE2ECF81E08093D8
:10DDD000E52B85E79CE680938E2390938F2312C0DA
:10DDE0008EEFDF91CF911F910F91FF90EF90DF9019
:10DDF000CF90BF90AF909F907F906F905F904F902B
:10DE00000C94E66C82E0DF91CF911F910F91FF900F
:10DE1000EF90DF90CF90BF90AF909F907F906F90EA
:10DE20005F904F900895CF93DF93CFE0DCE288813D
:10DE300099810E94524F8093AC23888199810E94DE
:10DE40004D4F8093AD23888199810E945C4F8093D0
:10DE5000AE23888199810E94614F8093AF2388818E
:10DE600099810E94684F6093B0237093B12380938F
:10DE7000B2239093B32381E00E947D5381E00E94FE
:10DE8000815380E00E94E35381E00E948F5781E03C
:10DE900080938D238FEF8093842388E29DE6809387
:10DEA0008E2390938F2383E08093E22B1092E52BB7
:10DEB00080E0DF91CF9108950E94136F10928D231F
:10DEC00080E008958091E22B833059F40E94664FE0
:10DED000813049F0E0918E23F0918F23809184234B
:10DEE000199483E0089582E008958DE79FE680937A
:10DEF000C9239093CA2382E008952F923F924F92B4
:10DF00005F926F927F928F929F92AF92BF92CF92C9
:10DF1000DF92EF92FF920F931F93CF93DF93CDB7D2
:10DF2000DEB7CA54D109CDBFDEBF98E19E01275E9E
:10DF30003F4F29AB3AABD901E92F1D92EA95E9F79A
:10DF4000285131091901D9011D929A95E9F724E068
:10DF50008202F00111242B96EEAFFFAF2B97E20D5A
:10DF6000F31D80E090E0A0E8BFE380839183A2836B
:10DF7000B383C090C123D090C223E090C323F0901C
:10DF8000C4234090BD235090BE236090BF23709067
:10DF9000C0238090B9239090BA23A090BB23B09067
:10DFA000BC23A5019401C301B2010E942ED718160B
:10DFB0005CF080E090E0A0E8BFE329968CAF9DAFD5
:10DFC000AEAFBFAF29970AC080E090E0A0E8BFEBFA
:10DFD00029968CAF9DAFAEAFBFAF2997A301920139
:10DFE000C501B4010E9485D50E949DD79B0177FF92
:10DFF00004C022273327261B370BB901882777FD5A
:10E000008095982F0E94D0D725966CAF7DAF8EAFAC
:10E010009FAF2597C0924E2CD0924F2CE092502C5F
:10E02000F092512C0E9424870E94D95920E030E0C0
:10E0300040E050E425966CAD7DAD8EAD9FAD25974B
:10E040000E9431D918166CF08091C5239091C62397
:10E05000A091C723B091C8238BAF9CAFADAFBEAF2B
:10E06000DBC02AE037ED43E25CE325966CAD7DAD85
:10E070008EAD9FAD25970E9431D918162CF709E176
:10E0800010E08AE0882E87ED982E83E2A82E8CE39C
:10E09000B82E412C512C32012B96AEADBFAD2B9733
:10E0A000A20DB31D58962196AEAFBFAF21974BAAD4
:10E0B0005CAA6DAA7EAA8FAA98AEA9AEBAAE29961E
:10E0C0002CAD3DAD4EAD5FAD29976FA978AD89AD53
:10E0D0009AAD0E94D3D99B01AC016091BD23709190
:10E0E000BE238091BF239091C0230E9486D52196A4
:10E0F000EEADFFAD21976083718382839383C092DD
:10E100004E2CD0924F2CE092502CF092512CB10119
:10E11000CE0149960E94A35780934B388111AAC023
:10E1200020E030E040E85FE36BA97CA98DA99EA9BF
:10E130000E9486D56BAB7CAB8DAB9EAB20E030E014
:10E1400048EC51E40E9435D79B01AC0160E070E0DF
:10E1500080E291E40E9436DA2B013C018091C523D4
:10E160009091C623A091C723B091C8238BAF9CAFD9
:10E17000ADAFBEAFC090C123D090C223E090C32307
:10E18000F090C423A7019601BC01CD010E9485D562
:10E190004B015C0120E030E040E251E4C301B201F8
:10E1A0000E9435D79B01AC01C501B4010E94D3D9AF
:10E1B0009B01AC01C701B6010E9486D56B017C01B1
:10E1C0002BA93CA94DA95EA9CA01B9010E9486D517
:10E1D00020E030E048EC51E40E9435D79B01AC01CF
:10E1E0006FA978AD89AD9AAD0E9486D56FAB78AF37
:10E1F00089AF9AAF9B01AC0125966CAD7DAD8EAD1C
:10E200009FAD25970E9431D9181634F40150110999
:10E210000115110509F053CF8BAD9CADADADBEAD71
:10E2200080934E2C90934F2CA093502CB093512C54
:10E230002B96EEADFFAD2B97E20DF31D8091B92328
:10E240009091BA23A091BB23B091BC23808F918F72
:10E25000A28FB38FB101CE0149960E94A35780933C
:10E260004B38811107C081E591E78093C9239093D2
:10E27000CA2382E0C65BDF4FCDBFDEBFDF91CF9107
:10E280001F910F91FF90EF90DF90CF90BF90AF90D4
:10E290009F908F907F906F905F904F903F902F90C6
:10E2A0000895CF93DF931F92CDB7DEB789830E9485
:10E2B00024874091D3235091D4236091D52370912A
:10E2C000D62389810E947E5D8091D0230E94E353F2
:10E2D0008091CF230E947D538091D1230E9481534E
:10E2E0008091D2230E948F578091CB239091CC2391
:10E2F000A091CD23B091CE2380934E2C90934F2CA0
:10E30000A093502CB093512C64E081E19CE20E94D8
:10E310006F4F0E94865A1092E22B83EA91E20E948C
:10E32000A6E480E00F90DF91CF9108950F931F93A3
:10E33000CF93C82F0FE01CE2F801808191810E94E9
:10E34000524F8093CF23F801808191810E944D4FDD
:10E350008093D023F801808191810E945C4F80934B
:10E36000D123F801808191810E94614F8093D22353
:10E37000F801808191810E94684F6093CB23709354
:10E38000CC238093CD239093CE238C2F0E94735D5A
:10E390006093D3237093D4238093D5239093D62373
:10E3A00081E00E947D5380E00E94815380E00E94C2
:10E3B000E35381E00E948F5740E050E060E271E457
:10E3C0004093C1235093C2236093C3237093C4230B
:10E3D00085E3C89FF0011124E955F54D4081518135
:10E3E000628173814093C5235093C6236093C723F2
:10E3F0007093C8236C2F8AE491E50E946450609367
:10E40000BD237093BE238093BF239093C0230E94AB
:10E410004B5E6093B9237093BA238093BB23909390
:10E42000BC23C093B82385E79FE68093C9239093CC
:10E43000CA2384E08093E22B80E0CF911F910F915B
:10E4400008958091E22B843059F40E94664F813008
:10E4500049F0E091C923F091CA238091B82319941F
:10E4600083E0089582E00895E091D923F0E0E55437
:10E47000F64D8381882341F08FE492E78093D72380
:10E480009093D82382E0089566E274E28EE094E2ED
:10E490000E94A35780934B38882371F308951F93EC
:10E4A000CF93DF93E091D923F0E0E554F64D81E07E
:10E4B0009381913009F080E08093EC2BCDEEDBE28C
:10E4C00010E0812F0E94129BAB01BC01812F0E94A2
:10E4D0007A54612F80910F2C9091102C0E946450DF
:10E4E00069937993899399931F5F163051F78DEA59
:10E4F00091E20E944B7E8BEB92E78093D72390931F
:10E50000D82382E0DF91CF911F9108951F93CF937D
:10E51000DF930E9424878091DA238093BB29E091C6
:10E52000D923F0E08091DB23E554F64D83870E94E8
:10E5300019C0CEEDD3E210E04991599169917991DA
:10E54000812F0E947E5D1F5F1630B1F78091DD2321
:10E550000E94E3538091DC230E94815364E081E1B7
:10E560009CE20E946F4F0E94865A1092E22BDF912C
:10E57000CF911F9108950E94867280E008950F93B5
:10E580001F93CF93DF93CDB7DEB7C058D109CDBF6E
:10E59000DEBF182F0E9467651E3F29F48AEB91E2C7
:10E5A0000E94BE6619C0812F0E941B5B1F928F9331
:10E5B00083E29CE39F938F938E010F5F1F4F1F9306
:10E5C0000F930E94FCE4C8010E94BE660F900F905A
:10E5D0000F900F900F900F9042E062E08AEF0E9440
:10E5E000CE660E9486728AEFC058DF4FCDBFDEBF75
:10E5F000DF91CF911F910F910895FF920F931F9379
:10E60000CF93DF931092EC2B82E08093E22B0EED00
:10E6100013E2C7EBDAE2F12C8F2D0E94735DF80153
:10E6200061937193819391938F01488159816A819C
:10E630007B818F2D0E947E5D6F2D80910F2C90919C
:10E64000102C0E946450F801648B758B868B978B1D
:10E65000F394E596F6E0FF12DFCF6EE074E286EF0A
:10E6600093E20E9419C62AE43CE042E85EE30E947D
:10E670002ED787FF03C08EEF0E94BF72C2E0D4E2A4
:10E6800013E069917991899199912C893D894E89FD
:10E690005F890E9485D59F772CEA35EC47E257E3E6
:10E6A0000E9431D918161CF4812F0E94BF721F5F7F
:10E6B000163039F784E08093D9238091CA2980935A
:10E6C000DB2381E08093CA298091BB298093DA23E0
:10E6D0001092BB290E9419C080910F2C9091102C90
:10E6E0000E944D4F8093DD2380910F2C9091102C30
:10E6F0000E945C4F8093DC2380E00E94815380E085
:10E700000E94E35380E00E9475B284E392E7809315
:10E71000D7239093D82382E0DF91CF911F910F915F
:10E72000FF9008950F931F93CF93DF938C01EB011C
:10E7300080915A2C882399F080914E2C90914F2CE7
:10E74000A091502CB091512CBC01CD019F772CEAA7
:10E7500035EC47E257E30E942ED787FD4FC08881F2
:10E760009981AA81BB81BC01CD019F772CEA35EC50
:10E7700047E257E30E9431D91816F4F48C819D8149
:10E78000AE81BF81BC01CD019F772CEA35EC47E219
:10E7900057E30E9431D918167CF488859985AA859B
:10E7A000BB85BC01CD019F772CEA35EC47E257E3EE
:10E7B0000E9431D9181624F188E1F801AEE0B4E2E4
:10E7C00001900D928A95E1F788E1FE01A6E2B4E29C
:10E7D00001900D928A95E1F788E1EDEEFBE2DF0111
:10E7E0001D928A95E9F782E08093EC2B8DEF92E7FA
:10E7F0008093D7239093D82380E003C08EE801C094
:10E8000086E8DF91CF911F910F9108958091E22BBF
:10E81000823021F08091EC2B823049F40E94664FC7
:10E82000813039F0E091D723F091D823199483E017
:10E83000089582E00895E3ECF7E380E2DF011D92A2
:10E840008A95E9F78FEE92E18093E1379093E23772
:10E850008083918308958091E1379091E2378F3ED4
:10E86000924111F08CE508958091C3379091C4379F
:10E870008F3E9241B9F780E00895CF93DF93C82F80
:10E88000CB01BA010E9482DA27E0C29FE001112485
:10E89000CD53D84C0E949DD76D837E838F839887FC
:10E8A000DF91CF91089597E0899FF0011124ED53F6
:10E8B000F84C65817681878190850E94D0D7089534
:10E8C0002F923F924F925F926F927F928F929F9280
:10E8D000AF92BF92CF92DF92EF92FF920F931F936E
:10E8E000CF93DF93CDB7DEB72797CDBFDEBF8C01C7
:10E8F0001B828091E12B823009F40CC7D801BC90B7
:10E90000B11035C780E06E01B3E0CB0ED11C3DC025
:10E91000F6018081811108C0B72CD7011C926E01CD
:10E92000B3E0CB0ED11C20C7883239F4B72CF701E5
:10E930001082FFEFCF1ADF0A17C78B33B9F3A82E67
:10E94000B12CC5010E94F6E2892B39F4B50184EEA1
:10E9500091E20E946FE3892B51F047018FEF881AF3
:10E96000980AC5010E941AE3D7018C937401BFEF86
:10E97000CB1ADB0AF70180818111CACFB72CD801ED
:10E980008C916E01B3E0CB0ED11CF8011CC08E320D
:10E99000E1F090E0C0970A9790F08181803391F484
:10E9A000828190E0C0970A9760F4DF01119611967A
:10E9B0008C9111978D938111FACF808104C0818150
:10E9C00001C080E331968111E2CFF601A080A11051
:10E9D00007C036C0D6011196AC90BFEFCB1ADB0A48
:10E9E00076018A2C912CC4010E940AE3892B91F7AD
:10E9F000C4010E9412E38D369105A1F4F6018181D4
:10EA000090E00E9412E38337910561F4D6011296DB
:10EA10008C9190E00E9412E38736910519F4F6017B
:10EA2000339602C0FE013396AA2061F08A2DD701E9
:10EA3000893209F41C9211968C918111F9CF02C090
:10EA4000FE013396BFE2BB1609F466C680818823B7
:10EA500019F0CF010E94CC5980E1E3EEF7E3DF012A
:10EA60001D928A95E9F78BE5EAE3FDE2DF01982F35
:10EA70001D929A95E9F7EFEDFCE2DF011D928A9570
:10EA8000E9F781E19CE20E944A4F8093E02C812CBF
:10EA9000912C80E8A82E8FE3B82E5524539492E051
:10EAA000492E24E0322E23C4C701B6010E94A2D70A
:10EAB000862F90E08F35910508F032C6FC01EC50AE
:10EAC000FF4F0C9479DF1092E02C50923B2D8091F7
:10EAD000E4378F5F8093E4370AC45092E02C509261
:10EAE0003B2D8091E4378F5F8093E43700C44092E0
:10EAF000E02C50923B2D8091E4378F5F8093E43778
:10EB0000F6C383E08093E02C50923B2D8091E43754
:10EB10008F5F8093E437EBC38DE08093DF2C5092BE
:10EB20003A2DE5C388E0B2C010920F2D50926A2DA5
:10EB30008091E5378F5F8093E537D9C350920F2DD1
:10EB400050926A2D8091E5378F5F8093E537CFC370
:10EB500040920F2D50926A2D8091E5378F5F809300
:10EB6000E537C5C31092102D50926B2D8091E83778
:10EB70008F5F8093E837BBC35092102D50926B2D5E
:10EB80008091E8378F5F8093E837B1C3C701B60142
:10EB90000E94EDDA6C837D838E839F8320E030E0DA
:10EBA00040E251E4C701B6010E94D3D96B017C0158
:10EBB00020E030E040E251E46C817D818E819F81D4
:10EBC0000E94D3D99B01AC01C701B6010E9485D533
:10EBD0000E94A2D7623001F128F4662341F061302F
:10EBE00089F09EC56330E9F0643001F199C5B5E064
:10EBF000B093DF2C50923A2D8091E3378F5F809352
:10EC0000E33775C33092DF2C60933A2D8091E33760
:10EC10008F5F8093E3376BC35092DF2C50923A2D75
:10EC200066C34092DF2C50923A2D61C383E08093FB
:10EC3000DF2C50923A2D5BC3C701B6010E94EDDA7A
:10EC40006C837D838E839F8320E030E040E251E43B
:10EC5000C701B6010E94D3D96B017C0120E030E0EE
:10EC600040E251E46C817D818E819F810E94D3D9E5
:10EC70009B01AC01C701B6010E9485D50E94A2D7B5
:10EC8000662319F0613061F04BC587E08093DF2C7B
:10EC900050923A2D8091E3378F5F8093E33727C3FB
:10ECA000E6E0E093DF2C60933A2D8091E3378F5FAD
:10ECB0008093E3371CC3C701B6010E94EDDA6C8371
:10ECC0007D838E839F8320E030E040E251E4C701E2
:10ECD000B6010E94D3D96B017C0120E030E040E214
:10ECE00051E46C817D818E819F810E94D3D99B01EB
:10ECF000AC01C701B6010E9485D50E94A2D762303F
:10ED000009F00EC58EE08093DF2C50923A2DEFC2B1
:10ED10005092122D50926D2DEAC25092112D5092A8
:10ED20006C2D8091EC378F5F8093EC37E0C240927E
:10ED3000112D50926C2D8091EC378F5F8093EC37C2
:10ED4000D6C283E016C03092112D50926C2D809166
:10ED5000EC378F5F8093EC37CAC2F5E0F093112D4A
:10ED600050926C2D8091EC378F5F8093EC37BFC24F
:10ED700086E08093112D50926C2D8091EC378F5F3F
:10ED80008093EC37B4C2C701B6010E94EDDA6C8300
:10ED90007D838E839F8320E030E040E251E4C70111
:10EDA000B6010E94D3D96B017C0120E030E040E243
:10EDB00051E46C817D818E819F810E94D3D99B011A
:10EDC000AC01C701B6010E9485D50E94A2D7662377
:10EDD00019F0613059F0A4C41092142D50926F2D87
:10EDE0008091ED378F5F8093ED3781C26093142D52
:10EDF00060936F2D8091ED378F5F8093ED3777C2F1
:10EE00004092142D50926F2D8091ED378F5F80933B
:10EE1000ED376DC23092E02C50923B2D8091E4375B
:10EE20008F5F8093E43763C2C701B6010E94EDDAB9
:10EE30006C837D838E839F8320E030E040E251E449
:10EE4000C701B6010E94D3D96B017C0120E030E0FC
:10EE500040E251E46C817D818E819F810E94D3D9F3
:10EE60009B01AC01C701B6010E9485D50E94A2D7C3
:10EE7000662319F0613059F053C41092152D509249
:10EE8000702D8091E6378F5F8093E63730C2109205
:10EE9000162D6093712D8091E6378F5F8093E63752
:10EEA00026C2C701B6010E94EDDA6C837D838E8392
:10EEB0009F8320E030E040E251E4C701B6010E94A8
:10EEC000D3D96B017C0120E030E040E251E46C8159
:10EED0007D818E819F810E94D3D99B01AC01C701A6
:10EEE000B6010E9485D50E94A2D7662319F0613031
:10EEF00059F016C45092152D5092702D8091E6371E
:10EF00008F5F8093E637F3C16093162D6093712D68
:10EF10008091E6378F5F8093E637E9C1C701B6017C
:10EF20000E94EDDA6C837D838E839F8320E030E046
:10EF300040E251E4C701B6010E94D3D96B017C01C4
:10EF400020E030E040E251E46C817D818E819F8140
:10EF50000E94D3D99B01AC01C701B6010E9485D59F
:10EF60000E94A2D7613089F028F06230A1F06330AE
:10EF7000C1F0D6C399E09093DF2C50923A2D809146
:10EF8000E3378F5F8093E337B2C1AAE0A093DF2C11
:10EF900060933A2DACC1BBE0B093DF2C50923A2D78
:10EFA000A6C1ECE0E093DF2C50923A2DA0C1109264
:10EFB0000A2D5092652D8091E7378F5F8093E73758
:10EFC00096C150920A2D5092652D8091E7378F5F40
:10EFD0008093E7378CC1C701B6010E94A2D7862F64
:10EFE00090E08D33910508F099C3FC01ED5AFE4F76
:10EFF0000C9479DF1092E12C50923C2D8091EE37E9
:10F000008F5F8093EE3773C15092E12C50923C2D6C
:10F010008091EE378F5F8093EE3769C150921C2D3F
:10F020005092772D8091F0378F5F8093F0375FC1DA
:10F0300040921C2D5092772D8091F0378F5F8093F6
:10F04000F03755C110921C2D5092772D8091F037DA
:10F050008F5F8093F0374BC15092192D5092742DD1
:10F0600046C150921A2D5092752D8091F1378F5FC5
:10F070008093F1373CC150921B2D5092762D809198
:10F08000F1378F5F8093F13732C110921B2D509270
:10F09000762D8091F1378F5F8093F13728C15092A0
:10F0A0000D2D5092682D8091F2378F5F8093F2374B
:10F0B0001EC110920D2D5092682D8091F2378F5FF6
:10F0C0008093F23714C150920B2D5092662D80918F
:10F0D000F2378F5F8093F2370AC15092252D5092FC
:10F0E000802D8091F2378F5F8093F23700C1C70186
:10F0F000B6010E94EDDA0E94A2D76093182D5092BB
:10F10000732DF5C0C092FE2CD092FF2CE092002D02
:10F11000F092012D8092592D90925A2DA0925B2D44
:10F12000B0925C2DE4C0C092262DD092272DE092A3
:10F13000282DF092292D8092812D9092822DA092DF
:10F14000832DB092842DD3C0C0921D2DD0921E2D40
:10F15000E0921F2DF092202D8092782D9092792DA3
:10F16000A0927A2DB0927B2DC2C0C092E62CD09294
:10F17000E72CE092E82CF092E92C8092412D9092BD
:10F18000422DA092432DB092442DB1C0C092EA2CE2
:10F19000D092EB2CE092EC2CF092ED2C8092452D4D
:10F1A0009092462DA092472DB092482DA0C0C092BB
:10F1B000EE2CD092EF2CE092F02CF092F12C809279
:10F1C000492D90924A2DA0924B2DB0924C2D8FC07C
:10F1D000C092F22CD092F32CE092F42CF092F52C09
:10F1E00080924D2D90924E2DA0924F2DB092502D89
:10F1F0007EC0C092F62CD092F72CE092F82CF092C0
:10F20000F92C8092512D9092522DA092532DB092B4
:10F21000542D6DC0C092FA2CD092FB2CE092FC2CA5
:10F22000F092FD2C8092552D9092562DA092572D44
:10F23000B092582D5CC0C0922E2DD0922F2DE0920E
:10F24000302DF092312D8092892D90928A2DA092AE
:10F250008B2DB0928C2D4BC0C092322DD092332D7D
:10F26000E092342DF092352D80928D2D90928E2D3E
:10F27000A0928F2DB092902D3AC0C092362DD09290
:10F28000372DE092382DF092392D8092912D909269
:10F29000922DA092932DB092942D29C0C0922A2D28
:10F2A000D0922B2DE0922C2DF0922D2D8092852D39
:10F2B0009092862DA092872DB092882D18C0C701FC
:10F2C000B6010E94A2D76093E22C7093E32C809346
:10F2D000E42C9093E52C81E090E0A0E0B0E08093F6
:10F2E0003D2D90933E2DA0933F2DB093402DD801FE
:10F2F0002C90222009F422C2822D90E00E9401E38A
:10F30000892B09F42DC23801BFEF6B1A7B0AF80173
:10F310008181803349F48281883531F40E5F1F4F3B
:10F32000C12CD12C7601FEC1BE016F5F7F4FC3019E
:10F330000E9499DF6B017C0109811A8160167106B8
:10F3400009F0F0C10FC280910A2D0E948F57182F2B
:10F3500001C010E06091592D70915A2D80915B2D64
:10F3600090915C2D0E94A2D7662359F06091FE2CEB
:10F370007091FF2C8091002D9091012D0E945E577D
:10F38000182F60915D2D70915E2D80915F2D909171
:10F39000602D0E94A2D7662371F06091022D7091BA
:10F3A000032D8091042D9091052D0E94A2D7862FC8
:10F3B0000E943A59182F6091612D7091622D8091B1
:10F3C000632D9091642D0E94A2D7662371F0609105
:10F3D000062D7091072D8091082D9091092D0E9486
:10F3E000A2D7862F0E947959182F6091782D70919D
:10F3F000792D80917A2D90917B2D0E94A2D7662342
:10F4000059F060911D2D70911E2D80911F2D9091AE
:10F41000202D0E94A9B2182F60917C2D70917D2D16
:10F4200080917E2D90917F2D0E94A2D7662371F04E
:10F430006091212D7091222D8091232D9091242D6A
:10F440000E94A2D7862F0E94B859182F8091732D41
:10F45000882329F08091182D0E94F757182F80914A
:10F46000742D882329F08091192D0E942B58182F74
:10F470008091772D882329F080911C2D0E9475B2F0
:10F48000182F8091752D882329F080911A2D0E94C4
:10F490006058182F8091762D882329F080911B2D9C
:10F4A0000E949458182F8091662D882329F080910E
:10F4B0000B2D0E940F59182F8091672D882329F05A
:10F4C00080910C2D0E944E59182F8091802D8823F9
:10F4D00029F08091252D0E948D59182F8091682D3B
:10F4E000882329F080910D2D0E940759182F8091B3
:10F4F000DF2C8D3029F080916A2D8823A9F00FC070
:10F500006091262D7091272D8091282D9091292D85
:10F510000E94975780934B38882369F32DC18091BF
:10F520000F2D0E947953182F80916B2D882329F07D
:10F530008091102D0E947D53182F80916C2D88236F
:10F5400029F08091112D0E94E353182F80916F2D87
:10F55000882329F08091142D0E949357182F8091B1
:10F56000702D882329F08091152D0E948153182F2A
:10F570004091DF2C50E04F30510508F0B4C0FA0143
:10F58000E057FE4F0C9479DF0E94E056182FABC075
:10F5900061E47DE286EE9CE20E94EB56182FA3C048
:10F5A0000E941F57182F9FC061E47DE286EE9CE207
:10F5B0000E942A57182F97C00E94136F182F93C0CC
:10F5C00061E47DE286EE9CE20E94AA54182F8BC073
:10F5D0000E945C6F182F87C061E47DE286EE9CE29A
:10F5E0000E949273182F7FC06091262D7091272D55
:10F5F0008091282D9091292D0E94A2D7862F41E439
:10F600005DE266EE7CE20E948553182F6CC061E4D7
:10F610007DE286EE9CE20E942755182F64C00E946E
:10F62000DA55182F60C00E944156182F5CC00E9406
:10F630007856182F58C06091122D81E19CE20E94EB
:10F64000E54F8091E02C843038F48230D8F4882360
:10F6500049F0813079F047C0843009F044C080938C
:10F66000152C41C061E47DE286EE9CE20E94B0561A
:10F67000182F39C061E47DE286EE9CE20E94A35718
:10F68000182F31C0A090362DB090372DC090382D56
:10F69000D090392DE090322DF090332D0091342D03
:10F6A0001091352D20912E2D30912F2D4091302D00
:10F6B0005091312D8F9380912D2D8F9380912C2DF2
:10F6C0008F9380912B2D8F9380912A2D8F9361E4BE
:10F6D0007DE286EE9CE20E94B488182F0F900F9076
:10F6E0000F900F900F9060E081E19CE20E94E54F47
:10F6F00080913C2D813061F48091E12C811104C016
:10F700000E94B95A812F38C00E94EA5A812F34C012
:10F71000812F32C08BEC30C083E02EC084E82CC037
:10F7200083E82AC0822D90E0FC01E154F109EA311E
:10F73000F105B0F7E156FE4F0C9479DF10924B388B
:10F740006091E22C7091E32C8091E42C9091E52C57
:10F750000E947F4F8091652D882309F4FACDF3CD67
:10F7600085E60AC086E608C0D8018C910EC96801FA
:10F770008B2D78017B2CD8C82796CDBFDEBFDF91BB
:10F78000CF911F910F91FF90EF90DF90CF90BF909E
:10F79000AF909F908F907F906F905F904F903F9031
:10F7A0002F900895CF93DF93EC016DE577E30E94EE
:10F7B000276680934B38811102C095E09F83DF91CB
:10F7C000CF910895FC018789908D0C94607483FF1C
:10F7D00006C0E091B329F091B42990E2958382FFAD
:10F7E00006C0E091B529F091B62990E2958381FF9A
:10F7F00006C0E091B729F091B82990E2958380FF87
:10F8000006C0E091B929F091BA2980E28583089574
:10F8100083FF06C0E091B329F091B42990E296836A
:10F8200082FF06C0E091B529F091B62990E2968357
:10F8300081FF06C0E091B729F091B82990E2968344
:10F8400080FF06C0E091B929F091BA2980E2868351
:10F85000089580914034811107C084E00E94E77BC5
:10F8600081E080934034089584E00E94087C1092E7
:10F8700040340895CF92DF92EF92FF920F931F933F
:10F88000CF93DF93C12C26E0D22EC092A329D09231
:10F89000A42930EAE32E36E0F32EE092A529F09277
:10F8A000A62900E816E00093A7291093A829C0E62E
:10F8B000D6E0C093A929D093AA29C092AB29D092AF
:10F8C000AC29C093AD29D093AE290093AF291093F2
:10F8D000B029E092B129F092B2292DEC3CEC4CED2C
:10F8E00050E40E9431D9C092B329D092B429E09259
:10F8F000B529F092B62918164CF4C093B729D093C5
:10F90000B8290093B9291093BA2908C00093B729E0
:10F910001093B829C093B929D093BA29DF91CF9118
:10F920001F910F91FF90EF90DF90CF9008950E946C
:10F93000D8D460E070E080E091E40E943A7C0C94BE
:10F94000F7D481E080934934089520E093E088ED76
:10F9500008B618BE84BF909380002091820021FDDC
:10F96000FCCF08BEFFCF8091493481110E94A57C55
:10F9700083E0089580914A34882341F0F89461E04F
:10F9800089E790E00E94DAD482E0089583E0089548
:10F99000CF93DF93CDB7DEB7AD97CDBFDEBF21E20A
:10F9A000E7EEF1E2DE01119601900D922A95E1F762
:10F9B00022E02093CA01DE019296E8E0F0E0249173
:10F9C0002D933196EE30F105D1F72DE228A7E0E135
:10F9D000F0E0E491EF7121E030E02C0F3D1F2E0F9D
:10F9E000311DF901208129A7E2E1F0E0E491EF71F6
:10F9F0009E012E0F311DF90121812AA7E4E1F0E0DB
:10FA0000E491EF719E012E0F311DF90121812BA789
:10FA10001CA61092CA0125E0FC012783BE016E5D81
:10FA20007F4F0E94276680934B38AD96CDBFDEBFD7
:10FA3000DF91CF91089581E080934A3480E008956A
:10FA4000CF93DF93EC0120E030E040E051E46985A2
:10FA50007A858B859C850E9431D918166CF0CE0171
:10FA60000E94516369857A858B859C850E943A7CCA
:10FA70000E9419C080E001C08DE6DF91CF9108950A
:10FA800065EC7CE30C94C9C567EA7CE30C94C9C5BA
:10FA900068E87CE30C94C9C56AE67CE30C94C9C5AC
:10FAA00066E57CE30C9474C5CF93DF938BE098E418
:10FAB0009F938F93C5E0D5E589818F9388818F933C
:10FAC0000E9408E485ED95E49F938F9389818F933D
:10FAD00088818F930E9408E48DE495E49F938F932F
:10FAE00089818F9388818F930E9408E483E894E44E
:10FAF0009F938F9389818F9388818F930E9408E4CD
:10FB00000E946FAC8DB79EB740968DBF9EBF80E0C0
:10FB1000DF91CF910895CF93DF938EE594E49F9387
:10FB20008F93C5E0D5E589818F9388818F930E945B
:10FB300008E480EF92E49F938F9389818F9388816B
:10FB40008F930E9408E485E691E49F938F938981C7
:10FB50008F9388818F930E9408E48DE495E49F93AE
:10FB60008F9389818F9388818F930E9408E483E823
:10FB700094E49F938F9389818F9388818F930E94C0
:10FB800008E48DB79EB744968DBF9EBF80E0DF919D
:10FB9000CF910895CF93DF9384E491E49F938F9363
:10FBA000C5E0D5E589818F9388818F930E9408E411
:10FBB00086EC9DE39F938F9389818F9388818F93A8
:10FBC0000E9408E483E894E49F938F9389818F9344
:10FBD00088818F930E9408E48DB79EB70C968DBFE5
:10FBE0009EBF80E0DF91CF910895CF93DF938EE9A0
:10FBF0009DE39F938F93C5E0D5E589818F9388819D
:10FC00008F930E9408E48DE29DE39F938F938981F7
:10FC10008F9388818F930E9408E483E894E49F93F4
:10FC20008F9389818F9388818F930E9408E48DB789
:10FC30009EB70C968DBF9EBF80E0DF91CF91089557
:10FC4000CF93DF938AE09DE39F938F93C5E0D5E543
:10FC500089818F9388818F930E9408E481EE9CE3D1
:10FC60009F938F9389818F9388818F930E9408E45B
:10FC700083E894E49F938F9389818F9388818F93F6
:10FC80000E9408E48DB79EB70C968DBF9EBF80E0A2
:10FC9000DF91CF9108952F923F924F925F926F9292
:10FCA0007F928F929F92AF92BF92CF92DF92EF920C
:10FCB000FF920F931F93CF93DF93CDB7DEB76A9771
:10FCC000CDBFDEBF5C010E9467652C011F86188ACC
:10FCD000198A1A8AF50101900020E9F73197EA198B
:10FCE000FB09E130F24008F002C2D5018C91882373
:10FCF00059F17501BFEFEB1AFB0A850120E02111D4
:10FD000015C0883229F08132C8F08F37B9F001C0B0
:10FD100021E06801EFEFCE1ADE0A90E02A8F0E9400
:10FD200012E3D8018C9386012A8D08C021E0893224
:10FD300009F420E0F80180830F5F1F4FD7018D91F8
:10FD40007D018111DCCF01C08501F8011082109284
:10FD50004B38FDE19F2EAAE36A2EA2E27A2E812C77
:10FD6000B6E02B2E03C09A9409F49CC18BE79CE269
:10FD7000A2E2B0E08B879C87AD87BE876B8A7C8AC6
:10FD80008D8A8DE79CE2A2E2B0E08F839887A987F5
:10FD9000BA87E8E0F2E2DE011196822D01900D9221
:10FDA0008A95E1F7C2010E946E648501075F1F4FCB
:10FDB00075019FEFA91AB90AD7016C9170E0CE01C5
:10FDC0000B960E946FE3892B21F487010E5D1F4F74
:10FDD00004C0A016B10661F793C16501BFEFAB1A6D
:10FDE000BB0AF601608170E0CE0143960E946FE38A
:10FDF000892B91F0D6011D928D0192012F5E3F4F0C
:10FE0000288F398F46E050E0B701C9010E949AE37C
:10FE10003AE0C30ED11C04C0A016B106F1F670C1C1
:10FE20005801D8013D908D01E32CF12CC7010E94AF
:10FE3000F6E2892B59F4B701CE0101960E946FE3D7
:10FE4000892B21F40C151D0559F75AC18501BEE611
:10FE50003B1641F0E2E23E120CC0D50111968C91A6
:10FE60008232A9F5F2011782118612861386148652
:10FE7000A3C0B0E3EB1AF108EAE0EE16F10418F0C3
:10FE8000FDE23F1217C0BE016A5E7F4FC5010E94AE
:10FE900099DFD20119966D937D938D939C931C9756
:10FEA0008E899F898A159B0509F42DC1E4E0179678
:10FEB000EC9382C0FBE73F124FC0E7E0D2011796F8
:10FEC000EC93FFEFAF1ABF0AE2E0FE2E95C02FEFD2
:10FED000A21AB20AE5E0D2011796EC9362E270E052
:10FEE000C5010E946FE38E8B9F8B009709F408C1B8
:10FEF000DC011C92F50101900020E9F73197EA1925
:10FF0000FB093397C8F0F80181818033A9F482811D
:10FF1000883791F440E050E060E070E0C5010E9455
:10FF20000AE1D20119966D937D938D939C931C9752
:10FF300083E017968C9308C0B501C2010E94276622
:10FF400080934B38811153C0AE88BF88BFEFAB1A86
:10FF5000BB0AAE8ABF8A30C0E4E73E120EC0E1E0C1
:10FF6000D2011796EC9380E090E0A0E8BFE3F201A5
:10FF700081879287A387B4871FC0F6E63F120CC023
:10FF8000E1E0D2011796EC93179719961D921D92F6
:10FF90001D921C921C9710C0BBE53B12B1C0F20130
:10FFA0002782B501C2010E94276680934B388111D8
:10FFB0001EC077E6F72E7DC0BE01695F7F4FC50189
:10FFC0000E94B4E35C01009709F49AC0DC018C91B3
:10FFD0008D3729F411968C91F50131965F018C32A1
:10FFE00009F48BC0FFEFAF1ABF0AF12C05C0F82E41
:10FFF00022E0281708F45DC08F858201035F1F4F40
:020000021000EC
:10000000882341F043E050E0BE01615F7F4FC801AB
:100010000E949AE3688D798DC8010E94C863D2015D
:1000200014968D939C9315978F3FBFEF9B07B9F163
:100030000E94F768882371F0888D998D0E94B163C2
:10004000882341F043E050E0688D798DCE010F9612
:100050000E949AE3F201428053804114510411F14D
:10006000F11081CE8091CF2E811108C088EC9EE2E4
:100070000E948C6080934B38F82E1BC08091E12B3E
:10008000823099F088EC9EE20E94626080934B3847
:1000900081110EC088EC9EE20E94DF600AC064E617
:1000A000F62E07C050E7F52E04C04BECF42E01C02D
:1000B000F82E42E060E08F2D0E94CE6681E00E9423
:1000C0002FAE6A96CDBFDEBFDF91CF911F910F910A
:1000D000FF90EF90DF90CF90BF90AF909F908F9068
:1000E0007F906F905F904F903F902F9008958BE698
:1000F00080934B383BE6F32EDCCF22E0F22E7CCF10
:100100009FE6F92ED6CF86E6F82ED3CF2F923F92D8
:100110004F925F926F927F928F929F92AF92BF9217
:10012000CF92DF92EF92FF920F931F93CF93DF93C3
:1001300000D000D0CDB7DEB78C0169837A834B83C2
:100140005C835A0128E0A21AB108A60EB71EDC0192
:1001500016967C907B01BFEFEB1AFB0A8BE7FB0145
:10016000808380E0912C95E0692E22E1422E22E2EC
:10017000522E3EE0232E32E2332E4DE7842EED82C6
:10018000FE82D80117969C919F3F09F429C18823CC
:1001900039F02CE2ED81FE8120833196ED83FE83E0
:1001A0008091F537811119C0C80141969F938F93B3
:1001B0003F922F923E813F938D818F930E94D3E493
:1001C000AD81BE81A80FB91FAD83BE830F900F9084
:1001D0000F900F900F900F9018C0C80141969F93F9
:1001E0008F935F924F92BE81BF93ED81EF930E94F8
:1001F000D3E42D813E81280F391F2D833E830F903C
:100200000F900F900F900F900F90D80117968C9130
:100210001797843059F51996CD90DD90ED90FC90AC
:100220001C97A7019601C701B6010E94F4DA81115B
:1002300017C0E894F7F82FEF3FEF4FE75FE7C701EC
:10024000B6010E94F4DA811121C12FEF3FEF4FE791
:100250005FE7C701B6010E942ED718160CF016C131
:10026000F801118612861386148610C1811113C0FD
:10027000E8E1F2E2AD81BE81862D01900D928A9572
:10028000E1F72D813E812C5F3F4F2D833E83D801C6
:1002900017968C9199C0823061F4F80184858F9310
:1002A00083858F9382858F9381858F93ADE1B2E2B1
:1002B00014C0833029F5D8011C968C911C978F931C
:1002C0001B968C911B978F931A968C911A978F93EC
:1002D00019968C918F93A3E2B2E2BF93AF93FE8104
:1002E000FF932D812F930E94D3E4AD81BE81A80F8F
:1002F000B11DAD83BE83F8018781CDBFDEBF64C071
:10030000853059F4D80158968C9158978F93579609
:100310008C918F93ABE2B2E20CC0863009F5D80124
:1003200058968C9158978F9357968C918F93A0E302
:10033000B2E2BF93AF93FE81FF932D812F930E9472
:10034000D3E4AD81BE81A80FB11DAD83BE83F8019A
:1003500087810F900F900F900F900F900F9034C0E7
:10036000813091F52CEA35EC47E257E3D801199634
:100370006D917D918D919C911C970E942ED787FF46
:1003800012C0E5E3F2E2AD81BE8186E001900D92FC
:100390008A95E1F7ED81FE813596ED83FE83D801E4
:1003A00017968C9111C0EBE3F2E2AD81BE81862DF0
:1003B00001900D928A95E1F7ED81FE813496ED83EF
:1003C000FE83D80117968C91873049F42BE7ED8195
:1003D000FE8120833196ED83FE8380E001C081E0C1
:1003E000AD81BE81AA15BB0518F08FEF9FEF65C0E8
:1003F000F801028113810115110549F0D801169603
:100400009C912FEF290D99153CF0992EBACEED80D5
:10041000FE807914B4F020C0ED81FE81D801CF01B7
:100420000196808216969C9016973FEF320F921697
:100430001CF4232FFC01F3CF8D839E838D0181E07B
:10044000A0CEF7012DE7CF01019620839A9479146D
:1004500014F4FC01F8CF7C018DE79AE0A0E0F701ED
:1004600080839183A283F2E0EF0EF11C89819A814F
:100470002B813C81820F931F8E159F0508F4B5CF09
:10048000C701A981BA818A1B9B0B17C0C8010E94B2
:100490000769F801418552856385748520858D81C2
:1004A0009E810E940DC82D813E81280F311D2D8314
:1004B0003E83D80117968C9187CF2696CDBFDEBF9D
:1004C000DF91CF911F910F91FF90EF90DF90CF9030
:1004D000BF90AF909F908F907F906F905F904F9064
:1004E0003F902F90089540E052E06DE575E30E9443
:1004F000868060910555709106558DE595E30C94C5
:1005000057E4CF92DF92EF92FF920F931F93CF9316
:10051000DF93CDB7DEB76B97CDBFDEBFF82E9091DE
:10052000F337992309F4F3C02FE6821310C00E9419
:1005300067656DE577E38EE594E30E94EDC7BC0146
:1005400086E091E20E94856608EC1EE24AC0809136
:10055000E12B08EC1EE2882309F443C0EE24EA9460
:10056000C8010E942E648823E1F1823029F4809131
:10057000FA37811120C01DC0843029F48091F737EB
:10058000811119C016C08530B1F48091F9378823E4
:1005900081F0F80181859285A385B485BC01CD01E8
:1005A0009F772CEA35EC47E257E30E942ED787FF6E
:1005B00002C0F801E782F8010281138101151105DB
:1005C00079F60FC0F801028113810115110549F474
:1005D00040E052E06DE575E38FEA9EE20E9486807E
:1005E00096C0F80197819F3F69F780913D348F93C2
:1005F00080913C348F931F92FF921F9281E08F93E2
:1006000080E492E29F938F939E012F5F3F4F790189
:10061000FF922F930E94D3E410923C3410923D3409
:10062000B701C8010E9427668091F437F8018683DC
:1006300086E0878386E690E0818B928B128213821C
:1006400040E052E06DE575E38FEA9EE20E9486800D
:10065000CDBFDEBF893F31E0930708F058C08C0161
:10066000FC01E35AFA4C2081203309F441C06C01AB
:1006700084ECC81A8EEFD80AD601AF5DBB4CB80126
:10068000615071098E918033D9F7625A7A4C7E019C
:1006900093E1E90EF11CC7012B8F0E9483E32B8DA0
:1006A0002C3241F0F601EF5DFB4C015011098291B3
:1006B0008C32D9F7B8018DE595E30E9416C9FF92F7
:1006C000EF929F938F938BE492E29F938F93025AC2
:1006D0001A4C1F930F930E94D3E4609105557091BB
:1006E00006558DE595E30E9457E4CDBFDEBF0FC0F0
:1006F0007E01F3E1EF0EF11CBC01625A7A4CC70196
:100700000E9483E39801245C3E4F6901CBCF6B9636
:10071000CDBFDEBFDF91CF911F910F91FF90EF9082
:10072000DF90CF900895613019F0623029F008957C
:1007300088EC9EE20C9473820C948182CF92DF92BB
:10074000EF92FF92FC01C184D284E384F48420E020
:1007500030E040EA50E4C701B6010E9431D91816D2
:100760000CF453C0C701B6010E94A2D76093F337BF
:100770001092F6371092F7371092F8371092F93737
:100780001092FA3720E030E040E85FE3C701B6019D
:100790000E9431D987FD03C081E08093F63720E0C5
:1007A00030E040E050E4C701B6010E9431D987FD36
:1007B00003C081E08093F73720E030E040E450E46C
:1007C000C701B6010E9431D987FD03C081E0809343
:1007D000F83720E030E040E850E4C701B6010E945D
:1007E00031D987FD03C081E08093F93720E030E004
:1007F00040EA50E4C701B6010E9431D987FD07C025
:1008000081E08093FA3780E003C08EE601C080E08B
:10081000FF90EF90DF90CF9008956DEA78E40C940C
:100820008AC566E578E40C948AC562E278E40C94A3
:100830008AC5BF92CF92DF92EF92FF920F931F93E0
:10084000CF93DF93CDB7DEB76897CDBFDEBF6B0127
:1008500028E1FC01DE01119601900D922A95E1F745
:1008600082EAE82E8AE2F82E8E010F5F1F4FB12C2C
:10087000F7018081823029F4F801108211821282FE
:100880001382809185538B1114C02091985330911D
:10089000995340919A5350919B53F8016081718113
:1008A000828193810E94D3D9F60160837183828310
:1008B00093838091A4538B1114C02091B75330912E
:1008C000B8534091B9535091BA53F8016081718186
:1008D000828193810E94D3D9F601648375838683D4
:1008E00097838091C3538B1114C02091D6533091BC
:1008F000D7534091D8535091D953F80160817181F9
:10090000828193810E94D3D9F601608771878287A3
:1009100093878091E2538B1114C02091F55330914D
:10092000F6534091F7535091F853F801608171816B
:10093000828193810E94D3D9F60164877587868767
:100940009787B394F5E3EF0EF11C0C5F1F4F86E021
:10095000B8128ECF6896CDBFDEBFDF91CF911F91C9
:100960000F91FF90EF90DF90CF90BF900895F89493
:100970000E94977C0E940E850E94F7D40E9477C93E
:100980000E94D4B60E941B740E9419C00E94F6A94E
:1009900040E060E080E00E946C690E94A4650E94D3
:1009A000FC840E9400870E9419540E94EFD4809119
:1009B000A20084608093A2008091A2008260809354
:1009C000A2008091A20081608093A20078940E948E
:1009D0006FAC0E944BC10E94C769FDCFE82FF0E0C9
:1009E000EE0FFF1FE752F74B659174914FE450E013
:1009F0008BEF97E30C9441E380913B34823041F4D8
:100A000040E060E081E00E946C6980E00E945C6BE5
:100A10000C94BECB682F81E00C9453CA10924C38D2
:100A200010924D3810924E3810924F380895CF934F
:100A3000DF93EC018C819D81880F991F880F991F8E
:100A400020914E3830914F38820F931F8093503849
:100A50009093513844E050E066E578E30E94EFD38C
:100A600040915638509157386091583870915938A4
:100A700049875A876B877C8780E0DF91CF91089503
:100A80008F929F92AF92BF92CF92DF92EF92FF929E
:100A9000CF93DF93EC018091E22B882369F089E00A
:100AA000DF91CF91FF90EF90DF90CF90BF90AF900C
:100AB0009F908F900C94F7AB89859A85AB85BC8508
:100AC0008093523890935338A0935438B09355384C
:100AD000CE010E94178580934B3881116EC0C98466
:100AE000DA84EB84FC84A7019601C701B6010E9459
:100AF000F4DA81112FC046015701E894B7F82FEFBF
:100B00003FEF4FE75FE7C501B4010E94F4DA8111BE
:100B10000AC02FEF3FEF4FE75FE7C501B4010E9426
:100B20002ED71816BCF08090523890905338A09071
:100B30005438B0905538A5019401C701B6010E9400
:100B400085D59F772CEA35EC47E257E30E9431D9EF
:100B5000181674F58091523890915338A0915438FA
:100B6000B09155388093563890935738A0935838A1
:100B7000B09359388C819D81880F991F880F991FD8
:100B800020914E3830914F38820F931F8093503808
:100B90009093513844E050E066E578E30E9480D4B9
:100BA0008090523890905338A0905438B090553877
:100BB00089869A86AB86BC8680E0DF91CF91FF90D4
:100BC000EF90DF90CF90BF90AF909F908F9008955F
:100BD0000E942FBC80E0089580915A3890915B3834
:100BE0008F3E924111F08EE508958091803890916A
:100BF00081388F3E9241B9F7809182389091833845
:100C00008F3E924181F780910B5090910C508F3E16
:100C1000924149F780910D5090910E508F3E924134
:100C200011F78091A0519091A1518F3E9241D9F638
:100C300080E0089594E0899FF0011124E65AF74C72
:100C40004283538364837583089594E0899FF00100
:100C50001124E35FFF4A45AB56AB67AB70AF089515
:100C60005F926F927F928F929F92AF92BF92CF923C
:100C7000DF92EF92FF920F931F93CF93DF93CDB745
:100C8000DEB76097CDBFDEBFBE016F5F7F4F82E4EE
:100C900090E50E941984CE0101964C018AEBA82EA2
:100CA00080E5B82E9AECC92E90E5D92E2AEDE22ED9
:100CB00020E5F22E0AEF10E53CE1632E34E5732EB9
:100CC000512CF40141915191619171914F01F501C4
:100CD00041935193619371935F01F6014193519355
:100CE000619371936F01F7014193519361937193F4
:100CF0007F01852D0E943D74F8011192119211928D
:100D000011928F01F3011082118212821382539487
:100D1000F8E16F0E711C84E05812D3CF6096CDBFFE
:100D2000DEBFDF91CF911F910F91FF90EF90DF9089
:100D3000CF90BF90AF909F908F907F906F905F907B
:100D400008958091843808951F93CF93DF938BE8A3
:100D500097E1E2E8F8E3DF019C011D922150304069
:100D6000E1F78FEE92E180938238909383388093FD
:100D70000B5090930C50CBE8D8E3C0938538D093B8
:100D80008638C0938738D0938838C0938938D093F9
:100D90008A3881E090E06FE47FE420E030E01CEBF3
:100DA000129FA001139F500D1124FA01EE57F74C2A
:100DB000D90111961A9F90011B9F300D11242557C0
:100DC000374C2387348761877287BA016557774C20
:100DD0009C0101968032910519F78CEB829FF001FE
:100DE000839FF00D1124EE57F74CC387D48761879A
:100DF000728780E280938438DF91CF911F910895AC
:100E0000CF93DF93EDE0F0E585E991E0DF01EC01C0
:100E10001D922197E9F7AAE5B8E388E2ED0119925E
:100E20008A95E9F78FEE92E18D939C9380938038B9
:100E300090938138808391838093A0519093A151A6
:100E4000DF91CF910C94A4860E941D910E94A486EC
:100E500080E00C94344FE0918538F0918638848599
:100E600081111BC022813381808191814CEBDF0194
:100E70001D924A95E9F7228333838083918381E031
:100E800084878091843881508093843882819381D3
:100E9000809385389093863805C08CE10E94F7AB2B
:100EA000E0E0F0E0CF010895A7E8B8E3ED91FC9110
:100EB0001197858781E0878782E08487828193818B
:100EC0008D939C9381E00E9480AF0C9475B9EF9252
:100ED000FF920F931F93CF93DF9300D01F92CDB754
:100EE000DEB78C014B835C8369837A830E942B87F6
:100EF000FC014B815C8169817A81009761F48EE00D
:100F00002496CDBFDEBFDF91CF911F910F91FF904F
:100F1000EF900C94695383E0858788EE95E884838D
:100F20009583068317838B017A0126E0D8014D91C2
:100F30005D916D917D918D01CF0185599F4FDC01B0
:100F40004D935D936D937C931397D7014D915D9174
:100F50006D917D917D01418B528B638B748B215000
:100F600034962111E3CF83E02496CDBFDEBFDF911D
:100F7000CF911F910F91FF90EF900C945487CF92D7
:100F8000DF92EF92FF926B017C010E942B8700970A
:100F900039F48EE0FF90EF90DF90CF900C9469537E
:100FA00022E438E8FC0124833583E556FF4FC082F4
:100FB000D182E282F38221E0FC01278782E00E9455
:100FC000548780E0FF90EF90DF90CF90089580915C
:100FD000893890918A38FC0124853EEF320F3230F7
:100FE00018F424E024870895243011F080E090E084
:100FF0000895E0918938F0918A3822813381808187
:1010000091814CEBDF011D924A95E9F722833383EE
:1010100080839183E0918938F0918A380280F3814E
:10102000E02DE0938938F0938A388485823011F47A
:1010300083E08487809184388F5F809384388FEF3A
:101040000E9480AF81E04091853850918638209190
:10105000893830918A384217530709F080E00895A3
:10106000BC016F5E7F4FDC011696ED91FC911797E6
:1010700085599F4F19950E94F98781110E94865AC0
:1010800080E0089585569F4F20E034E244E759E41C
:10109000FC0160817181828193810E94D3D90E9479
:1010A000A2D70E94CED70E9439BC0E94F987811135
:1010B0000E94865A80E008958091893890918A38FC
:1010C000FC0124853EEF320F323018F424E02487EF
:1010D0000895243011F080E090E00895CF93DF93DD
:1010E000C0918938D0918A388C859EEF980F9230C4
:1010F00018F484E08C8705C0843019F080E090E01B
:1011000010C02097D9F3DE011296ED91FC91139750
:101110008785882329F0EC17FD0711F0DF01F4CF54
:10112000CD01DF91CF910895CF93DF93EC012A8118
:101130003B81888199814CEBFB01DE0101900D928E
:101140004A95E1F72A833B8388839983DF91CF9186
:1011500008958FEE92E18093A2519093A3518093D2
:101160005F529093605208952F923F924F925F92F8
:101170006F927F928F929F92AF92BF92CF92DF92A7
:10118000EF92FF920F931F93CF93DF93CDB7DEB70C
:101190006A97CDBFDEBF4C011B0129013A01E986E8
:1011A000FA860B871C871A2D0B2DE8A8B9A8AAA8C8
:1011B0002BA9298380915A2C882399F080914E2C59
:1011C00090914F2CA091502CB091512CBC01CD018D
:1011D0009F772CEA35EC47E257E30E942ED787FD34
:1011E00011C78091852D9091862DA091872DB0916A
:1011F000882DBC01CD019F7731E03D832CEA35EC91
:1012000047E257E30E9431D9181614F01D8210C02E
:101210002DEC3CEC4CEC5DE360912A2D70912B2D74
:1012200080912C2D90912D2D0E942ED787FDECC6FC
:10123000F10180819181A281B381BC01CD019F77B1
:10124000F1E0FD872CEA35EC47E257E30E9431D903
:1012500018160CF01D86F10184819581A681B78155
:10126000BC01CD019F77F1E0F98B2CEA35EC47E228
:1012700057E30E9431D918160CF0198AF1018085C4
:101280009185A285B3852091892D30918A2D409139
:101290008B2D50918C2D2E8B3F8B488F598F209109
:1012A0008D2D30918E2D40918F2D5091902D2A8B28
:1012B0003B8B4C8B5D8B4091912D5091922D609189
:1012C000932D7091942DF0905B2CF11021C0109211
:1012D000EA5181E08093EB5182E08093EC513D81B3
:1012E000332341F04D85411195C65989511192C65C
:1012F0008CE9C1C6CB01BA019F772CEA35EC47E2F5
:1013000057E30E9431D918160CF089C68BE9B3C691
:10131000BC01CD019F77A1E0AA8F2CEA35EC47E212
:1013200057E30E9431D918160CF01A8EB1E0FB1267
:1013300016C01092EA5182E08093EB51F092EC518A
:10134000ED81EE2339F0FD85F11164C62A8D22234B
:1013500079F260C66A897B898C899D89CDCF32E01C
:10136000F31217C081E08093EA51F092EB51109292
:10137000EC514D81442341F0598951114BC68A8D5E
:10138000882309F4B5CF46C66E897F89888D998DEB
:10139000B3CFB101C4010E9483519D81992309F407
:1013A00051C02091162C3091172C4091182C50913F
:1013B000192C60916B2C70916C2C80916D2C9091FC
:1013C0006E2C0E9485D59F772CEA35EC47E257E3D7
:1013D0000E942ED787FF36C020911A2C30911B2CEB
:1013E00040911C2C50911D2C60916F2C7091702C91
:1013F0008091712C9091722C0E9485D59F772CEA58
:1014000035EC47E257E30E942ED787FF1BC020919F
:101410001E2C30911F2C4091202C5091212C60913A
:10142000732C7091742C8091752C9091762C0E9465
:1014300085D59F772CEA35EC47E257E30E942ED7FB
:1014400087FDE4C58CA98093152C81E19CE20E9464
:101450008B4F86E5E1E1FCE2A9E0B2E501900D9257
:101460008A95E1F788E1EBE6FCE2A5EAB1E50190B7
:101470000D928A95E1F780915C2C8111D5C523E30B
:1014800033E34BEC51E46E2D7B2D8A2D99810E9424
:10149000D3D94B015C016093D5517093D6518093A1
:1014A000D7519093D85123E333E34BEC51E4C3017C
:1014B000B2010E94D3D96093BD517093BE51809305
:1014C000BF519093C05123E333E34BEC51E4698562
:1014D0007A858B859C850E94D3D96093C151709386
:1014E000C2518093C3519093C45123E333E34BEC37
:1014F00051E4612F702FC6010E94D3D9162F072FF8
:10150000412F502FBC014093C5515093C651609359
:10151000C7517093C8518091262D9091272DA0918D
:10152000282DB091292DBC01CD019F770E940BD8A9
:101530000E94A2D76093E6517093E7518093E851DF
:101540009093E951A091EA51A98BB091EB51BA8BDC
:10155000EB2FF0E0ED83FE837F01EE0CFF1CEE0C21
:10156000FF1CF101EE0DFF1D80819181A281B381ED
:10157000BC01CD019F772CEA35EC47E257E30E948E
:101580002ED7D82EDD1CDD24DD1C3989232F30E039
:1015900029833A838901000F111F000F111FF101E8
:1015A000E00FF11F80819181A281B381BC01CD0147
:1015B0009F772CEA35EC47E257E30E942ED7881F2D
:1015C0008827881F8D218093E5512CEA35EC47E26E
:1015D00057E3C501B4019F770E9431D918160CF06A
:1015E000F9C0F801EA5EF34DD801A559B34D2D912C
:1015F0003D914D915C9160817181828193810E94C6
:1016000085D56B017C01ED81FE81EE0FFF1FEE0F92
:10161000FF1FEA5EF34DAD81BE81AA0FBB1FAA0F6B
:10162000BB1FA559B34D2D913D914D915C916081AA
:101630007181828193810E9485D569877A878B87A2
:101640009C87A5019401C501B4010E94D3D920E073
:1016500030E040E850E40E94D3D96D877E878F87C1
:10166000988BA7019601C701B6010E94D3D92B011F
:101670003C0129853A854B855C85CA01B9010E94E8
:10168000D3D99B01AC01C301B2010E9486D59B0155
:10169000AC016D857E858F8598890E9485D52B014B
:1016A0003C0120E030E0A9010E9431D91816C4F4B1
:1016B000C301B2010E94ACDA2B013C0129853A85B5
:1016C0004B855C85C701B6010E943ED99B01AC01E8
:1016D000C301B20190580E9435D72B013C0103C0D1
:1016E000412C512C32018091152C833021F477FA52
:1016F000709477F8709420E030E0A901C501B4013E
:101700000E942ED787FF04C077FA709477F8709400
:1017100009811A81000F111F000F111FA8014E55DA
:101720005E4A5A01A301920169857A858B859C8561
:101730000E94D3D99B01AC01C701B6010E9485D597
:1017400020E030E040E05FE30E94D3D9D5015B9612
:101750006D937D938D939C935E97AD80BE80AA0C14
:10176000BB1CAA0CBB1CF501EE55FE4A4F01A301A0
:101770009201C701B6010E94D3D99B01AC016985D2
:101780007A858B859C850E9486D520E030E040E0FC
:101790005FE30E94D3D9D4015B966D937D938D93C3
:1017A0009C935E97E091EC51F0E0EE0FFF1FEE0F7F
:1017B000FF1FEE55FE4A138E148E158E168EB091B5
:1017C000D551B987E091D651ED872090D75130900F
:1017D000D85125C05701F701EE55FE4A838D948DEF
:1017E000A58DB68D9C01AD015058F801EE55FE4A0D
:1017F000838D948DA58DB68DBC01CD0190580E942E
:101800003ED99B01AB01BC014093D5515093D651B9
:101810006093D7517093D85129873D871C01D80117
:10182000AE55BE4A5B96CD90DD90ED90FC905E97F4
:10183000E981FA81EE0FFF1FEE0FFF1FE25FFD4A05
:1018400013962D913D914D915C9116976081718118
:10185000828193810E9485D5A70196010E9485D53A
:1018600069837A838B839C83D501AE55BE4A5B9690
:101870004D905D906D907C905E97ED81FE81EE0FB6
:10188000FF1FEE0FFF1FE25FFD4A13962D913D9162
:101890004D915C91169760817181828193810E9444
:1018A00085D5A30192010E9485D56D837E838F83A8
:1018B00098879B01AC0169817A818B819C810E9410
:1018C0003ED929853D85A1010E9485D54B015C014A
:1018D000E894B7F820E030E040E85FE3C501B401E8
:1018E0000E9431D918160CF4C3C32AE037ED43EA3D
:1018F0005BE3C501B4010E942ED787FF12C02FE61B
:1019000032E143E85AE369857D85C1010E94D3D95C
:101910009B01AC01C501B4010E9431D918160CF429
:10192000A7C3A30192015058C701B60190580E9465
:10193000F9D54B015C016093CD517093CE518093EA
:10194000CF519093D05180915B2C813039F4412C50
:10195000512C30E8632E3FEB732E06C0412C512CE6
:1019600020E8622E2FE3722E8091E5518823D1F179
:101970006091E6517091E7518091E8519091E95161
:101980000E94CED76B017C012CEA35EC47E257E38D
:101990000E942ED787FD10C01091152C2BED3FE033
:1019A00049EC50E4C701B6010E94D3D99B01AC01B8
:1019B000C12CD12C7601B9C081E090E0A0E0B0E06C
:1019C0008093E6519093E751A093E851B093E95189
:1019D0001091152C2BED3FE049EC50E4C12CD12C9B
:1019E0007601A3C02D813E814F81588569817A811E
:1019F0008B819C810E94F9D569837A838B839C8338
:101A00006093D1517093D2518093D3519093D4511C
:101A1000A50194010E9485D56B017C019F772CEA7A
:101A200035EC47E257E30E942ED787FF18C010918C
:101A3000152C6091E6517091E7518091E851909199
:101A4000E9510E94CED72BED3FE049EC50E40E94D3
:101A5000D3D99B01AC01C12CD12C760166C0298160
:101A60003A814B815C81C501B4010E9431D91816BD
:101A7000F4F42BED3FE049EC50E4C301B2010E94C5
:101A8000D3D99B01AC0169817A818B819C810E94B1
:101A900086D56093D1517093D2518093D351909356
:101AA000D451A50194010E9485D56B017C01109150
:101AB000152C133099F06091E6517091E7518091A7
:101AC000E8519091E9510E94CED72BED3FE049ECCF
:101AD00050E40E94D3D99B01AC0127C02BED3FE01D
:101AE00049EC50E4C301B2010E94D3D99B01AC017F
:101AF000C701B6010E9485D57B018C016091E6513A
:101B00007091E7518091E8519091E9510E94CED7B0
:101B10002BED3FE049EC50E40E94D3D99B01AC018E
:101B2000C701D8016C017D010BC0123049F4C3011B
:101B3000B2010E94D3D9A70196010E9486D50AC09E
:101B4000C301B2010E94D3D99B01AC01C701B60108
:101B50000E9485D57B01AB01BC014093D9515093C4
:101B6000DA516093DB517093DC518C015090EC5151
:101B7000A52DB0E0FD01EE0FFF1FEE0FFF1FE25F8E
:101B8000FD4AAA0FBB1FAA0FBB1FAE55BE4A139634
:101B90002D913D914D915C9116976081718182816B
:101BA00093810E9485D54B015C016093DD51709358
:101BB000DE518093DF519093E0519701A801698530
:101BC0007D85C1010E94D3D96B017C016093E151F5
:101BD0007093E2518093E3519093E451A5019401F5
:101BE0000E943ED969837A838B839C836093C95119
:101BF0007093CA518093CB519093CC5180915A2CC1
:101C0000811117C0F0914E2CFD8340904F2C2091F4
